:100000000C9460180C9499180C9499180C949918E5
:100010000C94878B0C94878B0C94878B0C94878B18
:100020000C9499180C9499180C9499180C9499188C
:100030000C9499180C94EF720C9499180C949918CC
:100040000C9499180C9420710C945ACF0C94991814
:100050000C94C4400C94BA400C9499180C949918C0
:100060000C9499180C9499180C9499180C9499184C
:100070000C9499180C9499180C9499180C9499183C
:100080000C947E330C9499180C94991805A84CCDB7
:10009000B2D44EB93836A9020C50B9918688083CC2
:1000A000A6AAAA2ABE000000803F4E414E494E49F2
:1000B0005459494E46CDCCCC3D0AD7233C17B7D135
:1000C0003877CC2B329595E6241FB14F0A000020DB
:1000D000410000C84200401C4620BCBE4CCA1B0E5A
:1000E0005AAEC59D7400407A10F35A00A0724E18A3
:1000F000090010A5D4E80000E87648170000E40BDA
:1001000054020000CA9A3B000000E1F5050000809F
:10011000969800000040420F000000A086010000F9
:1001200000102700000000E8030000000064000049
:100130000000000A00000000000100000000002C88
:1001400076D888DC674F0823DFC1DFAE59E1B1B74D
:1001500096E5E3E453C63AE651997696E8E6C2841A
:1001600026EB898C9B62ED407C6FFCEFBC9C9F4032
:10017000F2BAA56FA5F490055A2AF75C936B6CF957
:10018000676DC11BFCE0E40D47FEF520E6B500D02D
:10019000ED902E0300943577050080841E08000042
:1001A000204E0A000000C80C333333330F986E1210
:1001B000831141EF8D2114893BE65516CFFEE6DB16
:1001C00018D1844B381BF77C1D901DA4BBE4242060
:1001D0003284725E228100C9F124ECA1E53D2743FF
:1001E0004F4D4D554E49434154494F4E004452598D
:1001F00052554E004552524F525300494E464F0001
:100200004543484F0053544F505045442E20005012
:1002100072696E7465722073746F707065642064A7
:10022000756520746F206572726F72732E20466937
:100230007820746865206572726F7220616E642028
:10024000757365204D39393920746F207265737468
:100250006172742E202854656D70657261747572B8
:10026000652069732072657365742E205365742050
:10027000697420616674657220726573746172744A
:10028000696E67290A004E6F20436865636B73755A
:100290006D2077697468206C696E65206E756D627B
:1002A00065722C204C617374204C696E653A200095
:1002B0004E6F20436865636B73756D207769746852
:1002C000206C696E65206E756D6265722C204C61C4
:1002D0007374204C696E653A2000636865636B73C4
:1002E000756D206D69736D617463682C204C61734A
:1002F00074204C696E653A20004C696E65204E751D
:100300006D626572206973206E6F74204C61737426
:10031000204C696E65204E756D6265722B312C2004
:100320004C617374204C696E653A20004D31313058
:100330000053657269616C20737461747573206D0C
:1003400069736D617463680A005344207265616467
:10035000206572726F720A002121204B494C4C209B
:1003600063617573656420627920746F6F206D75A9
:10037000636820696E6163746976652074696D6570
:10038000202D2063757272656E7420636F6D6D61D0
:100390006E643A20004D3235004D65646961204934
:1003A0006E73657274656400627573793A2070616A
:1003B0007573656420666F7220696E7075740A00CB
:1003C000627573793A2070617573656420666F7227
:1003D00020757365720A00627573793A2070726FC6
:1003E00063657373696E670A00506C65617365209D
:1003F0005265736574005052494E5445522048412D
:100400004C5445440025533A202553004B494C4C4D
:1004100045442E20005072696E7465722068616CCC
:100420007465642E206B696C6C28292063616C6C88
:100430006564210A0053544F505045442E2000500B
:1004400072696E7465722073746F70706564206475
:10045000756520746F206572726F72732E20466905
:100460007820746865206572726F7220616E6420F6
:10047000757365204D39393920746F207265737436
:100480006172742E202854656D7065726174757286
:10049000652069732072657365742E20536574201E
:1004A0006974206166746572207265737461727418
:1004B000696E67290A006563686F3A004572726F5A
:1004C000723A0042696C696E656172204C657665AE
:1004D0006C696E6720477269643A0A0021212053D3
:1004E000544F502063616C6C656420626563617574
:1004F0007365206F6620424C546F75636820657287
:10050000726F72202D207265737461727420776926
:100510007468204D3939390A0021212053544F5035
:100520002063616C6C65642062656361757365202E
:100530006F6620424C546F756368206572726F72EB
:10054000202D20726573746172742077697468203D
:100550004D3939390A0050726F62696E6720506FE9
:10056000696E740025532025692F2569002E0A0025
:100570002F0050726F62696E67206D65736820701E
:100580006F696E742000202844525952554E29003C
:10059000473239204175746F20426564204C65767E
:1005A000656C696E67003F20284C2C522C462C420B
:1005B00029206F7574206F6620626F756E64732ECC
:1005C0000A003F2856296572626F7365206C657654
:1005D000656C20696D706C61757369626C6520284B
:1005E000302D34292E0A00426164205A2076616C35
:1005F00075650A004E6F2062696C696E65617220D4
:10060000677269640A004732384C30004465766985
:100610006174696F6E0025533A2025730046696E38
:100620006973686564210A003A207A3A2000206FD5
:10063000662000476F696E6720746F3A2058004348
:10064000570A00206469723A0020616E676C653A4F
:10065000005374617274207261646975733A004D5D
:10066000343820506F696E740025533A2025642F6A
:10067000256400506F736974696F6E696E672074CA
:1006800068652070726F62652E2E2E0A003F4C65E1
:100690006773206F66206D6F76656D656E74206977
:1006A0006D706C61757369626C652028302D313511
:1006B000292E0A003F2028582C5929206F757420B4
:1006C0006F6620626F756E64732E0A0050726F62DF
:1006D00065206F7574206F6620626F756E6473009D
:1006E0003F53616D706C652073697A65206E6F741D
:1006F00020706C61757369626C652028342D35300B
:10070000292E0A004D3438205A2D50726F62652010
:100710005265706561746162696C697479205465B1
:1007200073740A003F2856296572626F7365206CE6
:100730006576656C20696D706C61757369626C6556
:100740002028302D34292E0A005374616E646172A2
:100750006420446576696174696F6E3A20002052A6
:10076000616E67653A2000204D61783A2000204D87
:10077000696E3A2000205369676D613A20004D652B
:10078000616E3A200020204D3230312058004D61FA
:100790007820416363656C65726174696F6E2028AF
:1007A000756E6974732F7332290020204D323033F7
:1007B0002058004D617820666565647261746573C8
:1007C0002028756E6974732F732900205200202031
:1007D0004D323034205000416363656C6572617442
:1007E000696F6E2028756E6974732F733229202803
:1007F000503C7072696E742D616363656C3E20526B
:100800003C726574726163742D616363656C3E2034
:10081000543C74726176656C2D616363656C3E292E
:1008200000204A0020540020530020204D32303553
:10083000204200416476616E6365642028423C6D0D
:10084000696E5F7365676D656E745F74696D655F12
:1008500075733E20533C6D696E5F666565647261B9
:1008600074653E20543C6D696E5F74726176656C90
:100870005F66656564726174653E204A3C6A756EA8
:10088000635F6465763E29002044002049002020F3
:100890004D333031205000486F74656E64205049EC
:1008A00044002E0A00206E6F742064697361626CCC
:1008B00065642E20536861726564207769746800EE
:1008C000203B204C6576656C696E67200020204DCA
:1008D0003432302053004175746F20426564204CDF
:1008E0006576656C696E6700204600204800202010
:1008F0004D3134352053004D6174657269616C204F
:1009000068656174757020706172616D657465727F
:100910007300203B2053656E736F722000204400EB
:1009200020204D34313220530046696C616D656E74
:10093000742072756E6F75742073656E736F7200BC
:10094000204A002020473239205720490020204DDE
:100950003134392043203B20556E69747320696E11
:100960002043656C736975730A0054656D70657218
:10097000617475726520556E69747300202047326A
:1009800031203B004C696E65617220556E6974734D
:100990000020496E76616C696420657874727564B4
:1009A00065722000536C6565702E2E2E005A205003
:1009B000726F62652050617374204265640A005A48
:1009C0002050726F6265205061737420426564002C
:1009D000205A3A200020593A200042656420583AB3
:1009E00020004D65736820706F696E74206F757498
:1009F000206F662072616E67650A00436C69636BE5
:100A000020746F20526573756D652E2E2E00616CFB
:100A1000736F20656E61626C6564290A004E6F20F9
:100A20004D6F76652E004E6F206D656469610A001A
:100A3000456E642066696C65206C6973740A0042B7
:100A40006567696E2066696C65206C6973740A005D
:100A5000286E6F2066696C6529004E6F74205344C0
:100A6000207072696E74696E670A00534420707258
:100A7000696E74696E6720627974652000437572CF
:100A800072656E742066696C653A20002E0A004417
:100A9000656C6574696F6E206661696C65642C2095
:100AA00046696C653A200046696C652064656C6532
:100AB0007465643A002569730025696D20256973A2
:100AC000002569682025696D202569730025696402
:100AD000202569682025696D2025697300256979BD
:100AE00020256964202569682025696D20256973A2
:100AF000005072696E742074696D653A20006F6BE6
:100B0000006F6666000002FB01F401ED01DF0144A5
:100B1000454255473A004D3131322053687574646F
:100B20006F776E004D3131332053004D6567612082
:100B30005A65726F204F46462E00434F4E46494736
:100B40005F4558504F5254004D4541545041434B1E
:100B500000434F4F4C45525F54454D504552415410
:100B6000555245004348414D4245525F54454D5012
:100B70004552415455524500424142595354455003
:100B800050494E470041524353004D4F54494F4E38
:100B90005F4D4F44455300544845524D414C5F50C2
:100BA000524F54454354494F4E00455854454E44C6
:100BB00045445F4D3230004C4F4E475F46494C45EF
:100BC0004E414D45004155544F5245504F52545F90
:100BD00053445F5354415455530053445F57524953
:100BE00054450052455045415400534443415244FA
:100BF0000050524F4D50545F535550504F52540077
:100C0000484F53545F414354494F4E5F434F4D4DFE
:100C1000414E445300454D455247454E43595F5060
:100C2000415253455200434153455F4C4947485454
:100C30005F4252494748544E45535300544F47472B
:100C40004C455F4C494748545300534F4654574115
:100C500052455F504F574552004255494C445F50F2
:100C6000455243454E54004C4556454C494E475F0E
:100C700044415441005A5F50524F42450052554E34
:100C80004F5554004155544F4C4556454C00505219
:100C9000494E545F4A4F420050524F4752455353BA
:100CA000004155544F5245504F52545F54454D509A
:100CB000004155544F5245504F52545F504F5300CE
:100CC000564F4C554D455452494300454550524F9F
:100CD0004D0042494E4152595F46494C455F54527E
:100CE000414E534645520053455249414C5F584F7F
:100CF0004E5F584F4646004649524D574152455F58
:100D00004E414D453A4D61726C696E20322E302E47
:100D1000392E332D6B6164312028446563203237CE
:100D200020323032312031333A34383A32352920CA
:100D3000534F555243455F434F44455F55524C3ADC
:100D40006769746875622E636F6D2F6B61642F4DD8
:100D500061726C696E2050524F544F434F4C5F5636
:100D6000455253494F4E3A312E30204D4143484968
:100D70004E455F545950453A4D656761205A65723A
:100D80006F2045585452554445525F434F554E5479
:100D90003A3120555549443A646266636364353597
:100DA0002D656262612D343631352D616264372DD7
:100DB0003139366161343338663330340A002F2FCD
:100DC000004D31343520533C696E6465783E206FA8
:100DD0007574206F662072616E67652028302D3132
:100DE000290A003F4A206F7574206F662072616E79
:100DF00067652028302E303120746F20302E332943
:100E00000A0020580020204D61783A200020002060
:100E1000204D696E3A2000203B200020204D3231C9
:100E20003120530046523A0020466C6F773A20003A
:100E3000206F7574206F662072616E67650A0053BB
:100E40006572766F20003A200020536572766F201D
:100E50000050726F6265204F6666736574205A0099
:100E600050726F6265204F6666736574205A006425
:100E7000697300656E0043290A0061626C65642035
:100E8000286D696E2074656D702000436F6C64205E
:100E900065787472756465732061726520004F46D1
:100EA00046004F4E006D6D00203B20446973746115
:100EB0006E6365200046696C616D656E74207275A5
:100EC0006E6F757420004F46460A004661646520C7
:100ED0004865696768742000426564204C657665E2
:100EE0006C696E6720004661696C656420746F20D0
:100EF000656E61626C6520426564204C6576656C48
:100F0000696E670A00496E76616C6964206D65736D
:100F1000682E0A004D34323120696E636F7272653B
:100F2000637420706172616D6574657220757361A0
:100F300067650A004D65736820706F696E74206F75
:100F40007574206F662072616E67650A00454550B2
:100F5000524F4D204F4B0A00290A0020746F200089
:100F60003F5A206F7574206F662072616E6765202E
:100F70002800290A0020746F20003F59206F7574E3
:100F8000206F662072616E676520282D00290A0097
:100F900020746F20003F58206F7574206F66207298
:100FA000616E676520282D004D383400446F6E65F2
:100FB000207072696E74696E672066696C650A00DC
:100FC0004D3737004D333100496E76616C696420CE
:100FD00065787472756465720A004361703A002026
:100FE000286D6D2900203B0020204D3835312058D8
:100FF000005A2D50726F6265204F666673657400EB
:10100000436F6F6C696E672E2E2E004865617469A0
:101010006E672E2E2E0045312025530020573A00B2
:1010200023646566696E652044454641554C545FAE
:10103000004B6420004B6920004B70200050494455
:10104000204175746F74756E652066696E6973688A
:101050006564212050757420746865206C61737418
:10106000204B702C204B6920616E64204B64206300
:101070006F6E7374616E74732066726F6D2062653B
:101080006C6F7720696E746F20436F6E6669677549
:10109000726174696F6E2E680A0050494420417570
:1010A000746F74756E65206661696C656421207467
:1010B000696D656F75740A00504944204175746FFD
:1010C00074756E65206661696C6564212054656D78
:1010D000706572617475726520746F6F20686967DE
:1010E000680A00504944204379636C6573002553B6
:1010F0002025692F256900204B643A2000204B6988
:101100003A2000204B703A200020436C61737369D1
:101110006320504944200A002054753A2000204B97
:10112000753A2000206D61783A2000206D696E3A92
:10113000200020643A200020626961733A20005741
:1011400061697420666F7220686561742075702E05
:101150002E2E00504944204175746F74756E6520C1
:1011600073746172740A00504944204175746F743D
:10117000756E65206661696C6564212054656D70CB
:101180006572617475726520746F6F206869676835
:101190000A00504944204175746F74756E6520666D
:1011A00061696C65642120426164206865617465D1
:1011B000722069640A00504944204175746F747547
:1011C0006E65004572723A207574663820666F6EDF
:1011D00074206E6F7420696E697469616C697A65D8
:1011E000642E004572723A207574663820666F6E00
:1011F00074206E6F7420696E697469616C697A65B8
:10120000642E004572723A207574663820666F6EDF
:1012100074206E6F7420696E697469616C697A6597
:10122000642E002568753A25303268750025303205
:1012300068753A2530326875002530326875272583
:101240003032687500256875642025303268753A3B
:1012500025303268750042656400456E636C6F73BB
:1012600075726500202020202020200020202020D2
:1012700000453A00523A00657272001FE0201020CB
:1012800010201010201020201020103030084004B2
:101290008003001FE03FF03FF03FF01FE01FE03F02
:1012A000F03FF03FF00FC0078003003FFFF0380031
:1012B0007030FC3020FC102078102030102C00D032
:1012C0002E31D02F7BD02F7BD02E31D02C00D020B0
:1012D000301020781020FC1030FC303800703FFFB8
:1012E000F03FFFF038007031863023871027879059
:1012F0002F87D02F03D02030102078102078102096
:1013000030102F03D02F87D0278790238710318666
:10131000303800703FFFF0001DC43F0000000C8615
:10132000198000000D0E198000000F0B19800000BD
:101330000D9F198000000DD3998000001CFBFF0059
:1013400000000000000000000000000000F380002A
:101350001F80007700001980005B1CF6131DAE5B38
:1013600035AB0635FB5B3DA70CBD9B4B30EB19B194
:101370009BE39D8E9F9D8E0001E0000000000120F8
:101380000000000001E0000000000C0F00FE07025A
:101390002503BB017FFE08FE08FE050808060000C5
:1013A00040F0C88888987810050808060000C0F842
:1013B0008888888888F80505050600012030F830FF
:1013C000200508080600002070F820202020E005F5
:1013D00009090600FF2070A8A8B8888870200705B2
:1013E00005070001D86C366CD80509090600FFF81E
:1013F000A88888888888A8F8050A0A0600FE205070
:1014000050505088A8A8887003030306000340A02A
:1014100040FFFFFFFFFFFFFFFFFFFFFFFFFFFFFF9B
:10142000FFFFFFFFFFFFFF0000000605FF010707AA
:10143000060200808080808000800303030601058F
:10144000A0A0A005060606000050F85050F8500570
:1014500009090600FF2070A8A07028A870200507C1
:1014600007060000C8C81020409898050707060026
:101470000040A0A040A890680103030602058080F8
:10148000800309090601FF20404080808040402001
:101490000309090601FF80404020202040408005CC
:1014A000070706000020A8702070A8200505050683
:1014B00000012020F820200203030601FFC0408025
:1014C000050101060003F8020202060100C0C00582
:1014D0000707060000081010204040800507070697
:1014E0000000708898A8C8887003070706010040AC
:1014F000C040404040E00507070600007088081023
:101500002040F8050707060000F80810300888702A
:1015100005070706000010305090F8101005070767
:10152000060000F880F0080888700507070600002C
:10153000304080F0888870050707060000F8081022
:101540001020202005070706000070888870888812
:10155000700507070600007088887808106002058B
:1015600005060100C0C000C0C00206060601FFC09B
:10157000C000C040800305050601012040804020D6
:10158000050303060002F800F803050506010180C3
:1015900040204080050707060000708810202000CA
:1015A000200507070600007088B8A8B880700507F6
:1015B00007060000708888F88888880507070600F5
:1015C00000F04848704848F005070706000070889A
:1015D0008080808870050707060000F0484848486A
:1015E00048F0050707060000F88080F08080F805C5
:1015F0000707060000F88080F08080800507070656
:1016000000007088808098887005070706000088B1
:101610008888F8888888030707060100E040404072
:101620004040E005070706000038101010109060D9
:101630000507070600008890A0C0A090880507074E
:10164000060000808080808080F805070706000083
:1016500088D8A8888888880507070600008888C871
:10166000A8988888050707060000708888888888F9
:1016700070050707060000F08888F0808080050765
:101680000706000070888888A8906805070706008C
:1016900000F08888F0A09088050707060000708891
:1016A0008070088870050707060000F820202020B9
:1016B000202005070706000088888888888870052C
:1016C000070706000088888888505020050707060D
:1016D000000088888888A8A85005070706000088A9
:1016E0008850205088880507070600008888502009
:1016F000202020050707060000F80810204080F889
:101700000309090601FFE080808080808080E00579
:101710000707060000804040201010080309090652
:1017200001FFE020202020202020E0050303060008
:10173000052050880501010600FEF8030303060199
:1017400005804020050505060000700878887805AA
:1017500007070600008080F0888888F005050506E8
:101760000000708080887005070706000008087870
:10177000888888780505050600007088F080700567
:101780000707060000304840E040404005070706D4
:1017900000FE7088888878087005070706000080BA
:1017A00080F0888888880307070601004000C04051
:1017B0004040E00409090601FE100030101010102E
:1017C000906005070706000080808890E0908803FD
:1017D0000707060100C04040404040E005050506FF
:1017E0000000D0A8A8A8A8050505060000B0C88874
:1017F0008888050505060000708888887005070739
:101800000600FEF0888888F080800507070600FE45
:1018100078888888780808050505060000B0C88023
:10182000808005050506000078807008F005070730
:101830000600002020F820202018050505060000DD
:1018400088888898680505050600008888885020E3
:101850000505050600008888A8A8500505050600AE
:101860000088502050880507070600FE88888850A9
:10187000204080050505060000F8102040F8030907
:10188000090601FF204040408040404020010909F6
:101890000602FF80808080808080808003090906A6
:1018A00001FF804040402040404080050303060087
:1018B0000248A890FF5045544700504C41005072D8
:1018C000696E742041626F72746564004D32350038
:1018D00050617573696E672E2E2E004D32340045AF
:1018E0004550524F4D2056657273696F6E20457298
:1018F000726F7200454550524F4D20496E646578B5
:10190000204572726F7200454550524F4D20435230
:1019100043204572726F72003F0049676E6F7265B7
:1019200000526573657400496E697469616C697A07
:101930006520454550524F4D0000FE0003FF8007D3
:10194000C7C00701E00000E00000F00000700400E4
:10195000700E00701F00703F80F00E00E00F01E07D
:1019600007C7C003FF8000FE0000FE0003FF8007E2
:10197000C7C00F01E00E00E03F80F01F00700E00B6
:10198000700400700000700000F00000E00701E04B
:1019900007C7C003FF8000FE000E000E000E000E01
:1019A000000E000E000E000E007FC03F801F000ED4
:1019B00000040004000E001F003F807FC00E000ED8
:1019C000000E000E000E000E000E000E00FFFFFFC6
:1019D0007F80FFC0FFC0FFC07F807F80FFC0FFC04F
:1019E000FFC03F001E000C0050726F6265205A203D
:1019F0004F6666736574002008204661637400209A
:101A000008204D6178002008204D696E004F666601
:101A1000004F6E004175746F74656D7000452073E2
:101A2000746570732F6D6D005A2053746570732F39
:101A30006D6D00592053746570732F6D6D005820C3
:101A400053746570732F6D6D00416476616E6365CC
:101A5000642053657474696E67730054656D7065B6
:101A60007261747572650053746570732F6D6D00CB
:101A7000436F6E66696775726174696F6E003F00CF
:101A80004E65787420436F726E657200446F6E65A8
:101A9000004E65787400486F6D696E672058595A1A
:101AA0000053746F72652053657474696E677300B8
:101AB0004C6F61642053657474696E67730042658E
:101AC00064205472616D6D696E670050726F62655B
:101AD000205A204F6666736574004661646520482D
:101AE0006569676874004F6666004F6E0042656402
:101AF000204C6576656C696E67004C6576656C2078
:101B0000426564004732394E0047323900417574EE
:101B10006F20486F6D65004D6F74696F6E0053578D
:101B20002D4D6F64650053746F77004465706C6F62
:101B3000790053656C662D54657374005265736546
:101B40007400436F6E66696775726174696F6E00C9
:101B5000526573746F72652044656661756C747349
:101B6000004C6F61642053657474696E6773005331
:101B7000746F72652053657474696E6773004F6685
:101B800066004F6E0052756E6F75742053656E73EC
:101B90006F7200424C546F7563680050726F6265DB
:101BA000205A204F666673657400416476616E63E7
:101BB00065642053657474696E6773004D61696E66
:101BC000003F004261636B0053746F70004D32320E
:101BD00000417474616368204D65646961004D3231
:101BE00031005072696E742066726F6D204D6564AD
:101BF00069610052656C65617365204D656469615A
:101C000000436F6E66696775726174696F6E005428
:101C1000656D7065726174757265004D6F74696F82
:101C20006E00526573756D65205072696E74005454
:101C3000756E650053746F70205072696E74005039
:101C400061757365205072696E7400496E666F200D
:101C500053637265656E000A4D3234004D32332095
:101C60002573003F005374617274205072696E7462
:101C70000043616E63656C005072696E740043616D
:101C80006E6E6F7420656E74657220737562646920
:101C9000723A200002202E2E000152656672657392
:101CA00068004D61696E002100486F74656E6420A4
:101CB000746F6F20636F6C64004261636B005072DD
:101CC0006F63656564004D6F74696F6E004469737E
:101CD00061626C65205374657070657273004D3875
:101CE00034004D34382050726F626520546573742F
:101CF000004732384F0A4D343820503130004265A9
:101D000064204C6576656C696E67004175746F2060
:101D1000486F6D6500473238004D61696E00BA1832
:101D2000B518436F6F6C646F776E005072656865AD
:101D3000617420240046616E205370656564004E16
:101D40006F7A7A6C65004D61696E0050726F6265E2
:101D5000205A204F666673657400466C6F770046A4
:101D6000616E205370656564004E6F7A7A6C650011
:101D70005370656564004D61696E00486F6D696EF2
:101D800067204661696C6564006F70656E0054522F
:101D900049474745524544003A200066696C616DE9
:101DA000656E74007A5F6D696E00795F6D696E00B3
:101DB000785F6D696E005265706F7274696E67202E
:101DC000656E6473746F70207374617475730A0048
:101DD00020746F6F206C6F6E6720657874727573F6
:101DE000696F6E2070726576656E7465640A002096
:101DF000636F6C6420657874727573696F6E2070A0
:101E0000726576656E7465640A00486F6D6520259D
:101E10007325732573204669727374005761726E5F
:101E2000696E673A20486F6D696E672042756D7004
:101E30002044697669736F72203C20310A000202E7
:101E4000040000E0C0000000C000000000000068C6
:101E5000430000634300007A430000A0400000A05C
:101E60004000000040FFFDFCFAF8F6F4F2F0EEEC62
:101E7000EAE9E7E5E3E1E0DEDCDAD9D7D5D4D2D090
:101E8000CFCDCBCAC8C7C5C3C2C0BFBDBCBAB9B726
:101E9000B6B4B3B2B0AFADACAAA9A8A6A5A4A2A18E
:101EA000A09E9D9C9A99989795949392908F8E8DD1
:101EB0008B8A8988878684838281807F7E7D7B7AF6
:101EC000797877767574737271706F6E6D6C6B6AFA
:101ED000696867666564636261605F5E5D5C5B5AEA
:101EE0005958585756555453525150504F4E4D4CC7
:101EF0004B4A4A4948474646454443424241403F8F
:101F00003E3E3D3C3B3B3A39383837363535343345
:101F100032323130302F2E2E2D2C2B2B2A292928EE
:101F2000272726252524232322212120201F1E1E8A
:101F30001D1C1C1B1B1A1919181817161615151419
:101F4000131312121111100F0F0E0E0D0D0C0C0B9E
:101F50000A0A090908080707060605050404030319
:101F600002020100000000000100000001000080EA
:101F700000555555000000400033333300AAAA2A0B
:101F8000004992240000002000C7711C0099991993
:101F900000D1451700555515003BB11300244912D7
:101FA0000011111100000010000F0F0F00E3380E98
:101FB0000043790D00CCCC0C00C3300C00E8A20B20
:101FC0000064210B00AAAA0A00703D0A009DD809EE
:101FD00000427B090092240900DCD30800888808AD
:101FE000001042080000000800F0C10700878707C2
:101FF0000075500700711C07003EEB0600A1BC06EF
:10200000006990060066660600703E0600611806CC
:102010000017F4050074D105005BB00500B290050F
:1020200000627205005555050078390500B81E0597
:1020300000050505004EEC040087D40400A1BD0492
:102040000090A7040049920400C17D0400EE6904D9
:1020500000C7560400444404005C32040008210414
:102060000041100400000004003FF00300F8E0030A
:102070000026D20300C3C30300CCB503003AA80373
:10208000000A9B0300388E0300C08103009F750384
:1020900000D0690300505E03001D53030034480361
:1020A00000913D03003333030016290300381F035A
:1020B0000097150300300C0300030303000BFA0222
:1020C0000049F10200BAE802005CE002002DD802EB
:1020D000002DD0020059C80200B0C0020031B90280
:1020E00000DAB10200AAAA0200A0A30200BC9C026E
:1020F00000FA9502005C8F0200DF880200828202F3
:1021000000457C02002776020027700200436A0225
:10211000007C640200D05E02003F590200C85302F6
:1021200000000061430000614300007A430000E0CA
:10213000C0000000C00000000053657474696E6741
:10214000732053746F726564000000FA430000FA54
:10215000430000A0400000C8410000A0420000A0D1
:10216000420000C8430080C043F4010000F40100B5
:1021700000640000008813000024F4D43050C38EA3
:1021800020C2A24017828B7011127A910D816CD9F6
:102190000AA861E108C7586607615143061E4B5DF6
:1021A00005C145A7041A411104093D98037139314D
:1021B000034036DB0265339102D4305402802E1D79
:1021C00002632CEE01752AC501B028A001102781F9
:1021D000018F2564012B244B01E0223401AC211F27
:1021E000018D200D01801FFC00841EED00971DDF76
:1021F00000B81CD200E61BC600201BBC00641AB24B
:1022000000B219A8000A19A0006A189900D1179104
:102210000040178B00B516840031167E00B3157987
:10222000003A157300C7146F0058146A00EE136665
:10223000008813630025135E00C7125B006C125701
:102240000015125400C111510070114F0021114BA3
:1022500000D61049008D104700461044000210427D
:1022600000C00F4000800F3E00420F3C00060F3BB5
:1022700000CB0E3800930E37005C0E3500270E346D
:1022800000F30D3200C10D3100900D3000600D2EB5
:1022900000320D2D00050D2C00D90C2B00AE0C29A1
:1022A00000850C29005C0C2700350C27000E0C263D
:1022B00000E80B2400C40B2400A00B23007D0B239B
:1022C000005A0B2100390B2100180B2000F80A1FBF
:1022D00000D90A1E00BB0A1E009D0A1D00800A1DAF
:1022E00000630A1C00470A1B002C0A1B00110A1A73
:1022F00000F7091A00DD091900C4091900AB091912
:1023000000920917007B091800630917004C091691
:102310000036091600200916000A091500F50815EF
:1023200000E0081400CC081400B8081400A4081435
:1023300000900813007D0812006B08130058081263
:102340000046081200340811002308110012081179
:102350000001081100F0071000E0071000D007107E
:1023600000C0071000B0070F00A107100091070E72
:102370000083070F0074070F0065070E0057070E54
:102380000049070E003B070D002E070E0020070D29
:102390000013070D0006070D00F9060C00ED060DF1
:1023A00000E0060C00D4060C00C8060C00BC060CAD
:1023B00000B0060C00A4060B0099060C008D060B5D
:1023C0000082060B0077060B006C060B0061060A04
:1023D0000057060B004C060A0042060A0038060A9F
:1023E000002E060A0024060A001A060A0010060932
:1023F0000007060A00FD050900F4050900EB0509C0
:1024000000E2050900D9050900D0050900C7050942
:1024100000BE050900B5050800AD050800A50509C1
:10242000009C050800940508008C05080084050838
:10243000007C050800740508006C050700650508A8
:10244000005D050700560508004E05070047050713
:10245000004005080038050700310507002A050778
:1024600000230507001C050600160507000F0507D9
:10247000000805060002050700FB040600F5040736
:1024800000EE040600E8040600E2040700DB040690
:1024900000D5040600CF040600C9040600C30406E4
:1024A00000BD040600B7040600B1040500AC040634
:1024B00000A6040600A00405009B04060095040580
:1024C00000900406008A04050085040500800406C7
:1024D000007A04050075040500700405006B04050E
:1024E0000066040500610405005C0405005704054E
:1024F00000520405004D040500480405004304058E
:10250000003E0404003A04050035040500300404CC
:10251000002C04050027040400230405001E040405
:10252000001A04040016040500110404000D04043C
:1025300000090405000404040000040400FC030472
:1025400000F8030400F4030400F0030400EC0304A7
:1025500000E8030400E4030400E0030400DC0304D7
:1025600000D8030400D4030400D0030400CC030407
:1025700000C8030300C503030024F404D9201BC4CE
:102580000C5C0E9804C4095F0265077101F405F93B
:1025900000FB04B30048048700C1036900580355D9
:1025A0000003034500BE023A008402310053022AB0
:1025B000002902250004022000E4011C00C80119C2
:1025C00000AF01170098011400840113007101107D
:1025D000006101100051010E0043010D0036010B96
:1025E000002B010B0020010B00150109000C010953
:1025F0000003010800FB000800F3000800EB0007DF
:1026000000E4000600DE000600D8000600D2000646
:1026100000CC000500C7000500C2000500BD000495
:1026200000B9000400B5000400B1000400AD0004CE
:1026300000A9000400A5000300A20003009F0004FD
:10264000009B000300980003009500020093000324
:1026500000900003008D0002008B00030088000240
:10266000008600020084000300810002007F000257
:10267000007D0002007B000200790002007700016B
:102680000076000200740002007200010071000276
:10269000006F0002006D0001006C0002006A000182
:1026A000006900020067000100660001006500018A
:1026B000006400020062000100610001006000018E
:1026C000005F0002005D0001005C0001005B000192
:1026D000005A000100590001005800010057000194
:1026E0000056000100550001005400010053000095
:1026F0000053000100520001005100010050000190
:10270000004F0001004E0000004E0001004D00018E
:10271000004C0001004B0000004B0001004A00018A
:102720000049000100480000004800010047000186
:102730000046000000460001004500000045000181
:10274000004400010043000000430001004200007B
:102750000042000100410000004100010040000172
:10276000003F0000003F0001003E0000003E00016D
:10277000003D0000003D0001003C0000003C000066
:10278000003C0001003B0000003B0001003A00005B
:10279000003A000100390000003900010038000053
:1027A0000038000000380001003700000037000149
:1027B0000036000000360000003600010035000041
:1027C0000035000000350001003400000034000036
:1027D000003400010033000000330000003300012A
:1027E0000032000000320000003200010031000021
:1027F0000031000000310001003000000030000016
:1028000000300001002F0000002F0000002F00000A
:10281000002F0001002E0000002E0000002E0001FD
:10282000002D0000002D0000002D0000002D0001F3
:10283000002C0000002C0000002C0000002C0001E7
:10284000002B0000002B0000002B0000002B0001DB
:10285000002A0000002A0000002A0000002A0001CF
:1028600000290000002900000029000000290000C4
:1028700000290001002800000028000000280000B6
:1028800000280000002800010027000000270000A9
:10289000002700000027000000270001002600009C
:1028A000002600000026000000260000002600018F
:1028B0000025000000250000002500000025000084
:1028C0000025000000250001002400000024000075
:1028D0000024000000240000002400010023000068
:1028E000002300000023000000230000002300005C
:1028F000002300000023000100220000002200004D
:10290000002200000022000000220000002200013E
:102910000021000000210000002100000021000033
:102920000021000000210000002100010020000023
:102930000020000000200000002000000020000017
:10294000002000000020000000200001001F000007
:10295000001F0000001F0000001F0000001F0000FB
:10296000001F0000001F0001001E0000001E0000EC
:10297000001E0000001E000000393000003325005A
:102980000087190000B00F0000DB080000BD040044
:1029900000740200003F01000020436F756E742038
:1029A000583A0045310045002C2073797374656DE9
:1029B0002073746F7070656421204865617465725E
:1029C0005F49443A200048656174696E672046613A
:1029D000696C65640048656174696E672066616949
:1029E0006C6564004572723A204D415854454D5013
:1029F000004D415854454D502074726967676572A7
:102A00006564004572723A204D494E54454D500060
:102A10004D494E54454D5020747269676765726523
:102A20006400202F0020403A007C3C3E5E2B3D3F5E
:102A30002F5B5D3B2C2A225C0043616E6E6F74201D
:102A40006F70656E20737562646972200053442054
:102A500063617264206F6B0A006F70656E526F6FF6
:102A600074206661696C65640A00766F6C756D65CB
:102A70002E696E6974206661696C65640A004E6F28
:102A800020534420636172640A002E0A006F70654F
:102A90006E206661696C65642C2046696C653A201D
:102AA0000046696C652073656C65637465640A0033
:102AB0002053697A653A200046696C65206F70651D
:102AC0006E65643A2000454E4420535542524F559E
:102AD00054494E450A002220706F73002220706115
:102AE00072656E743A2200535542524F5554494E06
:102AF000452043414C4C207461726765743A220052
:102B000053756263616C6C204F766572666C6F778B
:102B1000004578636565646564206D617820535570
:102B200042524F5554494E452064657074683A00CE
:102B3000667265736800646F696E67002066696C11
:102B4000653A20004E6F77200057726974696E678E
:102B500020746F2066696C653A20006D61726C6943
:102B60006E66772E6F726700322E302E392E332D1F
:102B70006B616431001FFFFFFFFFFFFF600000007B
:102B80000001FF400000000000FF80000000000086
:102B90007F83CF00000C303F87FF80000C301F8602
:102BA0007980000C000F8C30C7838C30E78C30CFDD
:102BB000C7CC31F38C30DCECEC33B98C30D86C6C96
:102BC00033198C30D06C0C33198C30D86C0C331911
:102BD0008C30DC6C0E3B198C30CF7C079F198C300D
:102BE000C77C038F19400000000000026000000055
:102BF0000000061FFFFFFFFFFFF870012C0190018E
:102C00002701B0012201C0011D01F00118011002CD
:102C1000130130020E016002090190020401C0029A
:102C2000FF000003FA004003F5008003F000D0032A
:102C3000EB002004E6007004E100E004DC00400545
:102C4000D700C005D2004006CD00D006C8008007DE
:102C5000C3003008BE00F008B900C009B400B00AD3
:102C6000AF00B00BAA00D00CA500000EA000500FC2
:102C70009B00C01096005012910000148C00C015EB
:102C80008700B0178200B0197D00D01B7800001EAD
:102C9000730040206E0090226900F02464004027F9
:102CA0005F0090295A00E02B5500102E5000203074
:102CB0004B0010324600E033410090353C001037A5
:102CC000370070383200A0392D00B03A2800A03B00
:102CD0002300603C1E00103D1900903D1400103E82
:102CE0000F00703E0A00C03E0500003F0000403F5C
:102CF000FBFF803FF6FFC03FF1FF2020506C616E6C
:102D00006E657242756666657242797465733A20C3
:102D1000002046726565204D656D6F72793A20001E
:102D200020436F6D70696C65643A2044656320329E
:102D30003720323032310A00204C617374205570D4
:102D400064617465643A20323032312D30392D306F
:102D500033207C20417574686F723A20286B61645F
:102D60002C20416E796375626963204D656761202F
:102D70005A65726F2041424C20313256290A004D6B
:102D800061726C696E20322E302E392E332D6B61BC
:102D900064310A0020536F66747761726520526552
:102DA0007365740A00205761746368646F6720520A
:102DB000657365740A002042726F776E206F7574B8
:102DC0002052657365740A002045787465726E61DF
:102DD0006C2052657365740A00506F776572557088
:102DE0000A0073746172740A004732385859004DF2
:102DF00031303031006572726F7220777269746998
:102E00006E6720746F2066696C650A00446F6E659A
:102E100020736176696E672066696C652E0A004DC5
:102E2000323900456E6473746F707300255320252A
:102E30006320256320256320256300205A3A002063
:102E4000593A0020583A00656E6473746F707320AD
:102E50006869743A2000000000010200090A0000BD
:102E6000000004030807000000000000000000004C
:102E7000000000000000004D6F76652025736D6D29
:102E8000004D6F766520302E316D6D004D6F76658B
:102E900020316D6D004D6F76652031306D6D004DC8
:102EA0006F76652041786973004D6F7665204578AF
:102EB000747275646572004D6F7665205A004D6FAF
:102EC00076652059004D6F76652058005072696E06
:102ED000742066726F6D204D6564696100FFFFFFAD
:102EE000205A3A200020593A200042656420583A7E
:102EF00020004D656761205A65726F2052656164DC
:102F0000792E005072696E74696E672E2E2E0050F5
:102F100072696E74205061757365640020450020ED
:102F20005A0020590020204D393220580053746532
:102F300070732070657220756E6974003B200022EA
:102F40000A00556E6B6E6F776E20636F6D6D616EEC
:102F5000643A2022006F6B00DB0FC93F45BCDA3FAB
:102F60008FB30240FCF0274056946140FE4B9B40DB
:102F700084A5D840E0231841346A5641E859974166
:102F800064DBD5416E271742B4B75542CE1A97423B
:102F9000C8AED542B5885A43D40684BFA65FA7BF42
:102FA0007443E0BF10B11AC01C2C58C0E8F697C09B
:102FB000B849D6C04E4E17C124D355C1802497C1FD
:102FC000A0B5D5C1121A17C244AE55C2781797C220
:102FD0006CACD5C267885AC320746F6F206C6F6E5B
:102FE0006720657874727573696F6E20707265768C
:102FF000656E7465640A0020636F6C642065787484
:10300000727573696F6E2070726576656E74656433
:103010000A006F6B0A00526573656E643A200020E7
:10302000453A00205A3A0020593A00583A00000028
:103030002200250028002B0000002100240027008A
:103040002A0002020202020202020404040404042E
:10305000040403030303030303030101010101014A
:103060000101010204081020408001020408102020
:103070004080010204081020408080402010080495
:1030800002014572726F722077726974696E6720EF
:10309000746F20454550524F4D210A005448455207
:1030A0004D414C2052554E4157415900546865726C
:1030B0006D616C2052756E6177617900FEDBC9E24B
:1030C00011241FBECFEFD0E4DEBFCDBF84B7809305
:1030D000541514BE0FB6F894A895809160008861CD
:1030E00080936000109260000FBE12E0A0E0B1E09B
:1030F000EEEFF3EE01E00BBF02C007900D92A8398E
:10310000B107D9F725E1A8E9B2E001C01D92A435C5
:10311000B207E1F718E1CFE5D8E104C02197FE013D
:103120000E94D2EECE35D107C9F70E94BADC0C94CA
:10313000F3F10C940000FC01A081B1811C92A281EA
:10314000B3818C918F5F8C930280F381E02D90810D
:103150008CE0989F800D1124EDE4F3E113AE84AF71
:103160000895FC0184910895FC01808108950097E1
:1031700051F0FC0180E09191992331F0907C9038DE
:10318000D1F38F5FF8CF80E00895119800C087FDDC
:1031900043C0419800C0119A00C000C0119800C0FF
:1031A00086FD46C0419800C0119A00C000C0119829
:1031B00000C085FD3BC0419800C0119A00C000C00E
:1031C000119800C084FD30C0419800C0119A00C021
:1031D00000C0119800C083FD25C0419800C0119A1D
:1031E00000C000C0119800C082FD1AC0419800C004
:1031F000119A00C000C0119800C081FD0FC0419815
:1032000000C0119A00C000C0119800C0419800C0D1
:10321000119A00C000C00895419ABCCF419AF0CFE6
:10322000419AE5CF419ADACF419ACFCF419AC4CFA4
:10323000419AB9CF90E080E00895CF93DF93DB010E
:10324000F9019C919130C1F0943080F094509C939E
:103250008830D1F480819181009771F0019791833A
:103260008083480F591FEA01188206C08C3539F453
:103270009C5F9C93943041F4DF91CF9108958B3300
:1032800039F781E08C93F8CF20813181B9016F5FEC
:103290007F4F71836083420F531FEA0188838081CF
:1032A00091818F3591056CF7E7CF0F931F9381E0E4
:1032B00000919F141091A0142091A1143091A21498
:1032C00040919B1450919C1460919D1470919E1498
:1032D000041715072607370708F480E01F910F91A0
:1032E000089590E080E008952091FD03833021F45B
:1032F00025FD0CC024FD0CC030E0A90102C055958D
:1033000047958A95E2F7CA018170089581E0089592
:1033100080E008958091190484FD0BC080911B0406
:1033200087FD07C090911C04937081E019F480E040
:10333000089581E008952FEB280F2A3108F047C047
:10334000E22FF0E08091190490911A04A0911B04DF
:10335000B0911C0404C0B695A795979587952A95BA
:10336000D2F780FD02C081700895E150FC4FE081EA
:10337000EE2341F180916C0790916D07E80FF92FD2
:10338000F11D808190ED980F9A3030F08E3251F41B
:10339000818180538A3098F4F093EE03E093ED033B
:1033A00081E008958D3211F08B3249F4818190EDE6
:1033B000980F9A3088F38E3211F48281EACFF0E0D0
:1033C000E0E0EACF1092EE031092ED03E9CF80E047
:1033D0000895CF93DF9385E4AEDF882309F188E079
:1033E0004091190450911A0460911B0470911C04BF
:1033F000972F9170C92F90E0D92FCC0FDD1F71FB53
:10340000222720F930E0220F331F220F331FC22B57
:1034100067FB442740F9C42B8C2BDF91CF91089593
:1034200080E0DECF88DF882341F081E02091ED034A
:103430003091EE03232B09F480E008951092B80335
:103440008091570190915801A0915901B0915A0172
:103450008093800590938105A0938205B0938305A6
:103460000895B0E0A0E0E7E3FAE10C94F6EE6B011A
:10347000E9014A3009F4D5C0453109F081C0DB01CA
:103480001296ED91FC91F28096818781139A00C08B
:103490000000E6E2F0E03197F0F7092F182FEF2C4B
:1034A000E29420EFE22230E1B32EBF0CE80188EF76
:1034B0006CDE00C0000086E290E00197F0F7BFE10B
:1034C000BF1508F49BC08F2D807780685EDE8E2D3F
:1034D0005CDE00C0000086E290E00197F0F780E833
:1034E00054DE80E052DE00C0000086E290E00197EA
:1034F000F0F78AEF4ADE00C0000086E290E0019714
:10350000F0F7005F1F4F8881807F3FDE89918295B1
:10351000807F3BDEC017D107B1F700C0000086E214
:1035200090E00197F0F7F394E0E1EE0EFB10BECFD0
:103530001398D6011296ED91FC9180819281980F9B
:1035400092832181921708F09FC194819F5F948399
:103550009381890F821710F08FEF820F838345814B
:1035600050E0440F551F70E060E0868197810E9413
:103570009FF181E0CDB7DEB7E9E00C9412EFDEC138
:10358000FB0102811381423309F485C108F48DC126
:10359000463409F475C1473409F482C14B3349F705
:1035A00089812B81D80112967C91129713963C91B8
:1035B000213009F4BFC1233009F0A0C148EF480F02
:1035C000582F91E0341708F490E031E0541708F0D8
:1035D00030E0492F432B61E0571708F460E04623A1
:1035E00011F4932331F2FA8030E0F901E156FE4FF5
:1035F000D08025563E4FF901E08099C180EE8F0DB5
:103600008068807FC2DD8F2D8295807FBEDD00C007
:10361000000086E290E00197F0F780E8B6DD80E8F0
:1036200061CF0B9A1398399A4198099A119A139A73
:1036300000C0000086E290E00197F0F788E790E094
:10364000CEE9DFE0FE013197F1F70197D9F788EF76
:103650009CDD00C0000086E290E00197F0F780E278
:1036600094DD80E092DD00C0000086E290E00197EA
:10367000F0F780E08ADD80E888DD00C0000086E2A7
:1036800090E00197F0F780E080DD80E17EDD00C012
:10369000000086E290E00197F0F7CE010197F1F784
:1036A000CE010197F1F7CE010197F1F7CE01019715
:1036B000F1F7CE010197F1F7CE010197F1F7CE01B5
:1036C0000197F1F7CE010197F1F7CE010197F1F7DC
:1036D000CE010197F1F7CE010197F1F7CE010197E5
:1036E000F1F7CE010197F1F7CE010197F1F721979C
:1036F000F1F780E24ADD80E448DD00C0000086E2A8
:1037000090E00197F0F780E240DD80E63EDD00C00A
:10371000000086E290E00197F0F7D0E0C0E08C2F47
:103720008077806832DD8D2F30DD00C0000086E2BA
:1037300090E00197F0F780E828DD80E026DD00C00A
:10374000000086E290E00197F0F78AEF1EDD00C0EE
:10375000000086E290E00197F0F780E2119800C047
:10376000419800C0119A00C000C0119800C0419853
:1037700000C0119A00C000C0119800C0419800C05C
:10378000119A00C000C0119800C0419800C0119A61
:1037900000C000C0119800C0419800C0119A00C03C
:1037A00000C0119800C0419800C0119A00C000C02C
:1037B000119800C0419800C0119A00C000C0119833
:1037C00000C0419800C0119A00C000C0119800C00C
:1037D000419800C0119A00C000C0119800C04198E3
:1037E00000C0119A00C000C0119800C0419800C0EC
:1037F000119A00C000C0119800C0419800C0119AF1
:1038000000C000C0119800C0419800C0119A00C0CB
:1038100000C0119800C0419800C0119A00C000C0BB
:10382000119800C0419800C0119A00C000C01198C2
:1038300000C0419800C0119A00C000C000C0000044
:10384000E6E2F0E03197F0F7815009F087CF88EF9A
:103850009CDC00C0000086E290E00197F0F7CF5FAB
:10386000D05FC03209F05BCF80E08FDC80EC8DDC74
:1038700000C0000086E290E00197F0F7139879CE3F
:10388000F8018581888375CE80E0CDB7DEB7E9E0A9
:103890000C9412EF53C0B901C8010E94A4CF69CEA5
:1038A000D80111968C91888364CE443191F04731D0
:1038B00009F05FCE1882D80112968C9112978983F5
:1038C00015968C91159781508A8313968C918B83D2
:1038D00050CED80115964C91159750E0440F551FC6
:1038E00070E060E016968D919C910E949FF1F80126
:1038F000128280818150838314823BCE381708F472
:1039000038CE871708F435CEFA80E12CD12C24303C
:1039100070F46ACEBE01C8010E94A4CF898198814B
:103920009D0D98838E0D8983FF0C09F422CEF7FE3E
:10393000F6CFF0CF58E0580F482F43CEEF92FF92CA
:103940000F931F93CF93DF93EC018B017A018A854C
:103950009B858617970731F0888199810E9491D1C4
:103960001B870A87B701888199810E9494C92E819B
:103970003F81820F932F911D9F838E8390E080E083
:10398000CDB7DEB7E6E00C9415EFB0E0A0E0EBECCD
:10399000FCE10C94F5EEEC017B018A018A859B85A4
:1039A0008617970731F0888199810E9491D1FB8613
:1039B000EA8688859985019609F5CC80DA808E8122
:1039C000D80EA880B980D5015596ED91FC91C5011E
:1039D0000995C80E780110E0F70121917F012111AE
:1039E0001FC08E819F81810F911D9F838E8390E0E8
:1039F00080E0CDB7DEB7EAE00C9411EFEE80FF80F7
:103A0000B801888199810E9494C98E0D9F2D911DC6
:103A1000288539852817390780F681E090E0E9CFBD
:103A20004C2D6D2DC5010E94E9D1D80E180FD4CFB1
:103A3000B0E0A0E0EEE1FDE10C94F8EEEC01D62E52
:103A40001CAD0BAD7C0184E0E80EF11CE98DFA8D14
:103A5000C7010995412F480F2D2D602FC7010E94E6
:103A6000E9D19BAD890F8BAF81E090E0CDB7DEB798
:103A7000E7E00C9414EFA6E0B0E0E1E4FDE10C9483
:103A8000EEEE7E836D83342EFC0140805180628097
:103A90007380C301B20120E13EE040E050E00E94AB
:103AA00035EE49015A0189018CE3C82ED12CE12C55
:103AB000F12CC301B201A70196010E9435EE698382
:103AC0007A838B839C83CA01B901A70196010E9466
:103AD00035EE6B017C01332061F1C301B20120E8B6
:103AE00031E541E050E00E9435EE29013A015901EB
:103AF000DF92CF92C40168E170E00E94ABEE9F9329
:103B00008F935F924F9285E492E19F938F93FE8112
:103B1000FF938D818F930E94A0E70FB6F894DEBFCC
:103B20000FBECDBF88E0FAE04F165104D8F089E00F
:103B300019C081149104D1F48A818F9399819F9344
:103B4000DF92CF9289E392E19F938F93EE81EF937F
:103B5000FD81FF930E94A0E70FB6F894DEBF0FBE71
:103B6000CDBF85E02696E1E10C940AEF04361105FD
:103B700068F4DF926F939F928F928DE292E19F9310
:103B80008F939E819F93ED81EF93E4CFDF926F93AC
:103B90009F928F9283E292E19F938F939E819F9356
:103BA000ED81EF930E94A0E70FB6F894DEBF0FBE41
:103BB000CDBF86E0D7CF682F70E090E080E00C9416
:103BC00091B08091ED039091EE03009731F04AE0BF
:103BD00050E070E060E00C9428E660E070E0CB011B
:103BE00008958091ED039091EE03009731F04AE043
:103BF00050E070E060E00C94FBE460E070E0CB012A
:103C00000895EFDF97FD0AC0ECDF6F3F7105810576
:103C1000910509F02CF4E5DF862F089580E00895E2
:103C20008FEF0895CF93C62FFDDB882311F0E9DFD6
:103C3000C82F8C2FCF9108958091ED039091EE03C2
:103C4000892B39F0DEDF91E0811101C090E0892FEE
:103C5000089591E0FCCFCF93DF93C82FD62FE2DBFE
:103C6000882321F0E9DFDF91CF9108958C2F63DB6A
:103C70008111F9CF8D2FF7CFB4DFCB010895CF930A
:103C8000DF93EB01CFDB882311F0F6DFEC01CE01EF
:103C9000DF91CF9108950F931F93CF938091ED0300
:103CA0009091EE030097D9F0FC018F01C1912C2F68
:103CB0002F7D81F0C53411F0C536B9F7F8011082B7
:103CC00070E060E00E94A5E3F801C083CF911F91EE
:103CD0000F91089570E060E00E94A5E3F7CF60E0E7
:103CE00070E0CB01F3CFCF92DF92EF92FF926A01A7
:103CF0007B0198DB882319F0CEDF6B017C01C701C3
:103D0000B601FF90EF90DF90CF900895CF92DF92B1
:103D1000EF92FF92CF93C82F0E9450CE6B017C018F
:103D200024EA30E74DE75FE36091310170913201A1
:103D300080913301909134010E9407E887FD18C0FB
:103D40008AEF90E0A0E0B0E08C0D9D1DAE1DBF1D80
:103D50008093680490936904A0936A04B0936B0401
:103D6000C0932701CF91FF90EF90DF90CF900895FF
:103D700080E090E0DC01E8CFCF93809129048111AD
:103D800054C0109288131092891310928A131092C3
:103D900056131092551310925813109257131092F5
:103DA0005A1381E08093591382E280935B1310923F
:103DB000601310925F13E4E7F3E122E833E18FEF41
:103DC00081932E173F07E1F7C1E0C093711325ECF3
:103DD0003EEA3093671320936613C09368131092E2
:103DE000691310926A1390E490936B1310926C1302
:103DF00024EC3EEA30938313209382132FE131E0C9
:103E000030935413209353139EE19093781391E1D0
:103E1000909379139CE1909376138093751380931C
:103E200074130E94E3CFC093290481E08093280497
:103E300084E692E19093841280938312109286120A
:103E40001092851253985B9A52985A9A3898409AD1
:103E50000E9485AB10927804CF910895FC0180E018
:103E6000309749F09491992331F0907C903809F083
:103E70008F5F3196F7CF0895B0E0A0E0E2E4FFE174
:103E80000C94F5EEEC015B018A01FB01099587FDBD
:103E900010C0C82ED12CF12CE12C2196F801C08243
:103EA000D182E282F382CE01CDB7DEB7EAE00C9494
:103EB00011EF982F907E903CA9F48F7190E0B0E0C4
:103EC000A0E06C017D0156E0CC0CDD1CEE1CFF1C5B
:103ED0005A95D1F7CE010196F50109958F73C82A3D
:103EE0002296DCCF982F907F903E11F58F7090E056
:103EF000B0E0A0E06C017D0136E0CC0CDD1CEE1CD6
:103F0000FF1C3A95D1F7CE010196F50109958F7303
:103F1000C82A46E0CC0CDD1CEE1CFF1C4A95D1F7EC
:103F2000CE010296F50109958F73C82A2396B6CF64
:103F3000982F987F903F79F5877090E0B0E0A0E0EF
:103F40006C017D0186E0CC0CDD1CEE1CFF1C8A950B
:103F5000D1F7CE010196F50109958F73C82A96E035
:103F6000CC0CDD1CEE1CFF1C9A95D1F7CE010296FD
:103F7000F50109958F73C82A26E0CC0CDD1CEE1CD8
:103F8000FF1C2A95D1F7CE010396F50109958F7391
:103F9000C82A249683CF982F907C903841F4807C57
:103FA000803869F42196CE01F5010995F8CF8E7F0E
:103FB0008D3F28F02196CE01F5010995F8CFC12C4F
:103FC000D12C76016BCF9CE0899F802D112491E04C
:103FD000980F909327042CE0280F2093560730E089
:103FE0002E5F3F4F409185134217130619F014F0CE
:103FF00080E00895209187139217D0F7662341F04F
:104000008E5F0E94C8D0809156078E5F0E94C8D0F4
:104010008091560790918513891750F3209187134B
:1040200090912704291720F3109288138093891305
:1040300081E0089520912604022E000C330B821794
:10404000130641F08093260469E873E181E593E16A
:104050000C9491D10895ACE0B0E0E1E3F0E20C946F
:10406000F7EE6F3F71058105910509F070F48DE45D
:1040700093E1DEDCE0915513F09156133196849173
:1040800090E02C96E8E00C9413EFF0908813E09009
:1040900089132091280421110FC043E052E16E2DB5
:1040A0008F2D0E9442D290E080E0F80EF0928813AB
:1040B000E09289139927E5CFC0905513D0905613FD
:1040C00021E533E13A8329832F2D30E03C832B8394
:1040D0002E2D30E03E832D8318861F822FEF3FEF79
:1040E0003A8729871C861B8605EC1CE19E012F5F01
:1040F0003F4FAB01BC01C6010E94D3AFB60181E5C1
:1041000093E10E9491D18F819885CFCF4F925F929A
:104110006F927F928F929F92BF92CF92DF92EF9297
:10412000FF920F931F93CF93DF93CDB7DEB72897FE
:104130000FB6F894DEBF0FBECDBF7C016A01490106
:10414000FB0190818CE0989F800D1124982FF7013E
:104150002081822F880F820F880F8093881390937D
:1041600089134115510561F1FA82E9827C836B83E1
:1041700001111FC0AE014B5F5F4FB401C6017CDE71
:104180006C016D817E818F81988561157105810536
:104190009105B1F060DFF70180818F5F8083853109
:1041A00048F3CE0101960E949B18E4CFB12C860102
:1041B00029C08A01B12C26C0452846284728B1F7D6
:1041C00028960FB6F894DEBF0FBECDBFDF91CF911A
:1041D0001F910F91FF90EF90DF90CF90BF909F9035
:1041E0008F907F906F905F904F900895B39407C029
:1041F000B1102DC001151105C9F20F5F1F4F011538
:104200001105A9F2AE014B5F5F4FB401C60134DE68
:104210006C014D805E806F8078844114510461048C
:104220007104A9F0F0E24F1651046104710401F326
:10423000D301C2018D97A109B1090297A105B1056A
:1042400030F04BE2441651046104710479F6F70131
:104250008081482F4B0D5527551F4631510534F0AD
:10426000853020F0CE0101960E949B1881E0411418
:1042700051046104710409F480E0B80EF7018081F3
:104280008B0D8083BB2009F497CFBA94AE014B5FAE
:104290005F4FB401C801F0DD8C016D817E818F819B
:1042A0009885D9DEEFCFCF93DF93FC0125AD2111A7
:1042B00004C021E025AF0E94E3CFC0915313D091F9
:1042C0005413E0918213F091831382E00995E091F9
:1042D0008213F091831381E0099530E020E044E1FE
:1042E000BE0181E593E10E94DECF24E833E147E19E
:1042F000BE0181E593E10E94DECFE0918213F0914F
:10430000831380E00995DF91CF9108954F925F92DA
:104310006F927F928F929F92AF92BF92CF92DF92D5
:10432000EF92FF92CF93DF9300D000D0CDB7DEB7EE
:104330000E9450CE6B017C01809127018F3FC1F11B
:104340000E9450CE8090680490906904A0906A0406
:10435000B0906B04681979098A099B0997FD28C0F8
:104360008091391390913A138F5F8F70891701F103
:10437000E0912701E53008F0DCC024E0E29FF00185
:104380001124ED55FE4F80819181A281B3818983F3
:104390009A83AB83BC8320E030E0A901BE016F5F4C
:1043A0007F4F87E791E00E9407C48FEF809327013A
:1043B0000E9485AB8091790482FFC4C0809177040C
:1043C00081111DC091E09093770480917E0489272C
:1043D0008093320710927E0483E080936C011092E8
:1043E00079040E9450CE6C507E4F8F4F9F4F609348
:1043F0007A0470937B0480937C0490937D04809175
:10440000730490917404A0917504B0917604A7018F
:104410009601281B390B4A0B5B0BDA01C901B7FF68
:1044200005C080917F04882309F4C5C1D701C60166
:104430008C599F4FAF4FBF4F809373049093740478
:10444000A0937504B093760460917804062E000C56
:10445000770B77FF03C0719561957109909178048E
:1044600080917204981371C0633008F06EC010928E
:1044700078048091780480937204643008F075C0E9
:10448000809132078111F3C080914B1390914C13AE
:104490008F519C4241F480912801882309F4F9C08E
:1044A0008150809328010E94007780908607909029
:1044B0008707A0908807B090890781110E940D7727
:1044C000D501C4013AE0B695A795979587953A9599
:1044D000D1F7009741E0A407B10520F08FEF9FEFDF
:1044E000A0E0B0E09695879520916C012111E3C082
:1044F00030917F0431118BC180914B1390914C13FB
:104500008F519C4209F46AC180918004811166C177
:1045100080916E0490916F04A0917004B091710429
:10452000C81AD90AEA0AFB0AF7FC66C10E94B58ECE
:1045300063C180916D0190916E01A0916F01B09166
:10454000700125CF109277045ACF633009F091CFD4
:104550008091780487FD07C081E0880F880F8093E1
:10456000780464E086CF8FEFF8CF8091550721E083
:1045700030E040E050E0882309F456C080905107B5
:1045800090905207A0905307B09054078114910463
:10459000A104B104E9F170E090E080E00E940BE832
:1045A00020E030E040E85EE30E946CE82B013C0133
:1045B000C701B601681979098A099B090E940BE8AD
:1045C0009B01AC01C301B2010E949FEF20E030E0EB
:1045D0004AE754E40E946CE84B015C0120E030E0C3
:1045E00040EA52E40E94C4F024E630E040E050E0AB
:1045F00087FF12C020E030E040EF51E4C501B40174
:104600000E94C4F02AE030E040E050E087FF04C0A0
:1046100021E030E040E050E0C0925107D0925207D4
:10462000E0925307F0925407A09178040A2E000CF0
:10463000BB0B0E947DEE24E030E040E050E00E94A1
:1046400057EE80914D0790914E07A0914F07B09182
:104650005007820F931FA41FB51F80934D0790939F
:104660004E07A0934F07B093500710927804D701DC
:10467000C6018856954CAF4FBF4F80936E04909300
:104680006F04A0937004B093710481E080936C0177
:10469000FBCE8CE08093280180916C0490916D0496
:1046A000009729F0019790936D0480936C0481E04A
:1046B00080936C01F8CE009741F040916C045091CA
:1046C0006D044817590708F017CF80917F048111B6
:1046D00011C0223038F0243008F43FC0243011F4E7
:1046E00010926C018DE493E1DEDD81E080934C0754
:1046F00080937F0483E09EDC81E080937113E091DE
:104700004B13F0914C13099510924C0780917F0444
:10471000811127C01092320780914B1390914C1356
:104720008F519C4209F0F0CE0E9450CEDC01CB01AB
:104730008C199D09AE09BF0980906C0490906D049E
:10474000B12CA12C88169906AA06BB0608F0D4CE77
:1047500090936D0480936C04CFCE81E080936C01C4
:10476000C1CF81E593E10E9461D191E0811101C047
:1047700090E090937F04882369F280914B1390918D
:104780004C138F519C42B9F40E9450CEDC01CB01F6
:104790008C199D09AE09BF09C0906C04D0906D04BE
:1047A000F12CE12CC816D906EA06FB0620F49093FA
:1047B0006D0480936C040F900F900F900F90DF9119
:1047C000CF91FF90EF90DF90CF90BF90AF909F90F0
:1047D0008F907F906F905F904F90089548E9C40E3E
:1047E0004AE3D41EE11CF11CC0926E04D0926F0407
:1047F000E0927004F092710480917F048111DBCF0C
:1048000080916C018130B9F610926C01D4CF009781
:1048100009F470CF52CFACE0B0E0E1E1F4E20C94E7
:10482000F7EEF0908813E09089132091280421116D
:1048300012C043EE51E16E2D8F2D0E9442D290E0C6
:1048400080E0F80EF0928813E092891399272C9655
:10485000E8E00C9413EFC0905513D090561321E567
:1048600033E13A8329832F2D30E03C832B832E2D97
:1048700030E03E832D8318861F827A8769871C86E5
:104880001B8605EC1CE19E012F5F3F4F41EB58E179
:10489000BC01C6010E9468B0B60181E593E10E94A7
:1048A00091D18F819885CDCFA4E0B0E0EAE5F4E224
:1048B0000C94F3EE7C01062F5A01122F862F660FFF
:1048C000990B9C0129563E4F690186E0882E912C58
:1048D00011160CF03DC0AE014F5F5F4F61EB78E108
:1048E000C701CADA7C0169817A818B819C8161155B
:1048F00071058105910561F16D33710581059105A2
:1049000009F450C06E3771058105910509F44AC05C
:104910006A3271058105910501F507FF11C08AE52D
:1049200092E10E3F11F086E592E136E01302B0010C
:10493000112471DF66E070E00E94BFEE161B60C0BC
:1049400065E470E080E090E086DB115069F510E0EE
:10495000812F2496ECE00C940FEF643271058105F1
:10496000910571F4A114B104D1F0E6E01E02B0018A
:104970001124C50150DFB4010E94BFEE161BA8CF61
:10498000603471058105910551F41150F601608183
:10499000062E000C770B880B990B5DDB99CF5BDB48
:1049A000115096CF07FDBBCF61E089819A81AB8121
:1049B000BC81CD97A105B10509F460E0600F6A30B4
:1049C000A4F01150862F6AE00E949EEE092F682FF6
:1049D000880F770B605D7F4F072E000C880B990BBB
:1049E0003ADB112309F4B3CF602F062E000C770BAE
:1049F000605D7F4F072E000C880B990B2CDB11504C
:104A0000112309F4A4CF86E01802B0011124C701D4
:104A100002DF66E070E00E94BFEE161B99CFEDE466
:104A2000F3E183AF64AF6FEF7FEFCA01F4CEACE088
:104A3000B0E0EDE1F5E20C94F7EEF0908813E09031
:104A4000891320912804211112C043EC51E16E2DED
:104A50008F2D0E9442D290E080E0F80EF0928813F1
:104A6000E092891399272C96E8E00C9413EFC090FC
:104A70005513D090561321E533E13A8329832F2D26
:104A800030E03C832B832E2D30E03E832D8318862F
:104A90001F827A8769871C861B8605EC1CE19E01B4
:104AA0002F5F3F4F44EB58E1BC01C6010E9468B044
:104AB000B60181E593E10E9491D18F819885CDCF98
:104AC0006FEF7FEFB4CFB0E0A0E0E9E6F5E20C9441
:104AD000F5EE5C016B01C2D9E82EC6010E94B71841
:104AE000F12C03E110E0081B1109C5E20E151F05AA
:104AF0000CF4CFE18C2F90E09C012E5F3F4F409152
:104B000085134217130609F08CF509972091871336
:104B1000281719065CF14091580750915907609188
:104B2000570710928813C093891325E1C501BCDE95
:104B3000D1E0C114D104A9F06AE370E080E090E014
:104B40008ADA0E151F05A4F4C45F80918513C81777
:104B500040F0209187134C2F4950550B2417150610
:104B60004CF4CDB7DEB7EAE00C9411EFD0E0E1CF22
:104B7000DD23B9F3802F880F080F000F00938813EF
:104B8000C093891360E270E080E090E064DAC601CF
:104B900097DFE7CFACE0B0E0E0EDF5E20C94F3EEA8
:104BA000982F862F6A017901B02E692F0CDA88239D
:104BB00009F487C010912804C701002371F14ED970
:104BC000A82E8090551390905613111142C02FEFCC
:104BD0003FEF122F23E12A194091580750915907AE
:104BE00060915707C60160DEAA2009F46AC0B6E0EA
:104BF0008B9F600111246AE370E080E090E02BDA83
:104C000057E0C516D10408F442C060E270E080E0CD
:104C100090E021DAC81AD90AF3CF0E94B718A82E5B
:104C20008090551390905613112389F2FE0133960C
:104C30008AE0DF011D928A95E9F781E593E19A8385
:104C400089830EE91CE19E012F5F3F4F44EB58E141
:104C500012C0FE0133968AE0DF011D928A95E9F7C2
:104C600081E593E19A8389830EE91CE19E012F5F20
:104C70003F4F41EB58E1B701C4010E9468B0B40155
:104C800081E593E10E9491D12F813885A2CF409197
:104C90005607212F30E0A6E0AA9EC00111242E5F06
:104CA0003F4F281739070CF49C0180E8821B809342
:104CB000881340938913BB2041F06FEF7FEFC7014A
:104CC000AADD2C96ECE00C940FEFC701F9DEF9CFCA
:104CD0000C94EEB04F925F926F927F928F929F9260
:104CE000BF92CF92DF92EF92FF920F931F93CF93D9
:104CF000DF9310921E0410921D042FE320932104D1
:104D00001092200410921F041092190410921A0499
:104D100010921B0410921C049C01F90190812F5FDA
:104D20003F4F9032D1F39E34C9F4818190ED980FBA
:104D30009A3020F08D3211F08B3281F432969F013F
:104D40002F5F3F4F808180538A3008F46DC09F01F0
:104D50002F5F3F4F8081803209F468C0F0936D0768
:104D6000E0936C078F010F5F1F4FC0816AE270E014
:104D7000C8010E94B9F1009731F0FC0131978081A0
:104D80008032E1F31182CD3421F0C43511F0C73403
:104D9000D9F5F80180810F5F1F4F8032D1F3805326
:104DA0008A3090F5C093210490E080E06AE0AF0182
:104DB0004F5F5F4F689F9001699F300D1124C901BB
:104DC000C0972081820F911D27FD9A95FA012081BD
:104DD00020532A3060F39093200480931F04DF0156
:104DE00031962C912032D9F3CD3461F58E31910575
:104DF00039F0F0F48731910519F08C31910511F5F6
:104E0000B0931E04A0931D04DF91CF911F910F91C9
:104E1000FF90EF90DF90CF90BF909F908F907F900A
:104E20006F905F904F900895F90189CFF9018FCF6E
:104E30008537910538F08737910510F3803A13E0F4
:104E40009107F1F280906C0790906D0740E050E080
:104E5000BA0130E020E0C12CD12C7601C394FD01D1
:104E60003196DC91DD2309F484C0D132F1F4CD34E4
:104E7000E1F480329105C9F44093190450931A0467
:104E800060931B0470931C04F0931E04E0931D04B4
:104E900063E270E0CF010E94B9F1009709F4B4CF4A
:104EA000FC011082B1CFDF01DACFD154DA3108F042
:104EB0005BC0DF011D91103291F0A0EDA10FAA306F
:104EC000E8F01E3271F4A181A053AA30B8F0211588
:104ED000310519F49F0121503109B12C13C0FD0196
:104EE000E8CF1D3211F01B3291F7A181B0EDBA0F5E
:104EF000BA3020F0AE3259F7A281E6CFBE2EB818F4
:104F0000309759F3AD2FB0E02601370104C0440CAF
:104F1000551C661C771CDA95D2F744295529662959
:104F20007729A150BC4FBC92A081A154AA3108F4AA
:104F3000BACFDF01D191DD2309F491CF00EDB02E7E
:104F4000BD0E19E01B15A8F713EDB12EBD0E11E033
:104F50001B1578F7DB3269F3FD013196DC91D03215
:104F600009F07DCFDF01F8CF21153105E9F69D016C
:104F7000DBCF30931E0420931D04409319045093FB
:104F80001A0460931B0470931C043ECFFC016591CE
:104F9000759185919491089580E00C94DF898F92AA
:104FA0009F92AF92BF92CF92DF92EF92FF92CF93F8
:104FB000DF93EC0180909A0490909B04A0909C0455
:104FC000B0909D0420E030E0A901C501B4010E9429
:104FD00007E8882309F452C0C880D980EA80FB80A2
:104FE000A7019601C501B4010E9407E818160CF04C
:104FF0004AC02091E9033091EA034091EB035091BC
:10500000EC03C701B6010E9407E8882321F1C09292
:10501000E903D092EA03E092EB03F092EC032091D3
:10502000E5033091E6034091E7035091E803C7019F
:10503000B6010E946CE89B01AC0160E070E080E882
:105040009FE30E9424EF60931401709315018093F5
:1050500016019093170160911401709115018091D0
:10506000160190911701DF91CF91FF90EF90DF90A3
:10507000CF90BF90AF909F908F90089560E070E0C8
:1050800080E89FE3F0CF60E070E0CB01ECCFB0E0D0
:10509000A0E0EDE4F8E20C94EFEEEC012091620563
:1050A000309163054091640550916505688179816F
:1050B0008A819B810E9424EF4B015C01209166054F
:1050C0003091670540916805509169056C817D813B
:1050D0008E819F810E9424EF6B017C01A5019401C8
:1050E00060910C0170910D0180910E0190910F0162
:1050F0000E9407E8882309F454C080920C01909222
:105100000D01A0920E01B0920F012091DD033091AC
:10511000DE034091DF035091E003C501B4010E941A
:105120006CE82B013C010E9438F04B015C0120E04F
:1051300030E040EA50E40E9407E8181634F4812C6D
:10514000912CC0EAAC2EC0E4BC2E20E030E0A901D6
:10515000C501B4010E94C4F087FF03C0812C912CCB
:105160005401A5019401C301B2010E9424EF609390
:10517000D5037093D6038093D7039093D803C501CA
:10518000B4010E9407F06093D303062E000C770B46
:105190006F5F7F4F6630710514F066E070E06093DA
:1051A000D103D0910A011091D303A7019601609118
:1051B00010017091110180911201909113010E94D0
:1051C00007E8811123C0D11375C02091B903309134
:1051D000BA034091BB035091BC036091D503709119
:1051E000D6038091D7039091D8030E946CE8209158
:1051F000BD033091BE034091BF035091C0030E9494
:1052000025EFCDB7DEB7E0E10C940BEFC0921001B3
:10521000D0921101E0921201F09213012091E1036A
:105220003091E2034091E3035091E403C701B601DA
:105230000E946CE84B015C010E9438F06B017C011C
:1052400020E030E040EA50E40E9407E8181634F409
:10525000C12CD12CB0EAEB2EB0E4FB2E20E030E0E4
:10526000A901C701B6010E94C4F087FF03C0C12C89
:10527000D12C7601A7019601C501B4010E9424EF4B
:105280006093D9037093DA038093DB039093DC037C
:10529000C701B6010E9407F06093D403062E000CEC
:1052A000770B6F5F7F4F6630710514F066E070E03A
:1052B0006093D203C091D403D11305C080910B0138
:1052C0008C1709F470C08091D3039091D40390930C
:1052D0000B0180930A010C2E000CDD0B27E012035A
:1052E000C0011124FC01EC0FFD1FEE0FFF1FEE0F9C
:1052F000FF1FE256FB4F2081318142815381209371
:10530000CD033093CE034093CF035093D00300914D
:10531000D203002E000C110BFC01E00FF11FEE0F69
:10532000FF1FEE0FFF1FE256FB4F608171818281EC
:1053300093810E9424EF6093C9037093CA03809302
:10534000CB039093CC032091D10337E02303F001EA
:105350001124CE0FDF1FCC0FDD1FCC0FDD1FC25677
:10536000DB4F288139814A815B812093C5033093CB
:10537000C6034093C7035093C803E00FF11FEE0F1D
:10538000FF1FEE0FFF1FE256FB4F6081718182818C
:1053900093810E9424EF6093C1037093C2038093B2
:1053A000C3039093C4038090D9039090DA03A09034
:1053B000DB03B090DC032091C9033091CA03409114
:1053C000CB035091CC03C501B4010E946CE820913D
:1053D000CD033091CE034091CF035091D0030E9472
:1053E00025EF6B017C01C092BD03D092BE03E09219
:1053F000BF03F092C0032091C1033091C2034091DA
:10540000C3035091C403C501B4010E946CE820910C
:10541000C5033091C6034091C7035091C8030E9451
:1054200025EFA70196010E9424EF6093B9037093C2
:10543000BA038093BB039093BC03C7CEACE0B0E04B
:10544000E4E2FAE20C94FCEE182F882379F020E0D5
:1054500030E0A90160916A0570916B0580916C053F
:1054600090916D050E9407E88823F1F080919904DE
:105470008117D1F00E942C748CE0EBE8F1E0DE01A2
:10548000119601900D928A95E1F7CE010196FFDD0C
:1054900080919904882361F087E791E00E948274EB
:1054A000109299040E9491872C96E3E00C9418EFD7
:1054B00081E08093990487E791E00E944E74F2CFD7
:1054C000CF92DF92EF92FF9280E0B8DF10926605F4
:1054D0001092670510926805109269051092620596
:1054E00010926305109264051092650510926E0586
:1054F00010926F05109270051092710510926A0556
:1055000010926B0510926C0510926D054EE954E0F7
:1055100027E0C12CD12C60ECE62E6FE7F62E90E050
:1055200080E0FC01EE0FFF1FEE0FFF1FE40FF51FE1
:10553000C082D182E282F38201968730910589F799
:105540002150445E5F4F2111EACFFF90EF90DF9032
:10555000CF9008954F925F926F927F928F929F9219
:10556000AF92BF92CF92DF92EF92FF921F93CF93B1
:10557000DF93EC01162F20919A0430919B04409107
:105580009C0450919D04688179818A819B810E944D
:1055900007E8882309F497C0B090990480E04EDFB3
:1055A000C880D980EA80FB8020E030E0A901C701F3
:1055B000B6010E94C4F087FF03C0C12CD12C760134
:1055C000C0929A04D0929B04E0929C04F0929D04B5
:1055D0002DEB37E346E855EBC701B6010E9407E81B
:1055E00087FD0BC02DEB37E346E855E3C701B60155
:1055F0000E94C4F018160CF076C0A701960160E076
:1056000070E080E89FE30E949FEF6093E503709352
:10561000E6038093E7039093E80380EF9FEFA9E709
:10562000B4EC8093E9039093EA03A093EB03B09367
:10563000EC03BB2009F447C04090770150907801FB
:105640006090790170907A0180907B0190907C014C
:10565000A0907D01B0907E01C0907F01D09080012C
:10566000E0908101F090820181E0E8DE112359F1A0
:10567000A301920160917701709178018091790185
:1056800090917A010E9407E881111BC0A501940145
:1056900060917B0170917C0180917D0190917E01F0
:1056A0000E9407E881110DC020917F013091800197
:1056B0004091810150918201C701B6010E9407E823
:1056C00081110E94DF87DF91CF911F91FF90EF90B2
:1056D000DF90CF90BF90AF909F908F907F906F9012
:1056E0005F904F90089560E070E0CB018ECF8F9275
:1056F0009F92AF92BF92CF92DF92EF92FF92C090B3
:105700006A05D0906B05E0906C05F0906D0520E087
:1057100030E0A901C701B6010E9407E88823E1F142
:10572000A701960160E070E080E89FE30E949FEF90
:105730006B017C0180906E0590906F05A0907005C4
:10574000B090710520E030E0A901C501B4010E94CC
:1057500007E8882329F1A501940160E070E080E862
:105760009FE30E949FEFC092DD03D092DE03E092A0
:10577000DF03F092E0036093E1037093E203809310
:10578000E3039093E403FF90EF90DF90CF90BF90FE
:10579000AF909F908F900895C12CD12C7601CACFE5
:1057A00060E070E0CB01DFCFCF92DF92EF92FF920B
:1057B0006B017C0183E3C816D104E104F10470F0AD
:1057C00082E3C81AD108E108F10862E370E080E0E2
:1057D00090E00E94C7CD0E94E171ECCFC701B601F5
:1057E0000E94C7CD0E94E171FF90EF90DF90CF90B3
:1057F0000895BC0190E080E00C9491B080916A071C
:10580000813069F09091A31492FB882780F992FF70
:1058100007C097FB882780F991E08927089581E0E8
:1058200008959091A31494FB882780F994FF06C0F3
:1058300081E09091A912911101C080E00895ACE03F
:10584000B0E0E5E2FCE20C94EFEE10925507809197
:10585000320710923207882361F020E040E070E0C8
:1058600060E086E299EA0E94798D2C96E0E10C9442
:105870000BEF2091390130913A0140914D07509141
:105880004E07CA01820F931F2436310509F0E9C380
:105890004730510544F006978A3091050CF0F0C36B
:1058A0008AE090E0F7C306964A3F5F4FACF38091E1
:1058B0004C07882309F4D0C160919512709196121B
:1058C000072E000C880B990B0E940DE811E0209127
:1058D00091123091921240919312509194120E9421
:1058E000C4F018160CF010E01093670480907F014C
:1058F00090908001A0908101B090820120E030E082
:10590000A901C501B4010E9407E8C12CD12CE0EA2D
:10591000EE2EE0ECFE2E87FD06C0C12CD12C70EAE5
:10592000E72E70E4F72E20E030E04AE754E4C501AA
:10593000B4010E946CE8A70196010E9425EF2DECAE
:105940003CEC4CEC5DE30E946CE80E9407F06B01BC
:105950007C0180E2F7FE09C0F094E094D094C094FA
:10596000C11CD11CE11CF11C8DE2409077015090CC
:1059700078016090790170907A0120917B013091DB
:105980007C0140917D0150917E0129873A874B87A8
:105990005C878093810460E230E1C31637E2D3066E
:1059A000E104F1048CF0C701B60120E137E240E0E8
:1059B00050E00E9457EECA01B9012AE030E040E011
:1059C00050E00E9457EE605D6093820460E248EE12
:1059D000C41643E0D406E104F1048CF0C701B6011B
:1059E00028EE33E040E050E00E9457EECA01B901D2
:1059F0002AE030E040E050E00E9457EE605D6093A6
:105A00008304C701B60124E630E040E050E00E9484
:105A100057EE6AE0862E912CA12CB12CCA01B90157
:105A2000A50194010E9457EE605D60938404C70154
:105A3000B601A50194010E9457EE6B01CA01B9019C
:105A4000A50194010E9457EECC2009F433C32EE245
:105A500020938504605D6093860450E3C50EC09278
:105A6000870461E874E08FE594E00E94C4F120E0CF
:105A700030E0A901C301B2010E9407E820E030E054
:105A800040E05FEB87FD04C020E030E040E05FE3F2
:105A9000C301B2010E9425EF0E9407F0CB010E94D2
:105AA000598CBC018AE594E00E94C4F120E030E00A
:105AB000A90169857A858B859C850E9407E820E08D
:105AC00030E040E05FEB87FD04C020E030E040E0E4
:105AD0005FE369857A858B859C850E9425EF0E940E
:105AE00007F0CB010E94598CBC0185E594E00E942F
:105AF000C4F18091A31400E117E283FD28C091DE78
:105B0000882309F4E9C280919B1490919C14A09180
:105B10009D14B0919E140097A105B10509F4DCC253
:105B2000BC01CD01615F784D8F4F9F4F20E137E27F
:105B300040E050E00E9435EE60919F147091A014F7
:105B40008091A1149091A2140E9435EE89010E94C7
:105B5000AF8B4B015C018D829E82AF82B886D62EC0
:105B6000809126018017C1F100932601C80164E6E7
:105B700070E00E94ABEE7B0188E48E9DB0018F9DAA
:105B8000700D112490E080E00E940BE82AE037EDD0
:105B900043E25CE30E946CE80E940CF060935404C2
:105BA0000115110509F09BC210924F041092450493
:105BB00080E8809344048FE494E0FC01019000208D
:105BC000E9F7CF018F549440982F990F890F880FD0
:105BD00090E8981B9093430480912501D816E1F139
:105BE0008092250141E08D819E81AF81B88580380A
:105BF0009145A140B10508F440E063E374E0CE01B3
:105C000005960E943B1D982F990F990F891B880FAD
:105C1000805880933204282D2370822EE9F40115D8
:105C20001105A9F0A0E1B7E2A01BB10B2D813E81C7
:105C30004F8158850E9473EE980150E040E00E9429
:105C400035EE211531054105510509F06EC210925E
:105C5000450480E8809344040E9450CE00912B04B8
:105C600010912C0420912D0430912E046B017C01A5
:105C7000C01AD10AE20AF30A9701860137FD11C062
:105C800020912A04209520932A046A547C4F8F4F38
:105C90009F4F60932B0470932C0480932D0490935A
:105CA0002E04D0902A0411E0D11001C010E081E050
:105CB0000E941A2080918513873180F48091871388
:105CC000843060F037E1E32E33E1F32E03E126E088
:105CD00044E069E081E593E10E9467D280918513F9
:105CE0008431B8F480918713823098F0DD2009F474
:105CF00035C280918A07882309F430C281EE92E18F
:105D00007C0102E123E042E068E681E593E10E9444
:105D100067D2809185138C3108F06EC0409091124B
:105D2000509092126090931270909412A0909512DD
:105D3000B0909612843198F480918713883078F06F
:105D40008091670480FF0DC283E992E17C010CE041
:105D500022E048E064E481E593E10E9467D280910B
:105D60008513883040F4B7FEFFC147E752E167E092
:105D700082E40E940F25809185138C31B0F48091CC
:105D80008713843190F020E030E040E05FE3C3010E
:105D9000B2010E9425EF0E9407F077FF0EC247E78D
:105DA00052E16CE182E40E940F25809185138C31D1
:105DB00018F5809187138431F8F080918A07882341
:105DC000D9F024E6829FC001112481589F4F6FEFC4
:105DD00070E00E94BFEECB010E94D88C27E6209392
:105DE00088132CE1209389130E94602565E270E0FE
:105DF00080E090E00E942B2014DD882379F18091CF
:105E00008513843358F5809187138A3238F107E07F
:105E100028E04AE26AE281E593E10E940ED105E0C2
:105E200022E04CE262E381E593E10E940ED124E09E
:105E30004AE061E38AE20E94DED0609153137091E0
:105E4000541382E380936D138BE280936E132DE6DF
:105E500033E142E381E593E10E94DECF8091851337
:105E6000853350F480918713813330F024E04AE485
:105E700061E386E30E94DED080918513843368F469
:105E800080918713823348F002E02091540442E36A
:105E900067E381E593E10E940ED180918513803301
:105EA00058F580918713883238F180913104811739
:105EB00051F080913004109331048F5F833008F0EB
:105EC000A5C180933004809130048111A2C18091DA
:105ED0004F04882389F0809143048093881380E3E2
:105EE000809389138FE494E00E94602565E270E05E
:105EF00080E090E00E942B2080918513883208F08A
:105F00005DC0809187138D3108F458C02BE040E8C4
:105F10006DE180E00E94DED080918513873208F029
:105F20004DC0809187138F3108F448C083E080937F
:105F3000881306E20093891368E570E080E090E042
:105F40000E942B208BE08093881300938913DD201F
:105F500009F491C18AE594E00E94602588E280936B
:105F6000881306E20093891369E570E080E090E011
:105F70000E942B2080E38093881300938913DD20F7
:105F800009F49EC185E594E00E9460258DE480932C
:105F9000881306E2009389136AE570E080E090E0E0
:105FA0000E942B2085E58093881300938913DD20C0
:105FB00009F4ABC18FE594E00E94602580918513C0
:105FC000833348F5809187138B3228F183E00E9458
:105FD0001A2083E08093881303E30093891366E01B
:105FE00070E080E090E00E942B2081E00E941A2067
:105FF0008091390190913A010E94D88C2CE0209335
:106000008813009389130E94602565E270E080E0A8
:1060100090E00E942B2080918513813408F025CCDC
:1060200080918713863308F420CC109288138EE376
:106030008093891382E290E10E94B718082F86317D
:1060400008F088C182E290E10E946025053109F4E0
:106050000CCC60E270E080E090E00E942B200F5FAB
:10606000F5CF243631054CF48536910504F58A3098
:10607000910534F48AE090E009C084369105BCF0C3
:10608000883EE3E09E0714F087EE93E02817390777
:1060900009F40DCC90933A018093390110924D0789
:1060A00010924E0710924F071092500700CC84E6D2
:1060B00090E0F0CF662351F02EE220938504605DDE
:1060C0006093860480E280938704CBCC80E2809347
:1060D000860480938504F6CF10E000E038CD2E2DA5
:1060E00080E2243628F08E2D64E60E9492EE805DD8
:1060F0008093850490E22A3040F03AE0822F632FAB
:106100000E9492EE0E9492EE905D90938604822F00
:106110006AE00E9492EE905D9093870465E874E0D7
:106120008FE494E00E94C4F146CD29833A834B83E7
:106130005C8381E0203831454140510508F480E01E
:10614000482F65E474E0CE0101960E943B1D982F14
:10615000990F990F891B880F80587CCD8BEA92E1AB
:10616000CFCD8BE792E1F2CDC5010E94D88CFC0126
:10617000808193E0803229F4818192E0803209F4B9
:1061800091E0892F880F880FE92EE81A8E2D855B04
:106190008093881387E08093891323E030E0291BE4
:1061A0003109CF01820F931F0E94602569E070E0E2
:1061B00080E090E00E942B20DECDCB010E94D88CA5
:1061C000FC01808193E0803229F4818192E0803269
:1061D00009F491E0892F880F880FF92EF81A8F2D76
:1061E000855B809388138CE18093891323E030E0F2
:1061F000291B3109CF01820F931F0E94602569E09E
:1062000070E080E090E00E942B20CFCD109230040F
:106210005ACE8230B1F480914504882391F044E74E
:1062200052E160E386E30E940F258091440480934D
:10623000881380E38093891385E494E00E946025AD
:106240005BCE80913304882309F456CE86E3809395
:10625000881300E3009389136FEF7FEF81E792E1EA
:106260000E940B2480913204809388130093891339
:1062700083E394E0E3CF87E00E943E8380FF15C074
:106280002AE5E22E24E0F22EF70161917F016623D8
:1062900009F464CE6F320CF06FE3062E000C770B1E
:1062A000880B990B0E942B20EFCF80915A0780FD1D
:1062B00051CE6FEF7FEF8CE692E10E940B244ECE21
:1062C00087E00E943E8381FF15C095E5E92E94E0AA
:1062D000F92EF70161917F01662309F457CE6F32E1
:1062E0000CF06FE3062E000C770B880B990B0E94C5
:1062F0002B20EFCF80915A0781FD44CE6FEF7FEFC7
:106300008CE692E10E940B2441CE87E00E943E83FE
:1063100082FF15C08FE5E82E84E0F82EF701619129
:106320007F01662309F44ACE6F320CF06FE3062E2C
:10633000000C770B880B990B0E942B20EFCF8091DC
:106340005A0782FD37CE6FEF7FEF84E692E10E941D
:106350000B2434CE80912F041817B1F00091211036
:1063600010932F0482E290E10E94B718081708F0FA
:1063700050C00F5FE02FF0E0EE5DFF4E8081807C2B
:106380008038B9F300932110E0902110F12C97018F
:106390002E5D3F4E7901C9010E94B718182F60E8A1
:1063A00070E0C7010E941725153108F05ECA60E24F
:1063B00070E080E090E00E942B20143109F455CA6F
:1063C00060E270E080E090E00E942B20133109F43D
:1063D0004CCA60E270E080E090E00E942B20123115
:1063E00009F443CA212F30E02E5F3F4F4AEF4203AA
:1063F000B001439F700D112460587F4F82E290E1FD
:106400000E94172560E270E080E090E00E942B205F
:106410002CCA10922110B8CF80916A07823059F0AF
:1064200000DA882349F08091A31482FB882780F941
:1064300091E08927089581E0089581E00895DC01C5
:10644000EC918E2F90E0FC01EE0FFF1FE80FF91F7B
:10645000E050FD4E80818F7780830895892B79F4F9
:106460001092900082E0809391001092950010921B
:106470009400C19A809171008260809371000895A8
:10648000B0E0A0E0E6E4F2E30C94F2EEEC017B0174
:1064900088818C3008F0A4C090E0FC01EE0FFF1F53
:1064A000E80FF91FE050FD4E80818F770E9419B3ED
:1064B00019821A8288812CE0622F0E9492EE829FBC
:1064C000B001112430E020E0AB01420F531FFA016C
:1064D000EE0FFF1FE40FF51FE050FD4E908197FD7A
:1064E00007C02F5F3F4F2C30310571F790E0B6DFCA
:1064F0007880072D10E06801CC0CDD1CF601E00F60
:10650000F11FE050FD4E80818068808377FC68C079
:1065100080E2E81682E0F8060CF03FC08A8128E5A8
:1065200032E0281B310987FD3395220F331F220FDC
:10653000331F032E000C440B550B898178E8872EFE
:10654000912C881A910887FD9394880C991C880CCB
:10655000991C092C000CAA08BB0860E070E0CB0174
:10656000F7FC0AC0B701653B710514F064EB70E0FD
:10657000072E000C880B990B281939094A095B0969
:106580000E9426EE24EB30E040E050E00E9457EEFF
:10659000820E931EA41EB51E74018BE08715D8F0E1
:1065A000298188E890E0821B910927FD9395880F47
:1065B000991F880F991FE816F906BCF402972FB7A8
:1065C000F894E601C00FD11FC050DD4E880F991F0F
:1065D0009A8389832FBF62E370E080E090E0E4D883
:1065E000CDB7DEB7EDE00C940EEF2A8188E592E09E
:1065F000821B910927FD9395880F991F880F991F7A
:10660000E816F906DCF6C701D9CFCF93DF93EB018B
:10661000682F70E085E293E133DF688179818A81B8
:106620009B81643F21E072078105910520F464EFAE
:1066300071E080E090E0B8D886B182958170DF91FA
:10664000CF910895A4E0B0E0E8E2F3E30C94FDEE0E
:106650008EEE92E0A0E0B0E089839A83AB83BC83A6
:10666000BE016F5F7F4F8AE5D0DF2496E2E00C9495
:1066700019EFA4E0B0E0EFE3F3E30C94FDEE8EEE4F
:1066800092E0A0E0B0E089839A83AB83BC83BE0133
:106690006F5F7F4F8AE0B9DF2496E2E00C9419EF38
:1066A000A4E0B0E0E6E5F3E30C94FDEE84EF91E0C6
:1066B000A0E0B0E089839A83AB83BC83BE016F5FA7
:1066C0007F4F8CE3A2DF2496E2E00C9419EFA4E064
:1066D000B0E0EDE6F3E30C94FDEE84EF91E0A0E092
:1066E000B0E089839A83AB83BC83BE016F5F7F4F29
:1066F00080EA8BDF2496E2E00C9419EF1F920F9250
:106700000FB60F9211240BB60F922F933F934F9316
:106710005F936F937F938F939F93AF93BF93EF9309
:10672000FF938091A80387FF27C0109295001092D5
:1067300094008091A8038F5F8093A8038091A803A1
:10674000082E000C990B209124132817190629F004
:1067500024F08091A8038C30DCF18091940090911A
:106760009500049680349C4908F47DC08091940083
:1067700090919500049679C08091A803082E000C92
:10678000990B209124132817190699F294F2E0919D
:10679000A8038E2FEE0F990BFC01EE0FFF1FE80FE1
:1067A000F91FE050FD4E808187FFC3CFE091A80321
:1067B0008E2FEE0F990BFC01EE0FFF1FE80FF91F54
:1067C000E050FD4E808160E08F770E946BCDB1CFAD
:1067D0002091940030919500E091A8038E2FEE0F48
:1067E000990BFC01EE0FFF1FE80FF91FE050FD4E63
:1067F00081819281820F931F9093990080939800DA
:10680000E091A8038E2FEE0F990BFC01EE0FFF1FF6
:10681000E80FF91FE050FD4E808187FF11C0E09125
:10682000A8038E2FEE0F990BFC01EE0FFF1FE80F50
:10683000F91FE050FD4E808161E08F770E946BCDA3
:10684000FF91EF91BF91AF919F918F917F916F9148
:106850005F914F913F912F910F900BBE0F900FBE04
:106860000F901F90189580E49CE990939900809375
:1068700098008FEF8093A803E3CF9091C00095FF1D
:10688000FCCF8093C6000895CF93DF93EC018991EC
:10689000882311F0F2DFFBCFDF91CF910895CF93E2
:1068A000DF93EC018991882311F0E7DFFBCF8DE0C6
:1068B000E4DF8AE0E2DFDF91CF910895CF93DF93A9
:1068C000EC01FE0184912196882311F0D6DFF9CFE7
:1068D000DF91CF9108950F931F93CF938C01C62F13
:1068E0008AED9FE0EBDFC801E9DF8AE3C6DF80E3E2
:1068F0008C0FC3DF8AE0C1DFCF911F910F91089504
:10690000CF92DF92EF92FF926A017B01D7DF42E0E4
:10691000C701B6010E9438B3FF90EF90DF90CF908F
:106920000895CF93DF9361EF7FE00E9485C4C0910B
:106930003413D0913513488159816A817B8188EE67
:106940009FE0DEDF4C815D816E817F8182E29FE28C
:10695000D7DF409130135091311360913213709111
:1069600033138FE19FE2CCDF85EE9FE0A7DF8FED51
:106970009FE0A4DF8AE081DFDF91CF910895C0DF3F
:106980008AE07BCFAEE4B0E0E8ECF4E30C94EDEE0B
:1069900070E060E085E40E943F1E9AA789A78111FC
:1069A0007CC26EEB70E083E50E943F1E3C0165E017
:1069B00070E083E40E943F1E8C0160E085E50E9448
:1069C0002B1E8DAF60E086EB91E10E941BA20E941E
:1069D00050CE69877A878B879C87809169019091D7
:1069E0006A010E976816790654F087E691E166DF32
:1069F0000E9409C5C25BDF4FE2E10C9409EF2985D3
:106A00003A854B855C85205E314B4F4F5F4F2BABFA
:106A10003CAB4DAB5EAB83E591E150DF0E9458711A
:106A20008FE78093971281E080936B0160E08FE3A2
:106A300091E10E941BA289859A85AB85BC85898BD3
:106A40009A8BAB8BBC8B8BA79CA7ADA7BEA7198ECF
:106A50001A8E1B8E1C8E19A21AA21BA21CA21982AE
:106A60001A821B821C822FE730E040E050E02D8725
:106A70003E874F87588B80E090E4ACE1B6E48D838D
:106A80009E83AF83B8871D8A1E8A1F8A188EFFE7F0
:106A9000CF2ED12CE12CF12C2F961FAE2F971FA6B5
:106AA00018AA19AA1AAA1DA21EA21FA218A691E02E
:106AB0009FAB312C212C812C912C54019301072C5C
:106AC000000C440B550B22962CAF3DAF4EAF5FAF81
:106AD0002297402F002E000C550B5CAF4BAFC3012B
:106AE0004E969C01092E000C440B550B26962CAF9C
:106AF0003DAF4EAF5FAF2697CC979C01990F440BEB
:106B0000550B2A962CAF3DAF4EAF5FAF2A9736E0BC
:106B1000631A7108C301072C000CAA0BBB0B2E963D
:106B20008CAF9DAFAEAFBFAF2E9780916B01882326
:106B300009F48DC00E9450CE2B013C0110918A05B2
:106B4000112309F473C00E94A87110928A058090E5
:106B5000911290909212A0909312B0909412A5016D
:106B600094016D897E898F89988D0E94C4F087FF7A
:106B700004C08D8A9E8AAF8AB88EA50194016D816A
:106B80007E818F8198850E9407E8181624F48D82F3
:106B90009E82AF82B88622966CAD7DAD8EAD9FADE4
:106BA00022970E940DE86D8F7E8F8F8F98A39FA9EB
:106BB0002D8D3E8D4F8D58A1992309F472C1C501C9
:106BC000B4010E94C4F018168CF5D301C2012989C2
:106BD0003A894B895C89821B930BA40BB50BAC01E2
:106BE000BD01485853416109710977FD1FC04D85AA
:106BF0005E856F8578894C195D096E097F097595E9
:106C0000679557954795409397128DA39EA3AFA381
:106C1000B8A78D8D9E8DAF8DB8A18D8B9E8BAF8BC0
:106C2000B88F49865A866B867C861FAA26966CADDD
:106C30007DAD8EAD9FAD26970E940DE8A501940114
:106C40000E9407E887FF21C088EB90E137DE1092B1
:106C50006B010E945871CCCE4BEEC42ED12CE12C8E
:106C6000F12C76C124E130E040E050E02D873E87F2
:106C70004F87588B34E1C32ED12CE12CF12C76C1F7
:106C8000CD86DE86EF86F88A71C1D301C2012BA5BD
:106C90003CA54DA55EA5821B930BA40BB50BB7FDC0
:106CA00047C089A50E94CD708AE0E7DDD301C2010B
:106CB0008053984FAF4FBF4F8BA79CA7ADA7BEA7E0
:106CC0002F969FAD2F9791116FC02FA538A949A975
:106CD0005AA9C501B4010E94C4F018160CF050C0A6
:106CE00020E030E040E050E4C501B4010E9425EF0F
:106CF0006FA778AB89AB9AABA3019201205E314BB1
:106D00004F4F5F4F2BAB3CAB4DAB5EAB2E966CAD9C
:106D10007DAD8EAD9FAD2E970E940DE8A50194012B
:106D20000E9407E8881F8827881F2F968FAF2F970C
:106D300089859A85AB85BC858D8F9E8FAF8FB8A3D3
:106D400029893A894B895C89281739074A075B07E3
:106D500020F42D8F3E8F4F8F58A38D8D9E8DAF8D3C
:106D6000B8A1481A590A6A0A7B0A91E849169FE4B1
:106D7000590692E16906710460F18AE990E166CFF3
:106D8000D301C2012BA93CA94DA95EA9821B930B7B
:106D9000A40BB50B46EC59E265ED79E2B7FDC8CF1F
:106DA00080E00E946771C4CF2A966CAD7DAD8EAD38
:106DB0009FAD2A970E940DE89B01AC01C501B4016B
:106DC0000E9407E887FFB4CF4CE950E36CEA70E318
:106DD000E7CFABADBCADA215B3050CF05BC0B3E023
:106DE0002B1631040CF456C08DE390E167DD80E290
:106DF00090E164DD49815A816B817C8189E390E176
:106E0000BEDD80E290E15ADD49A15AA16BA17CA1CF
:106E100085E390E1B4DD80E290E150DD498D5A8D4B
:106E20006B8D7C8D81E390E1AADD2DAD222309F4E9
:106E3000DFCD89819A81AB81BC8180939812909338
:106E40009912A0939A12B0939B122CEA35EC47E268
:106E50005EE369A17AA18BA19CA10E946CE860937A
:106E60009C1270939D1280939E1290939F1220E02B
:106E700030E543EC50E4698D7A8D8B8D9C8D0E94BA
:106E80006CE86093A0127093A1128093A212909369
:106E9000A312AECD0E94862148CE82E991E10EDD9B
:106EA000A9CDC501B4010E9407E887FFBFCED30179
:106EB000C20129853A854B855C85821B930BA40B07
:106EC000B50BAC01BD01485853416109710977FD0B
:106ED000ADCE2114310409F4FCC02DA13EA14FA177
:106EE00058A5280F391F4A1F5B1F298B3A8B4B8BE4
:106EF0005C8B2DA13EA14FA158A5281B390B4A0B35
:106F00005B0BC701B6010E9426EE29893A894B899D
:106F10005C890E9457EECD84DE84EF84F888C20E2F
:106F2000D31EE41EF51E34E1C316D104E104F104BE
:106F30000CF498CE4CEEC416D104E104F1040CF02C
:106F40008BCE50E8C516D104E104F1040CF498CEC0
:106F5000CD86DE86EF86F88A8EEF90E0A0E0B0E086
:106F60008C199D09AE09BF096C017D0187E391E190
:106F7000A5DC6D857E858F8598890E94682682E3D1
:106F800091E19CDCC701B6010E9468264D815E81BB
:106F90006F8178858BE291E1B3DC4D895E896F89E1
:106FA000788D84E291E1ACDC33E0231631040CF4FB
:106FB00090C0C701B6010E940DE820E030E040E833
:106FC00050E40E946CE869837A838B839C832D81D3
:106FD0003E814F8158856D897E898F89988D0E9469
:106FE00024EF2BED3FE049EC5FE30E946CE89B014E
:106FF000AC0169817A818B819C810E949FEF6FAB8C
:1070000078AF89AF9AAF69897A898B899C890E9408
:107010000DE82FE632E143E85AE30E946CE86D8305
:107020007E838F8398872AE939E949E15FE36FA975
:1070300078AD89AD9AAD0E946CE869837A838B83C1
:107040009C839B01AC010E9425EF2D813E814F81E5
:1070500058850E949FEF69A37AA38BA39CA320E08D
:1070600030E040E05EE36D817E818F8198850E94F3
:107070006CE829813A814B815C810E946CE8698FC0
:107080007A8F8B8F9C8F4FA958AD69AD7AAD8EE109
:1070900091E136DC4D815E816F81788588E191E1F7
:1070A0006EDC89E091E10ADC49815A816B817C8147
:1070B00083E091E125DC49A15AA16BA17CA18DEF70
:1070C00090E11EDC498D5A8D6B8D7C8D87EF90E1B0
:1070D00056DC8D859E85AF85B8898C0D9D1DAE1DB6
:1070E000BF1DB595A79597958795809397124CAD41
:1070F0004F930F933F922F9283EE90E19F938F9344
:107100002EEE30E13F932F931F920E94FEA15FEF7E
:10711000251A350A0FB6F894DEBF0FBECDBF2D8DF0
:107120003E8D4F8D58A12D833E834F835887498ACA
:107130005A8A6B8A7C8A1FAB79CD63E378E00E9420
:1071400085C460915C0D70915D0D80915E0D909194
:107150005F0D0E940BE8AB01BC018AE298E0D0DB36
:1071600040918C0D50918D0D60918E0D70918F0D11
:1071700087E298E0C5DB4091900D5091910D6091B0
:10718000920D7091930D84E298E0BADB40916E0706
:1071900050916F07609170077091710781E298E0DC
:1071A000EECBCF93DF9367ED77E00E9485C4CCE40C
:1071B000DDE04CA95DA96EA97FA98EEC97E0A0DB6C
:1071C00048AD59AD6AAD7BAD8BEC97E099DB4CAD2A
:1071D0005DAD6EAD7FAD84E298E0D1DBDF91CF9104
:1071E0000895CF93DF9363EB77E00E9485C4CCE4EE
:1071F000DDE04CA15DA16EA17FA18AEA97E080DB72
:1072000048A559A56AA57BA582E29FE279DB4CA53A
:107210005DA56EA57FA58FE19FE272DB48A959A904
:107220006AA97BA98CE19FE2AADBDF91CF91089547
:10723000CF93DF936EE877E00E9485C4CCE4DDE075
:10724000688179818A819B810E940BE8AB01BC0136
:1072500085E897E055DB6C817D818E819F810E945E
:107260000BE8AB01BC0182E29FE24ADB68857985CD
:107270008A859B850E940BE8AB01BC018FE19FE2F0
:107280003FDB6C857D858E859F850E940BE8AB0179
:10729000BC018CE19FE273DBDF91CF910895AF9247
:1072A000BF92CF92DF92EF920F931F93CF93DF9312
:1072B0005B01EA016901882309F452C08EE797E077
:1072C000FDDAF501608171818281938146E00E943F
:1072D00038B3E1100AC085E797E0F0DA6881798178
:1072E0008A819B8146E00E9438B38EE697E0E6DA19
:1072F000F601608171818281938143E00E9438B3FD
:1073000087E697E0DBDAF801608171818281938101
:1073100043E00E9438B38EE597E0D0DAF601208191
:10732000318142815381F801608171818281938131
:107330000E9424EF43E00E9438B3EE2099F08AE0E7
:107340009CDA89E497E0BADA688179818A819B8145
:1073500046E00E9438B38AE090DA8AE08EDA02C012
:10736000E110EFCFDF91CF911F910F91EF90DF9060
:10737000CF90BF90AF900895A6E5B0E0E2ECF9E3BE
:107380000C94EDEE2DB63EB687E00E945983811134
:107390000AC061E086E50E94121E8DA3853090F040
:1073A00084E297E08BDA0FB6F8943EBE0FBE2DBE96
:1073B0000FB6F8943EBE0FBE2DBECA5ADF4FE2E1B3
:1073C0000C9409EF2DA1222319F084E097E076DADE
:1073D0006AE080E50E94121E182F8CEF810F8F3219
:1073E00018F080EE96E0DECF60E085E40E942B1E70
:1073F000882309F447C031E038AFE0903413F090AF
:107400003513D7012D913D914D915C91609177019C
:10741000709178018091790190917A010E9425EF15
:10742000AB01BC0188E50E94731E69877A878B8750
:107430009C87F701248135814681578160917B01CA
:1074400070917C0180917D0190917E010E9425EFD9
:10745000AB01BC0189E50E94731E6D877E878F8713
:10746000988BBE01635F7F4FCE0109960E944BC58A
:1074700081110BC063E68CEC96E00E941BA284EBAA
:1074800096E090CF83E088AFB8CF8CE40E949B1940
:10749000082F882309F44EC10E94011E8EA380315B
:1074A00018F08DE896E07ECFFEA1F13009F444C1DA
:1074B00060E083E50E942B1E22968FAF22978823DF
:1074C00021F0011102C037E03EA38DA1833018F0F6
:1074D00083E796E0F3D99091990429969FAF299775
:1074E00080E00E941E2A0E94C4861D8A1E8A1F8A6E
:1074F000188E198E1A8E1B8E1C8E83EF9FE4A3ECC0
:10750000B7E48D8F9E8FAF8FB8A383EF9FE4A3EC7A
:10751000B7EC89A39AA3ABA3BCA3A12FB0E0BBABEC
:10752000AAABEDB7FEB724E0129FE019F1091124D0
:107530000FB6F894FEBF0FBEEDBF8DB79EB7019694
:1075400024969FAF8EAF24972DA148ADBE01635FF7
:107550007F4FCE0109960E9481C60E9450CE6115D0
:1075600071058105910511F00E949CE319AA1CAADE
:107570001DAA1EAA1FAAAEA1A150BB0B6396BFAF46
:10758000AEAF6397812F90E0B0E0A0E067968CAF3C
:107590009DAFAEAFBFAF6797B9A9AB2FB0E0BCA7A7
:1075A000ABA7EAA9FBA9AE17BF070CF07BC21196E7
:1075B000B8A7AFA3FF93EF93BF93AF938FE596E088
:1075C0009F938F9389E696E09F938F931F920E94DB
:1075D000FEA12DB73EB7275F3F4F0FB6F8943EBFD1
:1075E0000FBE2DBF3EA1332309F48CC10E944DE391
:1075F0002AE030E040E050E00E9457EE0E940DE8A3
:1076000020E030E040EA50E40E94C4F00FEF1FEFAA
:10761000181614F001E010E00E944DE328E631E076
:1076200040E050E00E9457EE0E940DE82B013C0123
:107630000E944DE327E130E040E050E00E9457EE29
:107640006B5F7F4F8F4F9F4F0E940DE869AF7AAFFE
:107650008BAF9CAF8DA18430B9F449AD5AAD6BAD01
:107660007CAD81E596E04CD9B301A20189E496E0B6
:1076700047D983E496E022D90130110511F483E45F
:10768000FCD88FE396E01AD9B801110F880B990B3B
:107690000E940DE821966CAF7DAF8EAF9FAF219712
:1076A00020E030E040E153E40E946CE82D966CAF9E
:1076B0007DAF8EAF9FAF2D971FA6EFA56396AEADA2
:1076C000BFAD6397EA171B060CF01CC12296FFADF5
:1076D0002297F11134C00E944DE324E130E040E0F4
:1076E00050E00E9457EE675E7F4F8F4F9F4F0E9482
:1076F0000DE821962CAD3DAD4EAD5FAD21970E94BA
:107700006CE89B01AC01C301B2010E9425EF2B0183
:107710003C0120E030E044EB53E40E9407E81816F7
:10772000ACF420E030E044EB53E4C301B2010E942A
:1077300024EFEDCF1EA2BCCE22E02EA3B9CE2D9613
:107740002CAD3DAD4EAD5FAD2D97DDCF20E030E0EF
:10775000A901C301B2010E94C4F087FF0BC020E061
:1077600030E044EB53E4C301B2010E9425EF2B014A
:107770003C01ECCF0091341310913513D8011496CD
:107780002D913D914D915C9117976D857E858F85EB
:1077900098890E9424EF61966CAF7DAF8EAF9FAF4A
:1077A000619726E33AEF4EE85CE3C301B2010E9421
:1077B0006CE86B017C010E949CEF28966CAF7DAF5A
:1077C0008EAF9FAF2897F80120813181428153818C
:1077D00069857A858B859C850E9424EF4B015C012D
:1077E00029AD3AAD4BAD5CAD28966CAD7DAD8EAD9F
:1077F0009FAD28970E946CE89B01AC01C501B401C4
:107800000E9425EF4B015C0189829A82AB82BC8287
:10781000C701B6010E94F9F029AD3AAD4BAD5CADA0
:107820000E946CE861962CAD3DAD4EAD5FAD6197A9
:107830000E9425EF6B017C01CD82DE82EF82F8860B
:1078400020E030E040EE50ECC501B4010E9407E8B2
:1078500087FF3AC080E090E0A0EEB0EC89839A8385
:10786000AB83BC8320E030E040E050ECC701B601C0
:107870000E9407E887FF37C080E090E0A0E0B0EC0E
:107880008D839E83AF83B887FDA1F43071F4498165
:107890005A816B817C8183E396E032D84D815E8191
:1078A0006F81788582E29FE26AD8198A1A8A1B8AD8
:1078B0001C8ABE016F5E7F4FCE0101960E94F0C709
:1078C0002FA52F5F2FA7F9CE20E030E041E653E44B
:1078D000C501B4010E94C4F0181624F680E090E0BF
:1078E000A1E6B3E4BBCF20E030E041E653E4C701BA
:1078F000B6010E94C4F018163CF680E090E0A1E6C4
:10790000B3E4BECF20E048ADBE01635F7F4FCE0140
:1079100009960E9481C64B015C01EBA5FCA5EE0F08
:10792000FF1FEE0FFF1F24968EAD9FAD2497E80F2B
:10793000F91F80829182A282B382A50194016D8D8C
:107940007E8D8F8D98A10E94C4F0181624F48D8E20
:107950009E8EAF8EB8A2A501940169A17AA18BA1D8
:107960009CA10E9407E887FF04C089A29AA2ABA24B
:10797000BCA2A50194016CA97DA98EA99FA90E9412
:1079800025EF6CAB7DAB8EAB9FAB8FA198A5092E7D
:10799000000CAA0BBB0B8FA398A7A9A7BAA7BC0181
:1079A000CD010E940DE86BA77CA78DA79EA79B0128
:1079B000AC016CA97DA98EA99FA90E949FEF2B0104
:1079C0003C014D8A5E8A6F8A788E2496AEADBFAD3B
:1079D0002497B8ABAFA710E0C12CD12C7601EFA54E
:1079E000F8A96191719181919191F8ABEFA7A301F1
:1079F00092010E9424EF9B01AC010E946CE89B0164
:107A0000AC01C701B6010E9425EF6B017C011F5F2D
:107A1000F9A9F11720F72BA53CA54DA55EA50E945D
:107A20009FEF0E9403F1698F7A8F8B8F9C8F2DA11E
:107A30002230A0F16FA178A589A59AA50E94EEB089
:107A40008EE296E00E945E3467966CAD7DAD8EADA1
:107A50009FAD67970E94EEB088E296E00E945E3488
:107A600043E0C501B4010E9438B380E20E943D3476
:107A700081E03DA133300CF480E0E12C8E010F5DFC
:107A80001F4F9E01235E3F4FAE01475E5F4FBE0119
:107A90006B5E7F4F04DC8AE00E943D3489A98F5FD2
:107AA00089AB7ACD0E94CC278DE196E00E945E34AE
:107AB00081E09DA119160CF080E0EE24E3948E0184
:107AC0000F5D1F4F9E01235E3F4FAE01475E5F4F2C
:107AD000BE016B5E7F4FE3DB698D7A8D8B8D9C8D54
:107AE0000052110926E042E00E94E4E29F938F9346
:107AF0008CE096E09F938F9386E196E09F938F931F
:107B00001F920E94FEA10E94AB8629968FAD2997F5
:107B10000E941E2A0E94DF8746CC8F929F92AF92CE
:107B2000BF92EF92FF920F931F93CF93DF9383EC5B
:107B300094E00E945E34C0E0D7E0D15021F080E2B2
:107B40000E943D34FACF8C2F0E94DB1DCF5FC730DF
:107B500099F78AE00E943D340EE914E0C0E080E22B
:107B60000E943D348C2F0E94DB1D7801D7E080E21B
:107B70000E943D34F70180809180A280B38020E094
:107B800030E0A901C501B4010E94C4F087FD03C023
:107B90008BE20E943D3443E0C501B4010E9438B33A
:107BA000D150FCE1EF0EF11CD111E1CF8AE00E942F
:107BB0003D34CF5F0C5F1F4FC73089F68AE00E94CB
:107BC0003D34DF91CF911F910F91FF90EF90BF90C7
:107BD000AF909F908F900895811107C08EE99EE02D
:107BE0000E945E348AE00C943D3482EA9EE0F8CF35
:107BF0008CEB94E00C945E3486EB94E00C945E3451
:107C0000CF9384E50E94121AC0E08823F1F00E940D
:107C1000011EC82F1816CCF4EFDF8DE40E943D340E
:107C200080911F04909120040E94F92B81E999E032
:107C30000E945E346C2FCC0F770B880B990B0E943F
:107C4000EEB08AE00E943D34CFEF8C2FCF910895A3
:107C5000CF93C82F67E978E00E946EC4C11101C0BC
:107C6000CBDF409198125091991260919A127091C5
:107C70009B128EE898E00E94803420E030E543ECCF
:107C800050E460919C1270919D1280919E1290918F
:107C90009F120E946CE8AB01BC018BE898E00E9447
:107CA00080342CEA35EC47E25EE36091A0127091DB
:107CB000A1128091A2129091A3120E946CE8AB01D4
:107CC000BC0188E898E00E9480348AE00E943D343C
:107CD000CF910895B0E0A0E0E0E7FEE30C94F7EE6A
:107CE00061E083E50E942B1EC1E0C82764E879E0CB
:107CF0008C2F0E946EC4C11101C07EDF8CE799E019
:107D00000E945E348FED9FE00E945E348AE00E9404
:107D10003D346AE679E08C2F0E946EC4C11101C027
:107D20006BDF8DE499E00E945E348C2F0E948EC43C
:107D30008C2F57DA8C2F7CDA8C2F33DA8C2FFDD9ED
:107D400066ED78E08C2F0E9485C4D09199048DEC6B
:107D500098E00E945E346D2F70E090E080E00E9419
:107D6000EEB040919A0450919B0460919C047091F4
:107D70009D048FE19FE20E94803480EC98E00E9495
:107D80005E348091990428DF20E030E0A901609101
:107D90006A0570916B0580916C0590916D050E944C
:107DA00007E8882399F18EE9E82E84E0F82E10E0A8
:107DB000670100E0C11101C01FDF83E499E00E9468
:107DC0005E34802F0E94DB1D80E499E00E945E34C7
:107DD000812F0E94DB1D8FE19FE20E945E34F6013D
:107DE000608171818281938145E00E9438B38AE08D
:107DF0000E943D340F5FFCE1CF0ED11C0730D1F65D
:107E00001F5F84E0E80EF11C173091F667EF78E011
:107E10008C2F0E946EC402E715E0D0E0C11101C0B2
:107E2000EBDE8EEE98E00E945E348D2F0E94DB1D0B
:107E3000F80160817181072E000C880B990B0E945C
:107E40000DE8AB01BC018BEE98E00E948034F80194
:107E5000E280F38088EE98E00E945E34C7010E94C1
:107E6000F92B8AE00E943D340C5F1F4FD13071F531
:107E70008C2FEEDE8C2F0E94913469E279E08C2FFA
:107E80000E9485C4C0915B0180E299E00E945E344B
:107E90006C2F70E090E080E00E94EEB040915701BE
:107EA000509158016091590170915A018DE199E00A
:107EB0000E94803482E199E00E945E3480915B01EF
:107EC0008BDECDB7DEB7E8E00C9413EFD1E0A6CFA0
:107ED000CF93DF93EB010E945E34BE01DD0F880B70
:107EE000990B0E94EEB0DF91CF9108950E945871D6
:107EF0000E94448C80912D07813099F079DE8FE3C8
:107F000094E00E945E3460E085E394E00E941BA24E
:107F10006EE571E080E090E00E94D42B81E08093D8
:107F20002D070895CF92DF92EF92FF921F93CF9388
:107F3000DF9300D000D0CDB7DEB78EEEC82E82E042
:107F4000D82EE12CF12CC982DA82EB82FC82BE01B0
:107F50006F5F7F4F8AE50E94053381110EC010E0EC
:107F6000812F0F900F900F900F90DF91CF911F9165
:107F7000FF90EF90DF90CF9008950E946733C98201
:107F8000DA82EB82FC82BE016F5F7F4F8AE50E943E
:107F90000533182F882319F32BDE89E195E00E9421
:107FA0005E34A4DFDDCFCF92DF92EF92FF921F937A
:107FB000CF93DF9300D000D0CDB7DEB78EEEC82EC2
:107FC00082E0D82EE12CF12CC982DA82EB82FC828D
:107FD000BE016F5F7F4F8AE00E94053381110EC0A2
:107FE00010E0812F0F900F900F900F90DF91CF91A5
:107FF0001F91FF90EF90DF90CF9008950E9467331C
:108000000E9422330E9439330E942233C982DA82CD
:10801000EB82FC82BE016F5F7F4F8AE00E940533D6
:10802000182F8823E9F2E4DD8CED94E00E945E34A1
:108030005DDFD7CFEC018B01F42E0E9458712097A1
:1080400009F47CC0D9DDCE010E945E348AE00E9432
:108050003D340115110511F406E71EE20E94BC1E15
:108060001F930F93DF93CF9385E094E09F938F93BB
:1080700081E08F930E94FEA10E94B58EC0915213A1
:10808000C695C6958DE493E10E945321DC2FDD0F48
:108090001D2F1C0F8DB79EB707960FB6F8949EBF85
:1080A0000FBE8DBF83E00E941A2010928813C093E8
:1080B000891382E290E10E94602510928813D09388
:1080C00089136FEF7FEF86EF93E00E940B241092ED
:1080D0008813109389136FEF7FEF89EE93E00E946E
:1080E0000B2481E593E10E9461D18111DBCF80DD1A
:1080F00085E194E00E945E3489EE93E0019739F0C7
:1081000000C00000EEE5F9E03197F0F7F7CFF89402
:1081100089EE93E0019739F000C00000E6EEF3E04D
:108120003197F0F7F7CF0E945871FF2021F00E949D
:10813000A473A895FECF0E945F73FBCF01151105B4
:1081400011F406E71EE2CCE0D4E088CF8091960DD2
:108150009091970D2FEF3FEF981751F0E92FF0E036
:10816000EA56F24F228130E09F5F9F779093970D00
:10817000C90108951F920F920FB60F9211240F900C
:108180000FBE0F901F9018951F920F920FB60F926F
:1081900011240BB60F922F938F939F93EF93FF931E
:1081A0009091C6002091970DE091960D81E08E0F81
:1081B0008F77281729F0F0E0EA56F24F9283E82FE4
:1081C000E093960DFF91EF919F918F912F910F90DA
:1081D0000BBE0F900FBE0F901F9018958EBD0DB463
:1081E00007FEFDCF08958FEF8EBD0DB407FEFDCFC6
:1081F0008EB50895909164009B7F90936400982FB2
:10820000906A96959CBD80FD03C091E0863009F48C
:1082100090E09DBD0895A8E0B0E0E1E1F1E40C94A8
:10822000EDEEB82E80917F0E843008F0F6C131E675
:10823000D32E80917F0E843008F021C18091960D5D
:108240009091970D891B8F7709F419C17FDF97FFF4
:108250000AC0CEDC81E393E00E945E348091960DEB
:108260008093970DE6CF8A3019F08D3009F0FEC06B
:1082700010927E0E80911C0E90911D0EFC01E85E06
:10828000F14F1682892B19F40E94E171D2CF10921E
:108290001D0E10921C0E0EE11EE0F801819180323D
:1082A00009F446C08E3409F09DC06CE273E0C80149
:1082B0000E9486E77C01892B41F06EE470E0C801E2
:1082C00004960E94B9F1009709F4C8014AE050E011
:1082D00070E060E001960E94FBE42B013C0180917C
:1082E000180E9091190EA0911A0EB0911B0E0196C6
:1082F000A11DB11D481659066A067B0629F060E0EB
:1083000089EF92E0EF2851F16AE270E0C8010E9423
:10831000E8F19C01009729F1982F901BF12C9923EB
:1083200049F09150F801E90FF11D8081F826F7CF4F
:108330008F01B3CF4AE050E070E060E0C9010196E0
:108340000E94FBE42F2D30E050E040E062177307FD
:108350008407950751F060E08AED92E00E94D8C34F
:1083600068CF60E080EB92E0F9CF4092180E509217
:10837000190E60921A0E70921B0E80912D0781309B
:10838000E1F467E470E0C8010E94B9F10097A9F038
:108390004AE050E070E060E001960E94FBE4623049
:1083A00071058105910548F48FE092E00E945E34EA
:1083B00060E085E092E00E941BA2F80180818D348C
:1083C00081F58381823309F445C0883301F180331C
:1083D00041F58181843329F58281813311F50E9431
:1083E000BB871FC08091A31480FFC7CF6FE17EE2DF
:1083F000C8010E9486E7009731F0FC018381805319
:108400008A3008F0BACF60E086E892E0A7CF828198
:10841000803339F48181813321F410926B01109201
:108420007E0480911E0E8B3309F403CF80917F0E62
:10843000843008F0FECE8091810E8D9DC001112404
:108440006EE17EE08E57914F0E94C4F180E00E9461
:1084500098C3EFCE8281813321F78181813309F77F
:1084600041E070E060E086E19BE0E4DD2CE13EE08D
:108470004EE15EE06EE77EE00E941D19DACE80914B
:10848000A31483FDCAC082FFC8C087FDC6C01A827C
:10849000198281E6F82E94E0E92E29E6D22E809109
:1084A0007F0E843008F0B9C00E9455198111B5C003
:1084B00041E050E0BE016D5F7F4F86EA92E10E948D
:1084C000DCD70B8110E0019711F00FEF1FEF8091C7
:1084D000AE129091AF12A091B012B091B1128093F0
:1084E0009F149093A014A093A114B093A2140E947F
:1084F00055190F3F100741F4811106C079DB89E45B
:1085000093E00E945E34CBCF4091810E242F30E067
:108510000A3061F00D3051F0882309F470C0898170
:108520009A81009719F001969A8389831092A90382
:1085300089819A81F29EF001F39EF00D1124E15899
:10854000F14FDF01A80FB91F13961C92892BA9F5D3
:108550000E94E1710E945519882309F4A0CF86EA90
:1085600092E10E94106D80919A148823F1F181505C
:1085700080939A148D9DC001112462E08558994F13
:108580000E94E3D9E0919A1424E0E29FF0011124C3
:10859000E958F94F408151816281738140939F1462
:1085A0005093A0146093A1147093A21486EA92E1F0
:1085B0000E94E1D60E94BCD272CF1A8219828381B6
:1085C0008D3479F48481823361F48581853349F473
:1085D000868180538A3028F08091A3148B7F80930A
:1085E000A31481E00E9498C3B5CF0E94AED28091BF
:1085F000A31488608093A314E0922D0750CF4F9D61
:10860000A00111244E57514F9E012F5F3F4F69EA41
:1086100073E0802F0E941D1942CF0E9450CE6B0143
:108620007C01BB2041F0C0922204D0922304E0924E
:108630002404F09225048091F9039091FA03A0910B
:10864000FB03B091FC030097A105B10529F140910E
:108650002204509123046091240470912504840F16
:10866000951FA61FB71FA7019601281B390B4A0BA0
:108670005B0BDA01C901B7FD0FC0BADA60916C0774
:1086800070916D0788E593E00E94A0D240E070E011
:1086900060E090E080E0E9CE8091190190911A01AC
:1086A000A0911B01B0911C01892B8A2B8B2B79F097
:1086B0009091391380913A13981709F4C4C0C0926D
:1086C0002204D0922304E0922404F09225048091A5
:1086D000AE039091AF03A091B003B091B1034601F6
:1086E0005701881A990AAA0ABB0AD501C401B7FD25
:1086F000C0C19091391380913A13209108019817C5
:1087000009F4D5C0E0913A133BE5E39FF001112451
:10871000EF50F84F8081281799F0809308010E944C
:1087200050CEB09008010B2D10E084E00E9419B3E8
:108730000115110509F0BEC060E084E00E946BCD18
:1087400080918905882309F487C100912F01109138
:108750003001C80102972091951230919612281786
:1087600039070CF479C180903A138C82812C912CBA
:108770005401809139132C81821709F4FDC0822F96
:1087800090E03BE5389FF001399FF00D1124E5564C
:10879000F84F458956896789708D452B462B472BA5
:1087A00081F4418D528D638D748D452B462B472B63
:1087B00041F4458D568D678D70A1452B462B472B77
:1087C000E9F14BE5489F9001499F300D1124C90103
:1087D0008556984F1C01FC016181728183819481CF
:1087E0000E9403F16D837E838F839887F10161A1DD
:1087F00072A183A194A10E940BE82B013C01F1011D
:1088000065A176A187A190A50E940BE89B01AC0110
:10881000C301B2010E949FEF2D813E814F81588597
:108820000E946CE82B013C01AC019B01C501B40125
:108830000E94C4F087FF02C0530142018C818F5F08
:108840008F708C8396CFBB2019F01092B2033FCF6C
:108850000E9450CE00912204109123042091240400
:10886000309125048090190190901A01A0901B016D
:10887000B0901C01080D191D2A1D3B1D601B710BBA
:10888000820B930B97FDE1CF8091B20381111FCF33
:1088900081E08093B20380E00E94747381E00E94C3
:1088A000747382E00E9474730E945F7310CF809192
:1088B0008A0731CF0F3F110511F461E03ECFEAE5A1
:1088C000FEE2E491E150EA3008F051C0F0E0E559F1
:1088D000FB4B0C94D2EE75447A447F448944B744F0
:1088E000B74493449B44A344AD4484B5806884BD9D
:1088F000B7BC26CF84B5806284BDB8BC21CF80913F
:108900008000806880938000109389000093880025
:1089100017CF8091800080628093800010938B003D
:1089200000938A000DCF8091B00080688093B000E2
:10893000B092B30005CF8091B00080628093B00008
:10894000B092B400FDCE809190008068809390003A
:108950001093990000939800F3CE8091900080626C
:108960008093900010939B0000939A00E9CE00380A
:1089700011050CF0A2CFE0CEB801110F880B990BB6
:108980000E940DE82B013C012091290130912A0120
:1089900040912B0150912C01C501B4010E946CE85B
:1089A000A30192010E9425EF4B015C0100912D0172
:1089B00010912E01AC019B01C301B2010E94C4F0D1
:1089C00018168CF0B801012E000C880B990B0E9430
:1089D0000DE82B013C01A50194010E9407E818163F
:1089E00014F4240135018090AA039090AB03A09069
:1089F000AC03B090AD03A3019201C501B4010E9484
:108A0000C4F01816D4F420E037ED43EA5CE3C30168
:108A1000B2010E946CE82B013C0128E431EE4AE7E8
:108A20005FE3C501B4010E946CE89B01AC01C30186
:108A3000B2010E9425EF2B013C014092AA03509203
:108A4000AB036092AC037092AD03C301B2010E940C
:108A500007F0CB010E9491CEF4E6CF0ED11CE11CB1
:108A6000F11CC092AE03D092AF03E092B003F0923B
:108A7000B1030E94E17180912D07882309F406C19A
:108A800080915B01882391F18091B80381112EC000
:108A90000E94FE2B882351F1F89480B182FB882735
:108AA00080F99091B30398278093B3038091840554
:108AB000892B809384056091800570918105809158
:108AC000820590918305789420E030E0A9010E940E
:108AD00007E887FF0BC081E08093B80385E993E046
:108AE0009093EB068093EA060E942C741091090182
:108AF000113061F18091A31480648093A31481E00C
:108B00008093090164EF71E080E090E00E94D42B33
:108B10000E94D1D48091A31484FFD0C0123028F4D5
:108B200060E089E993E00E941BA283E080936C01DE
:108B30000E9450CE6C597F4F8F4F9F4F60937304AC
:108B40007093740480937504909376040E9450CEC1
:108B50006B017C01109118011123F1F08091FE034B
:108B60008823D1F04091B4035091B5036091B603CE
:108B70007091B70346015701841A950AA60AB70AED
:108B8000B501A40177FD1AC0833009F492C00CF03E
:108B900081C081300CF086C0212F30E0A8EEB3E018
:108BA0000E9483EEC60ED71EE81EF91EC092B403C3
:108BB000D092B503E092B603F092B7030E948621EB
:108BC0008091F803882379F10E9450CE6B017C01DB
:108BD0008091F4039091F503A091F603B091F7030F
:108BE000A7019601281B390B4A0B5B0BDA01C9015F
:108BF000B7FD19C02091F80330E0A8EEB3E00E9461
:108C000083EEC60ED71EE81EF91EC092F403D09262
:108C1000F503E092F603F092F70380E00E94CD7036
:108C20008AE00E943D348091F303882379F10E9409
:108C300050CE6B017C018091EF039091F003A091E5
:108C4000F103B091F20346015701881A990AAA0A62
:108C5000BB0AD501C401B7FD19C02091F30330E070
:108C6000A8EEB3E00E9483EEC60ED71EE81EF91EE2
:108C7000C092EF03D092F003E092F103F092F2037E
:108C80000E94A5B38BE393E10E94A6722896E2E1CD
:108C90000C9409EF843009F07FCF0E94FC3D88EAF4
:108CA00093E004C00E94FC3D87ED93E00E945E3497
:108CB00073CF0E94FC3D80EC93E0F8CF112309F4C0
:108CC00045CF33CFA2E1B0E0E8E6F6E40C94EEEE57
:108CD00090914B0D93FD7FC0082F0E94003E182FEE
:108CE00087FD79C089E40E94121A882309F48BC099
:108CF0000E94011E282F30E01216130614F421E002
:108D000030E0220F331F220F331FF901EE58FA4FC4
:108D100080819181198A0E9491CE809195129091C3
:108D200096128635910574F0002381F00E94FC8B29
:108D30000DC082E50E94121A882309F46CC00E94BB
:108D40003C1EE9CF0E94448C0E9409C56091951297
:108D500070919612072E000C880B990B0E940DE85B
:108D6000209191123091921240919312509194124D
:108D70000E94C4F0181644F0298980E090E1222373
:108D800029F049894A8B48C08BE090E19F938F93EB
:108D900086E190E19F938F931F920E94FEA10F9016
:108DA0000F900F900F900F9031E03A8B35C060E03C
:108DB00070E0CB014FC0C701B6010E9407E887FFF2
:108DC0000EC080916B01882321F010926B010E94EC
:108DD00009C5309289056296E1E10C940AEF4601DB
:108DE000570100E098C08FE30E943D34CFC020E0DF
:108DF00030E040E450E40E94C4F018160CF004C1C6
:108E00002601370101C183E50E94121A898B811165
:108E100096CF01118ECF1A8A83E50E94121A8823F9
:108E200031F00E943C1E9093300180932F0182E428
:108E30000E94121A882331F00E943C1E90932E014A
:108E400080932D0186E40E949B19882309F4AFCFFB
:108E50000E944B1E6093290170932A0180932B017D
:108E600090932C013324339420E030E0A9010E9438
:108E700007E8811101C0312C30928905002309F4E3
:108E8000AACF5A89552309F4A6CF1092890581E00B
:108E900080936B011D821E821F82188619861A8696
:108EA0001B861C8680E09CE3ACE1B6E48D879E8740
:108EB000AF87B88B812C912C90E8A92E9FEBB92E0F
:108EC00000E0412C512C3201609195127091961264
:108ED000072E000C880B990B0E940DE86B017C019A
:108EE000A50194010E9407E88823A9F0209191121E
:108EF000309192124091931250919412998991114C
:108F00005ACFC701B6010E9407E8082F001F0027AB
:108F1000001F460157010E9450CE6B017C01DC010D
:108F2000CB0129853A854B855C85821B930BA40B6D
:108F3000B50BB7FD2EC0D701C60188519C4FAF4F6E
:108F4000BF4F89879A87AB87BC87812F0E94CD70DE
:108F50008CE190E10E945E3441145104610471047B
:108F600009F441CFC301B201605F784D8F4F9F4F2D
:108F70006C197D098E099F0928EE33E040E050E02E
:108F80000E9435EECA01B9010E9468268AE00E945B
:108F90003D3480E040D90E9450CE6093220470930B
:108FA00023048093240490932504209191123091FE
:108FB0009212409193125091941229833A834B83D9
:108FC0005C83C501B4010E9424EF9F7741145104D2
:108FD0006104710409F00BCF20E030E040E85FE36A
:108FE0000E9407E887FF10C03A89412C512C3201BA
:108FF000332331F085E0482E8DE0582E612C712C02
:109000004C0C5D1C6E1C7F1C0023C1F18D819E8168
:10901000AF81B885892B8A2B8B2B61F0D701C601D4
:109020002D813E814F815885821B930BA40BB50B7C
:10903000B7FD24C029813A814B815C816D857E8595
:109040008F8598890E9424EF20E030E040EC5FE3B8
:109050000E9407E887FDB5CED701C601805A954129
:10906000AF4FBF4F8D839E83AF83B88729813A81ED
:109070004B815C812D873E874F87588B80916B0198
:10908000882309F49ECE411451046104710461F0F7
:1090900030E1C31A37E2D30AE108F108C418D50851
:1090A000E608F708F7FE8DCE1A8A0ECFA5E4B0E0E9
:1090B000ECE5F8E40C94EDEE26968FAF2697209120
:1090C000FE0328AB81E08093FE03809121048D3460
:1090D00009F48CC3843511F40C94755C873491F4D5
:1090E00080911F04909120048D31910509F4FBC1FA
:1090F00008F082C08430910509F4A2C130F40297CF
:1091000008F4FBC00E9458C473C18531910509F46D
:109110006FC14C97B9F787E00E943E83811111C05F
:109120008091190490911A04A0911B04B0911C0421
:10913000EEE0B695A79597958795EA95D1F780FDCE
:1091400057C10E942C7410923C01609199048CE4E8
:109150000E942B1E982E80E00E941E2A0E9450CE54
:109160006093220470932304809324049093250435
:109170000E94C48681E08093E6060E94D088C09059
:109180001904D0901A04E0901B04F0901C0479E1BB
:10919000F694E794D794C7947A95D1F7C0FE0DC0A2
:1091A00081E00E943E83182F82E00E943E831111CD
:1091B0000C94225E11E0811101C010E0809119042D
:1091C00090911A04A0911B04B0911C0467E1B6951C
:1091D000A795979587956A95D1F780FF02C00C9463
:1091E000985C112311F40C949B5CA12E10E04C2D83
:1091F0004170B42E0C94B45C8A35910509F4E7C231
:1092000050F58E31910509F471C18A9709F07ACF32
:1092100080912D07833008F4EBC089E40E94121A74
:10922000082FF12C882319F00E943C1EF82E8AE4A6
:109230000E94121AE82E882309F4C7C10E943C1E1E
:10924000182F0111C5C1173008F4C8C182EE99E08A
:109250000E945E34CDC08B35910509F4BBC28C35BC
:10926000910509F04FCF47E9242E41E0342E57E70E
:10927000E52E51E0F52EC12CD12C10E0F1018191A9
:109280001F010E94121A082F882349F10E944B1EC9
:109290002B013C01D7012D913D914D915C910E9494
:1092A00024EF4B015C012DEB37E346E855EB0E94C0
:1092B00007E887FD0AC02DEB37E346E855E3C50113
:1092C000B4010E94C4F0181654F4133011F0C02EEB
:1092D0000D2DF7014082518262827382D02E1F5F72
:1092E000F4E0EF0EF11C143049F6CC2009F476C2FC
:1092F0000E9491870E94DF877BC080912D07833079
:1093000008F476C0F9E8CF2EF4E0DF2EA7E7EA2EC6
:10931000A1E0FA2E10E088E5810F0E94121A88233E
:1093200009F472C00E944B1E4B015C01812F0E9408
:109330007419882359F0D7012D913D914D915C917D
:10934000C501B4010E9425EF4B015C01F60180824A
:109350009182A282B3821F5FF4E0CF0ED11C24E081
:10936000E20EF11C1330B9F685E40E94121A88232C
:1093700009F455C00E944B1E6B017C0183E00E94E2
:109380007419882371F020918301309184014091F8
:10939000850150918601C701B6010E9425EF6B013E
:1093A0007C01C0929504D0929604E0929704F092CA
:1093B000980440E050E0BA0186E40E94731E20E069
:1093C00030E0A9010E94C4F0181684F40E944B1EDC
:1093D00029E838E848E85CE30E946CE860933501CE
:1093E0007093360180933701909338010E949C83DB
:1093F00026969FAD2697911102C00E9445C4A8A948
:10940000A093FE030C941C53F70180819181A281EB
:10941000B381F60180839183A283B3839CCF809133
:10942000830190918401A0918501B0918601809380
:10943000950490939604A0939704B0939804B9CFA1
:1094400080E50E94121AC12CD12C7601882321F0CC
:109450000E94E11D6B017C0183E50E94121A8823A2
:1094600061F00E944B1E20E030E04AE754E40E9485
:109470006CE80E940CF06B017C010E942C748091BE
:109480002210811105C060E084EA99E00E941BA2CD
:109490000E9450CEC60ED71EE81EF91E0E9450CE66
:1094A0006C197D098E099F0997FFA2CF80E00E9469
:1094B0000B41F4CF60E070E080EA90E40C94BD5C76
:1094C000A3019201C701B6010C94095D60E08FEB26
:1094D00099E00E941BA20E94FC3D8DEA99E00E9447
:1094E0005E340C94FA5D0E947E5E82CF009134134C
:1094F00010913513F80120813181428153816091AF
:109500007701709178018091790190917A010E94A0
:1095100025EFAB01BC0188E50E94731E69837A8345
:109520008B839C83D80114962D913D914D915C9134
:10953000179760917B0170917C0180917D019091E2
:109540007E010E9425EFAB01BC0189E50E94731EDC
:109550006D837E838F839887BE016B5F7F4FCE01C3
:1095600001960E944BC5882309F442CF80E00E94F7
:109570001E2A0E94C48661E085E40E942B1E21E021
:10958000482FBE016B5F7F4FCE0101960E9481C6BE
:109590006B017C0149815A816B817C818AED99E064
:1095A0000E9480344D815E816F81788585ED99E0E0
:1095B0000E948034B701A60180ED99E00E94BF347B
:1095C0000E94AB860E94DF8713CF10E0002331F0AA
:1095D000B6E0BF1508F43ACEE11035CE80E1E7E7FA
:1095E000F1E0A9E8B4E001900D928A95E1F700233B
:1095F00019F16F2DFF0C770B880B990B0E940DE86A
:1096000020916A0530916B0540916C0550916D0574
:109610000E946CE8209162053091630540916405D9
:10962000509165050E9425EF6093890470938A0428
:1096300080938B0490938C04EE2019F1612F110F0D
:10964000770B880B990B0E940DE820916E053091E5
:109650006F0540917005509171050E946CE8209152
:1096600066053091670540916805509169050E9433
:1096700025EF60938D0470938E0480938F049093F4
:10968000900460E080E50E942B1E8823C1F1002336
:10969000D1F0E0913413F091351320813181428172
:1096A00053816091890470918A0480918B04909118
:1096B0008C040E9424EF6093890470938A04809341
:1096C0008B0490938C04EE20D1F0E0913413F09150
:1096D0003513248135814681578160918D047091C5
:1096E0008E0480918F04909190040E9424EF6093E7
:1096F0008D0470938E0480938F049093900440E0C7
:1097000050E0BA0186E40E94731E6B017C0120E0E8
:1097100030E0A9010E94C4F087FF03C0C12CD12C06
:10972000760129E838E848E85CE3C701B6010E9401
:109730006CE86B017C018090350190903601A0901F
:109740003701B090380120E030E0A9010E9407E81D
:10975000882341F0C0923501D0923601E092370162
:10976000F09238010091390110913A0184E690E0BD
:1097700090933A0180933901C0907101D0907201A9
:10978000E0907301F090740180E090E0A0E8BFE306
:109790008093710190937201A0937301B09374014F
:1097A0000E949C838092350190923601A0923701ED
:1097B000B092380110933A0100933901C0927101BF
:1097C000D0927201E0927301F092740111CE109266
:1097D000FD030ECE8FE08093FD030ACEDD2009F459
:1097E00089CD83E891E00E94958184CD80911F040A
:1097F000909120048237910511F40C94385508F0AB
:109800006FC18B34910509F4EFC608F0E9C08831C7
:10981000910509F40FC508F0BAC08231910509F429
:10982000F6C708F06EC08230910508F479C44197FC
:1098300009F068CC0E948A19882309F4CDC40E94DB
:10984000E91900917B05102F1095182309F4D0CD4C
:10985000F12CE12CD12CA12EB12CC5010E2C02C073
:10986000959587950A94E2F780FF08C08E2D0E9497
:10987000AB73F701EC5DFD4F8081D82A8FEFE81ABA
:10988000F80A93E0E916F10441F713FF05C00E94BE
:109890006D73AD2DA360DA2E102B10951D2109F4E8
:1098A000A7CD88E20E943D34F12CE12CC12ED12CB1
:1098B000C6010E2C02C0959587950A94E2F780FFA9
:1098C00009C0F701E956FE4F80810E943D3480E2D5
:1098D0000E943D34BFEFEB1AFB0AE3E0EE16F10401
:1098E00039F713FF09C085E40E943D3480E30E94EC
:1098F0003D3480E20E943D348EE09AE00E945E3466
:1099000077CD8531910509F47FC458F5449709F066
:10991000F9CB8091A31484FF70C48FE39AE00E9476
:109920005E348091A31484FF17C08CED92E10E94F5
:109930003F6E8BE1ECEDF2E1DE01119601900D92AC
:109940008A95E1F770E060E0CE0101960E9415DB98
:10995000CE0101960E940F7080E39AE00E945E346F
:1099600047CD8631910509F452C4479709F0CACB17
:1099700080911D0490911E04FC012191222309F481
:1099800055C42032D1F7DF0111971C92F6CF8D31EB
:10999000910509F4DDC4A0F48A31910509F463C48A
:1099A00008F453C48B31910509F478C44C9709F03D
:1099B000A9CB80911D0490911E040E9497D918CDC7
:1099C0008F31910509F46AC508F4C8C48032910545
:1099D00009F41FC5C09709F095CB0E94BC3908CD8A
:1099E0008836910509F40CC608F046C08235910509
:1099F00009F4FDC6F0F48D34910509F4FDC508F4B1
:109A0000F7C58135910509F07DCB0E943D74109218
:109A10008A070E9458710E94448C68EE73E080E0CF
:109A200090E00E94D42B60E08BE29BE00E941BA29E
:109A3000DFCC8435910509F4EAC608F4E0C6853523
:109A4000910509F47EC78C35910509F05BCB0E9426
:109A5000003E87FDCDCC8091190484FD97C780918D
:109A60001B0487FD93C780911C04837009F08EC787
:109A700081E00E948EC4BCCC8D36910509F4C5C529
:109A800098F48A36910509F4DCC508F4C3C58B3611
:109A9000910509F40FC68C36910509F033CB10926D
:109AA0007E0410926B01A4CC8F36910509F420C678
:109AB00008F40BC68037910509F456C68137910525
:109AC00009F020CB83E50E94121A882309F458C6B6
:109AD0000E94011E8D3308F04EC68093180188CC79
:109AE0008D3221E0920711F40C94A35808F0F4C1D0
:109AF0008B39910509F454C608F0F4C087379105F5
:109B000011F40C94895508F0BAC08537910509F411
:109B1000B7C708F0C5C78337910509F0F3CA87EFC7
:109B20009CE00E945E3460E087EE9CE00E946B3413
:109B300060E082ED9CE00E946B3461E08BEC9CE085
:109B40000E946B3460E080EC9CE00E946B3461E02A
:109B500081EB9CE00E946B3461E081EA9CE00E9412
:109B60006B3460E088E99CE00E946B3461E08EE831
:109B70009CE00E946B3461E084E89CE00E946B34BE
:109B800061E08DE79CE00E946B3461E085E79CE03A
:109B90000E946B3461E087E69CE00E946B3460E0D9
:109BA00089E59CE00E946B3460E08AE49CE00E94BE
:109BB0006B3460E08CE39CE00E946B3460E086E2F2
:109BC0009CE00E946B3460E085E19CE00E946B3475
:109BD00060E080E09CE00E946B3460E081EF9BE0FD
:109BE0000E946B3461E08AEE9BE00E946B3460E07F
:109BF00083EE9BE00E946B3461E08AED9BE00E9463
:109C00006B3460E085EC9BE00E946B3460E087EB96
:109C10009BE00E946B3460E08AEA9BE00E946B3418
:109C200061E087E99BE00E946B3460E08AE89BE09A
:109C30000E946B3460E085E89BE00E946B3461E039
:109C400088E79BE00E946B3460E084E69BE00E9422
:109C50006B3460E081E59BE00E946B3460E082E859
:109C600092E10E947119682F617088E49BE00E9464
:109C70006B3460E08AE39BE00E946B34B9CB893798
:109C8000910509F453C708F448C78139910509F4CF
:109C900055C78A39910509F035CA83E50E94121A21
:109CA000882309F4A5CB0E94011E182F8C3308F0DD
:109CB0008CE38093F3030E9450CE6B017C01212F33
:109CC00030E0A8EEB3E00E9483EEC60ED71EE81E79
:109CD000F91EC092EF03D092F003E092F103F092EC
:109CE000F20386CB833D910511F40C940257C0F525
:109CF0008B3C910509F4A1C7B0F4893C910509F0AA
:109D000001CA8091190484FD6EC780911B04887874
:109D100009F069C780911C04837009F064C781E071
:109D20000E94183965CB8C3C910509F4BAC78D3C6B
:109D3000910509F0E7C98091190481FF02C00C94D4
:109D4000A65680911A0481FF02C00C94A6568091F9
:109D50001B048C7009F0FAC781E00E949D3848CB43
:109D60008D3D910511F40C94965708F045C08C3D3B
:109D7000910509F0C7C982E40E949B19882341F02C
:109D80008091390190913A0190931E0180931D01B9
:109D900082E50E949B19882341F080911D019091DA
:109DA0001E0190933A018093390183E50E94121AB3
:109DB000882331F00E943C1E90933A018093390130
:109DC0008091190490911A04A0911B04B0911C0475
:109DD000892B8A2B8B2B09F00BCB60913901709169
:109DE0003A0184E29EE00E94683F85E20E943D3491
:109DF0008AE00E943D34FCCA883141E0940711F4A6
:109E00000C94E3578232914009F07CC98AE50E94A4
:109E1000121A882311F40C947E580E944B1E20E0E5
:109E200030E040E050EC0E94C4F0C12CD12CE12C79
:109E300050ECF52E87FD13C00E944B1E20E030E051
:109E400040E050E40E9407E8C12CD12CE12C40E412
:109E5000F42E181624F00E944B1E6B017C012091F9
:109E6000680D3091690D40916A0D50916B0DC701DD
:109E7000B6010E946CE80E9407F0CB010E942CC53D
:109E800061E080E50E942B1E882311F40C94845815
:109E9000A7019601609130137091311380913213B4
:109EA000909133130E9425EF609330137093311318
:109EB00080933213909333130E94FC3D40913013F2
:109EC00050913113609132137091331380E69EE00C
:109ED0000E94BF340C948458843FA1E09A0711F487
:109EE0000C946C5B08F0ADC08239E1E09E0711F480
:109EF0000C943B59F0F48F3221E0920711F40C944A
:109F0000335910F40C94ED58803941E0940711F462
:109F10000C9437598139914009F0F4C883E50E94C7
:109F20009B19811165CA81E00E94DF890E94DF8749
:109F30005FCA8C39A1E09A0711F40C94415938F4A6
:109F40008A39914009F0DEC80E94BB8751CA843A21
:109F5000F1E09F0711F40C94A959853A914009F05A
:109F6000D1C86FEF7FEF89E40E943F1E8C016FEF35
:109F70007FEF8AE40E943F1E7C018AE50E94121A4C
:109F8000D12C811108C081E50E94121AD82E882395
:109F900011F40C941A5EC02E81E0800F883010F00E
:109FA0000C94645BBE2C81E08E0D883010F00C9414
:109FB000645B102F0E944B1E2B013C01A02E07FD5D
:109FC000A12C17FF02C046E0C42E8E2DE7FCE12C29
:109FD00087FF02C036E0B32E27E0322ECA1408F401
:109FE00007CAFE2C3A9C40011124BF1410F40C94B3
:109FF000615B0F2D10E020E030E0A901DD2069F069
:10A00000F401E00FF11FEE0FFF1FEE0FFF1FE256EE
:10A01000FB4F2081318142815381080D191D000FB2
:10A02000111F000F111F02561B4FC301B2010E94E6
:10A0300025EFD8016D937D938D939C931397F394A3
:10A04000D4CF8C3032E0930711F40C947C5B20F574
:10A05000863F51E0950711F40C94745B10F40C9456
:10A06000705B873FB1E09B0711F40C94785B883FED
:10A07000914009F047C881E080937A050E944A8F99
:10A0800010927A05882309F4B3C90E94FC3D8DE43F
:10A090009FE00E945E34ACC9803AF3E09F0709F468
:10A0A000EFC1A0F48335934009F02CC880911B04C4
:10A0B00087FF02C00C94945B80911C04837011F0A4
:10A0C0000C94945B81E00E94913492C9873E43E0F6
:10A0D000940711F40C94655C893E934009F012C812
:10A0E0000E942C748091A314877F8B7F8093A3148C
:10A0F0000E94AF8B6D3371058105910520F084ECD2
:10A100009FE00E94265E80EC9FE00E94265E8CEA23
:10A110009FE00E945E3488EA9FE00E94265E68C944
:10A1200080E50E94121AC12CD12C7601882321F0DF
:10A130000E94E11D6B017C0183E50E94121A8823B5
:10A1400061F00E944B1E20E030E04AE754E40E9498
:10A150006CE80E940CF06B017C010E942C748091D1
:10A160001D0490911E04009711F10E9493C210915A
:10A17000FE0383E08093FE0381E080937E04C1149C
:10A18000D104E104F10431F00E9450CEC60ED71E76
:10A19000E81EF91E80917E048823B9F0C114D10411
:10A1A000E104F10451F480E00E940B41F3CF60E040
:10A1B0008BEF99E00E941BA2DACF0E9450CE6C195F
:10A1C0007D098E099F0997FDEECF10927E041093B2
:10A1D000FE030E9409C50CC960E08DE19AE00E946F
:10A1E0001BA280E00E94AB7381E00E94AB7382E00F
:10A1F0000E94AB730E946D73FBC80E94FC3D86E217
:10A200009AE00E945E34F4C80E94D1D4F1C88091D3
:10A21000A31482FF02C087FFEBC80E94AED28091D8
:10A22000A3148F7E80648093A314E2C860E00E9430
:10A23000E3D9DEC80E94112C882321F00E94BCD2F1
:10A240000E94FC8B0E9409C5D3C88091A31482FF91
:10A2500005C087FD03C08B7F8093A3140E942F8CC1
:10A260000E9409C5C5C88091A31484FFC1C883E5B5
:10A270000E94121A882309F4BBC80E94F11DAB0189
:10A28000BC0140939F145093A0146093A114709349
:10A29000A21486EA92E10E94E1D6AAC8809119042C
:10A2A00090911A04A0911B04B0911C0432E0B69561
:10A2B000A795979587953A95D1F780FF1CC08DE7B4
:10A2C0009AE00E945E348091A912882379F0BE0141
:10A2D0006F5F7F4F86EA92E10E94336DCE01019657
:10A2E0000E9444348AE00E943D3482C880E59AE0AE
:10A2F0000E945E34F7CF8091A31482FF24C0C090E7
:10A300009F14D090A014E090A114F090A2148BE6BA
:10A310009AE00E945E34C701B6010E9491B08FE2BC
:10A320000E943D3460919B1470919C1480919D1407
:10A3300090919E140E9491B08DE00E943D348AE07D
:10A340000E943D3455C88AE59AE00E945E3450C8A8
:10A350008091A3148E7F8093A3144AC88091A31484
:10A3600084FF46C80E94CBD68091A31484FF40C8C6
:10A3700040911D0450911E04BE01645E7F4F80E039
:10A380000E94B8C28C01009709F432C86C8D7D8D93
:10A3900019821C8222E0AC01CE0101960E94147049
:10A3A000811115C0F12CCE0101960E940F70FF2083
:10A3B00019F1B80187EA9AE00E94A0D210929F1486
:10A3C0001092A0141092A1141092A21411C8CE01E0
:10A3D00001960E9466D7882329F361E0CE01019699
:10A3E0000E94196D0097F1F225EEDC012C931C827E
:10A3F0000E94F8D2F82ED7CF8FE89AE00E945E3400
:10A40000C8010E9444348CE89AE00E945E340C94A7
:10A41000F8498091A31482FF03C087FF0E942C7427
:10A420008091A31484FD02C00C94F84960E080E59B
:10A430000E942B1E182F682F80911D0490911E04DE
:10A440000E94E3D983E50E94121A882381F00E94BA
:10A45000F11DAB01BC0140939F145093A014609375
:10A46000A1147093A21486EA92E10E94E1D60E94A0
:10A47000BCD211110C94F8490E94FC8B0C94F84941
:10A4800020911D0430911E049091A314926090932A
:10A49000A314C9010E9497D90C94F8490E94AF8B6C
:10A4A0006B017C0120E831E541E050E00E9435EE8F
:10A4B000C9016DE671E00E94ABEE4B015C01C70182
:10A4C000B60120E13EE040E050E00E9435EECA01D6
:10A4D000B90128E130E040E050E00E9435EE2B0168
:10A4E0003C011B01C701B6012CE330E040E050E025
:10A4F0000E9435EE6B017C01CA01B9012CE330E00A
:10A5000040E050E00E9435EE8E010F5F1F4F811436
:10A51000910419F1DF92CF927F936F935F924F92E4
:10A52000BF92AF929F928F928DED9AE09F938F93FF
:10A530001F930F930E94A0E70FB6F894DEBF0FBEE3
:10A54000CDBFC8010E9493C20E94FC3DB80181EFBB
:10A550009AE00E94A0D20C94F849A114B10489F0A9
:10A56000DF92CF927F936F935F924F92BF92AF92A1
:10A570008DEC9AE09F938F931F930F930E94A0E717
:10A58000DBCF4114510479F0DF92CF927F936F9328
:10A590005F924F9281EC9AE09F938F931F930F935A
:10A5A0000E94A0E7C9CF6115710569F0DF92CF92D3
:10A5B0007F936F9389EB9AE09F938F931F930F93F1
:10A5C0000E94A0E7B9CFDF92CF9285EB9AE09F93EC
:10A5D0008F931F930F930E94A0E70F900F900F90FF
:10A5E0000F900F900F90ADCF0E94FC8B0C94F84908
:10A5F0000E942F8C0C94F8490E94448C0C94F849CA
:10A6000080E00E9462460C94F84981E00E94624614
:10A610000C94F8490E94003E182F87FD0AC08EEF67
:10A620009AE00E945E34812F0E94CD708AE00E94E1
:10A630003D3498A99093FE03CB5BDF4FE2E10C948D
:10A6400009EF60E080E50E94121E81110C94F84928
:10A650008091190490911A04A0911B04B0911C04DC
:10A6600060918A07062F10E080FD02C00FEF10E016
:10A6700089E40E94121A882311F40C940E5E0E9441
:10A68000011E90E01816190614F481E090E0880F7E
:10A69000991F880F991FFC01EE58FA4F0281138110
:10A6A0000F3F110519F010F00FEF10E000938A072B
:10A6B0000C94F84960E080E50E94121E81110C9410
:10A6C000F84910928A070C94F8498EE40E94121AF5
:10A6D000882311F40C94F8490E94F11D6093180E20
:10A6E0007093190E80931A0E90931B0E0C94F849D8
:10A6F00083E50E94121A882321F00E94011E809394
:10A700004B0D0E94FC3D8FE09BE00E945E348091E7
:10A710004B0D882331F110E000E020E080914B0DDB
:10A7200090E0002E02C0959587950A94E2F780FF8D
:10A7300012C0FF24F394F20E222319F08CE20E943F
:10A740003D34F801EE0FFF1FEB5FF44F85919491BC
:10A750000E945E342F2D0F5F1F4F05301105F1F65B
:10A76000C1CD81E09BE0C4CD41E070E060E086E1D6
:10A770009BE00E941A408CE3809318010C94F849E6
:10A780000E94FC3D1091180184E29BE00E945E341F
:10A79000812F0E94DB1D8AE00E943D340C94F84911
:10A7A00083E50E94121A882311F40C94F8490E9440
:10A7B000011E182F8C3308F08CE38093F8030E945D
:10A7C00050CE6B017C01212F30E0A8EEB3E00E9457
:10A7D00083EEC60ED71EE81EF91EC092F403D09277
:10A7E000F503E092F603F092F7030C94F849809198
:10A7F000FD038F7D80618093FD030C94F849809167
:10A80000FD038F7E80628093FD030C94F84983E5FD
:10A810000E94121A8823F1F00E9450CE6093220405
:10A820007093230480932404909325040E944B1E6C
:10A8300020E030E04AE754E40E946CE80E940CF00B
:10A840006093190170931A0180931B0190931C016E
:10A850000C94F8490E948A19882309F46EC00E945A
:10A860002C740E94E919082F10917B05182311F40C
:10A870000C94F849F12CE12CC82ED12CAA24A394D5
:10A88000B12CC6010E2C02C0959587950A94E2F76B
:10A8900080FF12C08E2D0E947473882369F0F70127
:10A8A000EC5DFD4F808195010E2C01C0220F0A94B2
:10A8B000EAF7822B80951823AFEFEA1AFA0AB3E081
:10A8C000EB16F104F1F603FF04C00E945F738111DF
:10A8D000147FF12CE12CC12ED12CC6010E2C02C00C
:10A8E000959587950A94E2F780FF0FC0F701E95626
:10A8F000FE4F80810E943D34F701EC5DFD4F908159
:10A9000080917B0589230E94C4DBEFEFEE1AFE0ADB
:10A91000F3E0EF16F10409F713FD02C00C94F849B7
:10A9200085E40E943D3480E30E943D3480917B05A4
:10A9300083700E94C4DB0C94F8490E943D740C940F
:10A94000F84983E50E949B19882311F40C94F84977
:10A950000E9450CE609322047093230480932404B9
:10A96000909325040E944B1E20E030E04AE754E417
:10A970000E946CE80E940CF06093F9037093FA0354
:10A980008093FB039093FC030C94F849B7E9CB2E1A
:10A99000B1E0DB2E1CE4E12E1DE0F12E10E0D6012B
:10A9A0008D916D010E94121A882349F0133089F0AD
:10A9B0000E944B1EF701648B758B868B978B1F5FF4
:10A9C000F4E0EF0EF11C143051F70E9404740C9463
:10A9D000F8490E944B1E4B015C0120E030E040EA48
:10A9E00051E40E9407E887FF3AC0A50194016091F5
:10A9F0006C0D70916D0D80916E0D90916F0D0E9498
:10AA00009FEF2B013C01AC019B0160917C0D70918B
:10AA10007D0D80917E0D90917F0D0E946CE860937A
:10AA20007C0D70937D0D80937E0D90937F0D6091D2
:10AA30007E0770917F0780918007909181070E9427
:10AA40000BE8A30192010E946CE80E940CF0609355
:10AA50007E0770937F078093800790938107809291
:10AA60006C0D90926D0DA0926E0DB0926F0DA7CFF0
:10AA70000E94A5B38BE393E10E94A6720C94F8495F
:10AA800080911D0490911E04009709F4DBCBDC013A
:10AA90002C91222309F4D6CB0E9493C20C94F8493E
:10AAA00000911D0410911E0494E0F12C40E091509F
:10AAB000F9F0F8018081282F2B7F213499F421812E
:10AAC0002133B1F4813411F1853409F441E0980166
:10AAD0002E5F3F4F89012F5F3F4FF8018081803209
:10AAE000C9F3E5CF803521F4818180538A3078F332
:10AAF00041110E94FC3DFF2021F08EEB9DE00E9461
:10AB00005E34C8010E944F340C94F849FF24F3943A
:10AB1000DECF0E948A880C94F84981E08093E60693
:10AB20008093E5060E94D0880C94F8491092E606BE
:10AB30001092E5060E94D0880C94F84970E060E01D
:10AB400083E50E943F1E823040F00E94F83D81EC78
:10AB50009DE00E945E340C94F8498C01112788E432
:10AB60000E94121A8823A9F00E943C1E8A3A91057D
:10AB700074F10E943C1E863F910564F50E943C1EC4
:10AB8000F801EE0FFF1FEE0FFF1FEE58FA4F9183F3
:10AB9000808386E40E94121A882311F40C94F849E9
:10ABA0000E943C1E97FD19C00E943C1E8F3F9105DC
:10ABB00009F0B4F40E943C1E000F111F000F111F7A
:10ABC000F801EE58FA4F938382830C94F8498AEA8D
:10ABD00090E0D6CF85EF90E0D3CF90E080E0ECCF4F
:10ABE0008FEF90E0E9CF0E94003E87FF02C00C94F7
:10ABF000F84907E911E05CE4E52E5DE0F52E6BE92C
:10AC0000C62E61E0D62ED8018D918D010E94121AB8
:10AC1000882359F00E944B1E0E940CF0F7016083BC
:10AC20007183828393830E94C073F4E0EF0EF11C62
:10AC3000C016D10641F70C94F8498091190484FD9F
:10AC40000DC080911B04887849F480911C048370A6
:10AC500029F481E00E94F1380C94F8490E94003EEA
:10AC600087FF02C00C94F84947E9E42E41E0F42E36
:10AC700010E000E0D7018D917D010E94121A882317
:10AC800049F00E944B1EF801E45BF24F64A375A3E8
:10AC900086A397A30C5F1F4F0031110559F70C9441
:10ACA000F84980911A0487FD09C080911B048E70B9
:10ACB00029F481E00E94D1380C94F84983E50E9480
:10ACC000121A882391F00E944B1E6093800D70939E
:10ACD000810D8093820D9093830D6093880D709306
:10ACE000890D80938A0D90938B0D80E50E94121A36
:10ACF000882351F00E944B1E6093800D7093810D4C
:10AD00008093820D9093830D82E50E94121A88230E
:10AD100051F00E944B1E6093840D7093850D8093BB
:10AD2000860D9093870D84E50E94121A882311F4F2
:10AD30000C94F8490E944B1E6093880D7093890D06
:10AD400080938A0D90938B0D0C94F84982E40E94B5
:10AD5000121A882351F00E94E11D60935C0D7093DC
:10AD60005D0D80935E0D90935F0D83E50E94121A36
:10AD7000882351F00E944B1E60938C0D70938D0DB3
:10AD800080938E0D90938F0D84E50E94121A882374
:10AD900051F00E944B1E6093900D7093910D809323
:10ADA000920D9093930D8AE40E94121A882311F455
:10ADB0000C94F8490E944B1E6B017C012AE037ED90
:10ADC00043E25CE30E94C4F087FD14C02AE939E93C
:10ADD00049E95EE3C701B6010E9407E8181654F07E
:10ADE000C0926E07D0926F07E0927007F0927107E1
:10ADF0000C94F8490E94F83D83EE9DE00E945E3479
:10AE00000C94F84983E50E949B19882331F00E9435
:10AE10001C1E80933B010C94F84910913B01105D7E
:10AE20008BE19EE00E945E34812F0E943D3487E1D9
:10AE30009EE00E945E3480913B010E94EC3D209197
:10AE40003D0130913E0140913F01509140012CA3C2
:10AE50003DA34EA35FA340904101509042016090FA
:10AE60004301709044018090450190904601A0906C
:10AE70004701B0904801C0904901D0904A01E0904C
:10AE80004B01F0904C0180914D0190914E01A091A9
:10AE90004F01B091500188A799A7AAA7BBA72091FD
:10AEA00051013091520140915301509154012CA70E
:10AEB0003DA74EA75FA78FE09EE00E945E344CA1A5
:10AEC0005DA16EA17FA182E09EE00E948034B3016B
:10AED000A20182E29FE20E948034B501A4018FE1C9
:10AEE0009FE20E9480348DE09EE00E945E3485E007
:10AEF0009EE00E945E34B701A60182E09EE00E94BF
:10AF0000803448A559A56AA57BA582E29FE20E94EC
:10AF100080344CA55DA56EA57FA58FE19FE20E94C0
:10AF200080348AE00E943D340C94F8490E94003E2F
:10AF3000082F87FF02C00C94F84983E50E94121A7B
:10AF4000002E000C110B7801EE0CFF1C882309F178
:10AF50000E943C1EF701EB5AFE4F91838083000F45
:10AF6000111F000F111F0F581E4FBC01990F880BA6
:10AF7000990B0E940DE82AE037ED43E25CE30E9462
:10AF80006CE8D8016D937D938D939C9313970C94EB
:10AF9000F8490E94FC3D85E40E943D3480E3800F27
:10AFA0000E943D34F701EB5AFE4F6081718188E2C7
:10AFB0009EE00E94683F85E20E943D348AE00E9444
:10AFC0003D340C94F84980E50E94121A882311F44C
:10AFD0000C94F8490E943C1E8C01892B09F081C019
:10AFE00083E50E94121A882389F00E943C1E97FD77
:10AFF00007C0BC0185E293E10E9440320C94F849FD
:10B0000085E293E10E941F320C94F8490E94FC3DB6
:10B0100070E060E089E49EE00E94683F8091271321
:10B02000F8E5CF2EF2E0DF2EC81AD10887FDD394C1
:10B03000CC0CDD1CCC0CDD1C0D2C000CEE08FF082C
:10B0400080912613B8E88B2E912C881A910887FDE1
:10B050009394880C991C880C991C092C000CAA0844
:10B06000BB088091251390E08F3FC9F1FC01EE0FE2
:10B07000FF1FE80FF91FE050FD4E8181928173E0C0
:10B08000880F991F7A95E1F7B0E0A0E0E4E0B5956C
:10B09000A79597958795EA95D1F702969C012F5F22
:10B0A0003F4F032E000C440B550B281939094A0950
:10B0B0005B09A4EBB0E00E9473EEA701960128198A
:10B0C00039094A095B090E9457EEB90186E49EE0FE
:10B0D0000E94683F8AE00E943D340C94F84980E069
:10B0E000DDCF0E94F83DB8018FE39EE00E94683FEB
:10B0F00080E39EE00E945E340C94F84983E50E9450
:10B10000121A81110C940D4F80911B0487FD14C0FD
:10B1100080911C04837081F40E94FC3D40913013A7
:10B1200050913113609132137091331381E59EE099
:10B130000E94BF340C94F84982E50E949B1981114A
:10B14000EBCF0C94F8498091190483FD09C08091DC
:10B150001A04817829F481E00E94283E0C94F84971
:10B1600080E50E94121A882351F00E944B1E6093C2
:10B1700098127093991280939A1290939B1289E47B
:10B180000E94121A882381F00E944B1E2CEA35EC93
:10B1900047E25EE30E946CE860939C1270939D12FC
:10B1A00080939E1290939F1284E40E94121A882327
:10B1B00011F40C94F8490E944B1E20E030E543EC5A
:10B1C00050E40E946CE86093A0127093A1128093E7
:10B1D000A2129093A3120C94F84983E50E949B1944
:10B1E000182F882369F00E943C1E9C0190937601E1
:10B1F0008093750191E0232B09F090E090937F12EA
:10B2000080E50E949B19882361F02091750130919F
:10B210007601232B11F00E941C1E80937F120C9448
:10B22000F84911110C94F8490E94FC3D8BE89EE00E
:10B230000E945E3480917F12882391F083E79EE024
:10B240000E945E3460917501709176018AE79EE0FC
:10B250000E94683F86E79EE00E945E340C94F849A5
:10B260008FE69EE0EDCF0E94C2340C94F8490E9414
:10B270002C740C94F8490E94CC270E94DF870C9410
:10B28000F8498091190483FD2AC080911B048670BF
:10B2900031F50E94FC3D85EB9EE00E945E3480917A
:10B2A0005B018823C9F082EA9EE00E945E344091EF
:10B2B0005701509158016091590170915A0188EAE3
:10B2C0009EE00E94803485EA9EE00E945E348AE01F
:10B2D0000E943D340C94F8498EE99EE0E6CFC09080
:10B2E0001904D0901A04E0901B04F0901C0431E182
:10B2F000F694E794D794C7943A95D1F7B1E0CB226E
:10B30000DD24EE24FF2483E50E949B19182FC1142D
:10B31000D104E104F10411F4882341F00E941E1AC3
:10B32000112321F00E941C1E80935B0184E40E9483
:10B330009B19882311F40C94F8490E944B1E6093CA
:10B340005701709358018093590190935A010C94BE
:10B35000F84983E50E949B19182F882309F426C118
:10B360000E941C1E8CA3209177013091780140919E
:10B37000790150917A012DAB3EAB4FAB58AF809124
:10B380007B0190917C01A0917D01B0917E0189AFFC
:10B390009AAFABAFBCAF20917F013091800140915B
:10B3A00081015091820121962CAF3DAF4EAF5FAF2E
:10B3B0002197112331F03CA1311103C080E00E949C
:10B3C0001E2A8091190490911A04A0911B04B09137
:10B3D0001C0425E1B695A795979587952A95D1F7F1
:10B3E0009C01AD01217033274427552729AB3AAB87
:10B3F0004BAB5CAB20E030E0A90160916A05709135
:10B400006B0580916C0590916D050E9407E888237B
:10B4100009F4D0C083E40E949B19882309F49AC0E0
:10B420000E944B1E25966CAF7DAF8EAF9FAF2597C8
:10B430004EE954E059A748A78A0157E05CA7412C80
:10B44000512CE8EC6E2EE2EC7E2E812C912CF8EC47
:10B45000AF2EF2E4BF2E312C212CF101EE0FFF1F95
:10B46000EE0FFF1FE00FF11FC080D180E280F3805C
:10B47000A7019601C501B4010E9407E8181614F44B
:10B4800046015701A7019601C301B2010E94C4F011
:10B4900087FF02C0260137018FEF281A380A97E08C
:10B4A00029163104D1F6ACA5A150ACA7045E1F4FFC
:10B4B000A111D1CFA3019201C501B4010E9425EFD2
:10B4C00020E030E040E05FE30E946CE825962CAD80
:10B4D0003DAD4EAD5FAD25970E9425EF4B015C0160
:10B4E0002DEB37E346E855EB0E9407E887FD0AC0DD
:10B4F0002DEB37E346E855E3C501B4010E94C4F0E3
:10B50000181644F580E00E941E2A67E0F62E08A572
:10B5100019A557E0E52EF801619171918191919102
:10B520008F016F01F4E0CF1AD108A50194010E94A8
:10B5300024EFD6016D937D938D939C931397EA949A
:10B54000E110E9CFFA94E8A5F9A57C96F9A7E8A758
:10B55000F110DDCF89A99AA9ABA9BCA9892B8A2BA7
:10B560008B2B81F020E030E0A90160916A05709199
:10B570006B0580916C0590916D050E9407E8811123
:10B580000E948D3D8AE50E949B19882359F00E94F4
:10B590004B1E69837A838B839C8360E0CE01019686
:10B5A0000E94AA2A8CA10E941E2A15C0E09199042B
:10B5B000ECA3D9CEFCA1F11108C029A93AA94BA945
:10B5C0005CA9232B242B252BE9F20E94FC3D85E06E
:10B5D0009FE00E945E349CA1992351F080919904D0
:10B5E000811106C00E94F83D86EE9EE00E945E3406
:10B5F0000E94FC3D88ED9EE00E945E34809199049B
:10B600000E94EC3D0E94FC3D8BEC9EE00E945E346B
:10B61000C0909A04D0909B04E0909C04F0909D040C
:10B6200020E030E0A901C701B6010E94C4F018165D
:10B630000CF042C042E0C701B6010E9438B38DE071
:10B640000E943D348AE00E943D3420917701309180
:10B6500078014091790150917A016DA97EA98FA955
:10B6600098AD0E9407E881110C947A4920917B01E2
:10B6700030917C0140917D0150917E0169AD7AADA0
:10B680008BAD9CAD0E9407E881110C947A49209102
:10B690007F0130918001409181015091820121967A
:10B6A0006CAD7DAD8EAD9FAD21970E9407E88111F5
:10B6B0000C947A490C94F84986EC9EE00E945E3422
:10B6C000C4CFA3940C94EE4F0E94F83D84E39FE016
:10B6D0000E945E340C94F8490E9454A20C94F849DC
:10B6E0000E9444920C94F8490E94DA880C94F8491C
:10B6F0000E946A3E0C94F8498091A31482FF0CC00A
:10B7000087FD0AC00E94112C9091A31480FB97F929
:10B710009093A3140C94F84984FD02C00C94F8494A
:10B720000E94CBD60C94F8494090281350902913CE
:10B7300060902A1370902B1320912C1330912D13AD
:10B7400040912E1350912F132CA33DA34EA35FA322
:10B75000C0903013D0903113E0903213F090331337
:10B7600088E50E94121A182F882309F482C00E94CB
:10B770004B1E4B015C0120E030E041E653EC0E949F
:10B78000C4F087FD0BC020E030E041E653E4C50182
:10B79000B4010E9407E818160CF06DC061EE70E06D
:10B7A00085E99FE00E94683F61EE70E080E99FE0DC
:10B7B0000E94683F8DE89FE00E945E3410E089E5BA
:10B7C0000E94121A882341F10E944B1E4B015C011A
:10B7D00020E030E041E653EC0E94C4F087FD0BC04E
:10B7E00020E030E041E653E4C501B4010E9407E8DF
:10B7F00018160CF043C061EE70E08AE79FE00E94EB
:10B80000683F61EE70E085E79FE00E94683F82E755
:10B810009FE00E945E3410E08AE50E94121A88239D
:10B8200091F10E944B1E6B017C0120E030E040EA68
:10B8300051EC0E94C4F087FD0AC020E030E040EAED
:10B8400051E4C701B6010E9407E81816E4F46CEE53
:10B850007FEF80E69FE00E94683F64E170E08BE547
:10B860009FE00E94683F88E59FE00E945E340C9450
:10B87000F84911E0A4CF24013501A1CF8CA29DA2EB
:10B88000AEA2BFA2C9CF112311F40C94F849409283
:10B8900028135092291360922A1370922B138CA1B3
:10B8A0009DA1AEA1BFA180932C1390932D13A093C3
:10B8B0002E13B0932F13C0923013D0923113E09215
:10B8C0003213F09233130C94F84983E080932D07E0
:10B8D0001092771060E083E50E942B1E81110C947A
:10B8E000F8490E94AFC30C94F84900911F041091CD
:10B8F00020040E9450CE609322047093230480930E
:10B90000240490932504002311F40C94F8490E9418
:10B91000FC3D84E50E943D34802F0E94DB1D80E2C7
:10B920000E943D3488EC9FE00E945E340C94F849FC
:10B9300011110FC011E08091190490911A04A09187
:10B940001B04B0911C043B2F3170A32E31130C94B7
:10B95000F7488C2D8170A12E81130C94F74811E0CB
:10B96000AA24A394BB24B39482E50E94121A8823CC
:10B9700011F40C945A4A0E944B1E68A379A38AA31F
:10B980009BA320E030E0A9010E9407E8882379F01A
:10B99000111105C0A11003C0BB2009F42BC1CE01B9
:10B9A00080960E94BBC40E9467330E9422331123F9
:10B9B00009F48AC0AA2009F484C010927701109279
:10B9C00078011092790110927A0110927B01109205
:10B9D0007C0110927D0110927E010E9491878DE47E
:10B9E0009EE10E94C6276B017C0181E59EE10E94D9
:10B9F000C6272B013C01AC019B01C701B6010E9487
:10BA0000C4F0181614F00C94604AA7019601C30103
:10BA1000B2010E949FEF9B01AC010E946CE820E004
:10BA200030E040E85FE30E9425EF0E9403F121E04F
:10BA300030E048E452E40E946CE869837A838B83A7
:10BA40009C8380917F0190918001A0918101B091B0
:10BA500082018CA39DA3AEA3BFA320E030E040EC05
:10BA60005FE3C301B2010E946CE82B013C0177FA4D
:10BA7000709477F8709420E030E040EC5FE3C70109
:10BA8000B6010E946CE89058DE0111966D01ECA0A1
:10BA9000FDA00EA11FA1A30192010E94E3860E94B6
:10BAA000798B10927701109278011092790110929F
:10BAB0007A0110927B0110927C0110927D0110920C
:10BAC0007E0180E00E94478AAA2019F081E00E944E
:10BAD000478ABB2009F48EC083E00E9459838111FC
:10BAE00089C00E94918780917F0190918001A091EF
:10BAF0008101B09182018093950490939604A09364
:10BB00009704B09398040091341310913513F80101
:10BB1000C080D180E280F380A701960160E070E0F0
:10BB200080EE92E40E9424EF6093890470938A046B
:10BB300080938B0490938C04D80114964D905D9063
:10BB40006D907C901797A301920160E070E080EE09
:10BB500092E40E9424EF60938D0470938E0480938E
:10BB60008F04909390042DE030E044EE52E4C30142
:10BB7000B2010E94C4F0181614F40C94664A2EE028
:10BB800030E042EE52ECC301B2010E9407E887FFA9
:10BB900002C00C94664A2DE030E04EEE52E4C7013C
:10BBA000B6010E9407E8181614F40C94664A2EE0B9
:10BBB00030E042EE52ECC701B6010E94C4F087FFAC
:10BBC00002C00C94664A1C8E1D8E1E8E1F8E88E04D
:10BBD000E9E8F4E0DE01119601900D928A95E1F713
:10BBE000BE01645E7F4FCE0101960E94F0C782E0E5
:10BBF0000E94478A0E9491878091E5068093E6061D
:10BC0000992019F081E00E941E2A0E94AB8683E0F1
:10BC100080936C010E94DF870C94F84983E50E94B1
:10BC2000121A882311F40C9450530E94F11D8B01B9
:10BC30000C9450530E94F83D84E19FE00E945E34D2
:10BC40000C94F849882309F475CE89CEB0E0A0E0C1
:10BC5000ECE2FEE50C94EFEE7C014DB65EB6609032
:10BC60006C0770906D078DB69EB66AE070E0C701F4
:10BC70000E9444E76C018C010E191F09892B21F4E5
:10BC8000C7010E9456E78C01C80101962DB73EB747
:10BC9000281B390B0FB6F8943EBF0FBE2DBF8DB7D2
:10BCA0009EB701965C01A801B7010E9477E7F501F4
:10BCB000E00FF11F1082C5010E946A2681E00E94F8
:10BCC0005648C114D10451F076019FEFE91AF90AE0
:10BCD0000FB6F8949EBE0FBE8DBEC5CF0FB6F894BA
:10BCE0009EBE0FBE8DBEC3010E946A260FB6F89499
:10BCF0005EBE0FBE4DBEE0E10C940BEFA2E4B0E0DF
:10BD0000E4E8FEE50C94EDEE0E9450CE6093220430
:10BD100070932304809324049093250480919904C4
:10BD2000811145C08091190490911A04A0911B04BF
:10BD3000B0911C043DE0B695A795979587953A95E7
:10BD4000D1F780FF03C086E096E080DF87E00E94A5
:10BD50005983811133C080919904888B8091190493
:10BD600090911A04A0911B04B0911C04AC01BD0178
:10BD700026E176956795579547952A95D1F740FF27
:10BD8000EDC020E030E0A90160916A0570916B057B
:10BD900080916C0590916D050E9407E8811113C098
:10BDA0000E94F83D84EF95E00E945E3407C060E099
:10BDB0008FE40E942B1E882309F4B4CFCE5BDF4FA3
:10BDC000E2E10C9409EF8AE50E94121A8823E9F057
:10BDD0000E944B1E6B017C0120E030E040E251EC00
:10BDE000C701B6010E9407E887FD0AC020E030E0E5
:10BDF00040E251E4C701B6010E94C4F0181674F481
:10BE00000E94F83D87EE95E0CFCFC0907F01D090A3
:10BE10008001E0908101F0908201DECF40E050E0AF
:10BE200060EC7FE788E50E94731E2B013C0140E037
:10BE300050E060EC7FE789E50E94731E6BAB7CAB42
:10BE40008DAB9EAB6FEF89E40E94121E6FEF8AE408
:10BE50000E94121E8BA09CA0ADA0BEA020E030E0EE
:10BE600040E05FE3C501B4010E946CE820916205E7
:10BE70003091630540916405509165050E9424EF5F
:10BE8000A30192010E9425EFA50194010E949FEF5A
:10BE90000E9407F02B013C01162F8FA098A4A9A4A3
:10BEA000BAA420E030E040E05FE3C501B4010E94A5
:10BEB0006CE82091660530916705409168055091C6
:10BEC00069050E9424EF2BA93CA94DA95EA90E94F7
:10BED00025EFA50194010E949FEF0E9407F0062F15
:10BEE000042C000C550857FC31C027E042165104C1
:10BEF0007CF5062E000C770B77FD2CC067307105A2
:10BF00005CF5173008F05ACF073008F057CF80E0C3
:10BF10000E941E2A37E01302F0011124E00FF11DE8
:10BF200007FDFA95EE0FFF1FEE0FFF1FE256FB4FC6
:10BF3000C082D182E282F38288890E941E2A888987
:10BF4000882309F43BCF0E94DF8738CF10E0D1CFA0
:10BF500016E0CFCF00E0D5CF06E0D3CFE9E0B6952D
:10BF6000A79597958795EA95D1F780FD0CC070E06D
:10BF700060E086E50E943F1E9A838983059730F032
:10BF800082EC95E011CF0E94602A18CF60E084E433
:10BF90000E942B1E8F8740E050E0BA018AE50E9484
:10BFA000731E6BA77CA78DA79EA740E050E669EFA4
:10BFB00075E483E50E94731E29E838E848E85CE3ED
:10BFC0000E946CE860936D0170936E0180936F0125
:10BFD00090937001E0903413F0903513D7014D9099
:10BFE0005D906D907C9020E030E040EE50E4C30125
:10BFF000B2010E9424EF4B015C0120E030E040E2FE
:10C0000051E40E94C4F087FF06C0812C912C70E29D
:10C01000A72E71E4B72E20E030E041E653E4C301DF
:10C02000B2010E9425EF6FAB78AF89AF9AAF20E0E5
:10C0300030E047E553E40E9407E8181644F480E036
:10C0400090E0A7E5B3E48FAB98AFA9AFBAAFD70143
:10C050001496CD90DD90ED90FC90179720E030E0A5
:10C0600040E050E4C701B6010E9424EF2B013C01DF
:10C0700020E030E040E251E40E94C4F087FF06C0B7
:10C08000412C512C60E2662E61E4762E20E030E0F7
:10C0900041E653E4C701B6010E9425EF6BAB7CABD0
:10C0A0008DAB9EAB20E030E047E553E40E9407E80B
:10C0B000181644F480E090E0A7E5B3E48BAB9CABAA
:10C0C000ADABBEAB88E40E949B19882309F4F8C18C
:10C0D0000E944B1E0E9407F023966CAF7DAF8EAF7F
:10C0E0009FAF239721966EAD7FAD219777FF02C05A
:10C0F0006F5F7F4F7595679571956195710960596F
:10C100007F4F072E000C880B990B0E940DE86B01E6
:10C110007C01CBAEDCAEEDAEFEAEA30192010E947F
:10C12000C4F087FF04C04BAE5CAE6DAE7EAEA50121
:10C130009401C701B6010E94C4F087FF02C07501D7
:10C140006401CB8ADC8AED8AFE8A8BAD9CADADADF5
:10C15000BEAD8F8B988FA98FBA8F2196AEADBFAD34
:10C160002197BD01BB0F880B990B0E940DE84B0175
:10C170005C01A70196010E9425EF6B017C012FA9AC
:10C1800038AD49AD5AAD0E9407E8181624F4CFA87F
:10C19000D8ACE9ACFAACCB8EDC8EED8EFE8E2BAD3E
:10C1A0003CAD4DAD5EADC501B4010E9425EF6B0104
:10C1B0007C012BA93CA94DA95EA90E9407E818168D
:10C1C00024F4CBA8DCA8EDA8FEA8CF8ED8A2E9A2C3
:10C1D000FAA2BE01695E7F4FCE0143960E944BC515
:10C1E000882309F496C1BE01615E7F4FCE014B9654
:10C1F0000E944BC5E82E882309F48BC12F89388D06
:10C20000498D5A8D6F8D78A189A19AA10E9424EF42
:10C210002BEA3AEA4AE25EE30E946CE84B015C01D9
:10C220002B893C894D895E896B8D7C8D8D8D9E8D92
:10C230000E9424EF2BEA3AEA4AE25EE30E946CE8AD
:10C240006BA37CA38DA39EA38FA298A6A9A6BAA632
:10C2500089819A811816190674F480E995E00E9484
:10C260005E348F85882321F086E895E00E945E3455
:10C270008AE00E943D340E942C740E94C48680E0B3
:10C280000E941E2A80E090E0A0E2B1E48FA798AB64
:10C29000A9ABBAABCE018F960E94BBC420916A05B0
:10C2A00030916B0540916C0550916D056BA17CA19F
:10C2B0008DA19EA10E9407E8811130C020916E05DA
:10C2C00030916F0540917005509171056FA178A56F
:10C2D00089A59AA50E9407E8811120C020916205D6
:10C2E0003091630540916405509165056B897C89A7
:10C2F0008D899E890E9407E8811110C020916605F2
:10C300003091670540916805509169056F89788D76
:10C31000898D9A8D0E9407E88823A9F00E94602ADF
:10C3200088E0FE01B396AAE6B5E001900D928A95E9
:10C33000E1F788E0FE017396A2E6B5E001900D9268
:10C340008A95E1F7188A60E085E40E942B1ECC24D0
:10C35000C394811102C043E0C42E1B861C861D8637
:10C360001E861A8ADE2C97E0792E26E5A22E25E07D
:10C37000B22E34E6832E35E0932E8A8987300CF076
:10C38000D4C0DD2009F4C8C066246394B7E0BBAB19
:10C3900090E021E0D226879DF02C1124F394998B14
:10C3A00019896A89FBA91F1709F4BCC0062E000C65
:10C3B000770B880B990B0E940DE82FA138A549A592
:10C3C0005AA50E946CE82F89388D498D5A8D0E949C
:10C3D00025EF1B012C01612F110F770B880B990B97
:10C3E0000E940DE82BA13CA14DA15EA10E946CE82A
:10C3F0002B893C894D895E890E9425EF6B837C8364
:10C400008D839E832F82388649865A8689819A81B8
:10C41000892B89F082E795E00E945E348F2D0E947F
:10C42000DB1D61E370E080E795E00E94683F8DE6E8
:10C4300095E00E945E341F9221E32F931F92FF929A
:10C44000BF92AF929F928F921F920E94FEA129816C
:10C450004C2DBE01695F7F4FCE0103960E9481C6BD
:10C460009B01AC012B873C874D875E8709898A89B0
:10C47000672D060380011124080F111D87FD1A95F1
:10C48000000F111F000F111F02561B4F6BA57CA53B
:10C490008DA59EA50E9425EFD8016D937D938D9368
:10C4A0009C931397188A81E00E940B41F394898929
:10C4B000860D898B0FB6F894DEBF0FBECDBF70CF4F
:10C4C000B301A20186E40E94731E6B017C01B501D9
:10C4D000A4018CE40E94731E6B8B7C8B8D8B9E8BD6
:10C4E000CF8AD88EE98EFA8E4BA95CA96DA97EA958
:10C4F00082E40E94731E6B017C014FA958AD69ADA7
:10C500007AAD82E50E94731E6B8F7C8F8D8F9E8F1C
:10C510005CCE86EA95E048CC66246A94EFEFEBABFC
:10C5200096E037CF6F5F6A8B28CF0E9409C50E94C3
:10C53000CC27882359F088890E941E2A80E090E049
:10C54000A0ECBFE78B879C87AD87BE870E948D3D9F
:10C550000E94772B8F85811122C08FE791E00E9486
:10C56000CF274B015C0187E791E00E944728A50196
:10C5700094010E946CE89B01AC0160917F01709175
:10C58000800180918101909182010E9424EF60934B
:10C590007F017093800180938101909382018F8548
:10C5A0008111E888E09299040E94AB8680919904F9
:10C5B000882309F4C8CC0E949187C5CCCF93DF9320
:10C5C000C091800E81E6C89FE0011124CE57D14F63
:10C5D00080914B0D80FF05C00E94FC3DCE010E9462
:10C5E0004F34CE010E946A2680E00E945648DF91B7
:10C5F000CF910895A0E1B0E0E0E0F3E60C94FBEE0B
:10C600008C01DC01ED91FC910280F381E02DBE01F3
:10C610006F5F7F4F0995882309F45DC08981807C15
:10C6200091F56F81637070E0762F6627770F770F33
:10C630008885B4E08B9FC0011124682B792B8985F4
:10C640008295869586958370682B6F5F7F4F90E00B
:10C6500080E02A852370220F3B8537FB332730F992
:10C66000232B3E813F70230F3327331F275031097F
:10C6700004C0660F771F881F991F2A95D2F760960E
:10C68000E4E00C9417EF803419F56885669566959B
:10C6900070E090E080E0CB01772766272A85622B47
:10C6A000098510E0102F0027012E000C220B330B00
:10C6B000602B712B822B932B6F5F7F4F8F4F9F4F80
:10C6C0004AE0660F771F881F991F4A95D1F7D7CF89
:10C6D0008BE0F801848360E070E0CB01D0CF089557
:10C6E000FC0182810895FC0190E1A2E6B6E0019090
:10C6F0000D929A95E1F70895EF92FF920F931F9391
:10C70000E0927C05F0927D0500937E0510937F05F5
:10C71000B62F172F022FF32E242F582FB0938505F5
:10C7200010938605509387056FEFFF27B01B1F09F5
:10C73000520B30F450951095B195160B560B662799
:10C740006093A402A6E0BA9F00929802712DEE2792
:10C750001A9F700DE11D5A9FE00D70939902E093AE
:10C760009A02AFE0BA9F00929C02712DEE271A9FA9
:10C77000700DE11D5A9FE00D70939D02E0939E02A3
:10C78000AAE0BA9F0092A002712DEE271A9F700DA9
:10C79000E11D5A9FE00D7093A102E093A2021F9148
:10C7A0000F91FF90EF900895A5E0B0E0EAEDF3E679
:10C7B0000C94F4EE6F3671058105910578F4FB0158
:10C7C000EE0FFF1FEE0FFF1FEB59F04E65917591B5
:10C7D000859194912596EBE00C9410EFF62EE72EC0
:10C7E000282FE5E6FEE10027BB275F2D8E2D922F37
:10C7F000992341F4982F852FB85F992319F4982F26
:10C800008827B85F903138F482959295582F5F70E1
:10C81000807F952BBC5F903428F4880F991F880F78
:10C82000991FBE5F903818F4880F991FB395880F31
:10C83000991FE90FF01F549181E09927B85079F1C1
:10C84000C0F0B0FF02C0550F881FB1FF04C0550FE4
:10C85000881F550F881FB2FF06C082955295152F6D
:10C860001F70507F812BB3FF1AC0982F852F55273B
:10C8700016C0B195B0FF02C085955795B1FF04C0B1
:10C880008595579585955795B2FF05C08295507F40
:10C890005295582B8F70B3FF02C0582F8827BB24A6
:10C8A0007727AA27B2E0F59EB0187109A00BB00B4C
:10C8B000E59E7019A109B00B259FA019B109F89E3A
:10C8C0007019A109B00BE89EA019B109289FB019F1
:10C8D000F99EA019B109E99EB0195B9DA12C99247C
:10C8E0004427662733278B9DA00C911C401F601F97
:10C8F000301F9B9D900C411D601F301F579FA00C47
:10C90000911C401F601F301F879F900C411D601FAE
:10C91000301F979F400D611D301F5A9F900C411D85
:10C92000601F301F8A9F400D611D301F9A9F600D50
:10C93000311D5B9F400D611D301F8B9F600D311DB0
:10C940009B9F300DB1E0AA277727BB24F49EB01837
:10C950007109A00BB00BE49E7019A109B00B249FC4
:10C96000A019B109F69E7019A109B00BE69EA01995
:10C97000B109269FB019F39EA019B109E39EB01921
:10C98000BF187E09A20B20F0B1E04B0F601F301FD3
:10C990001124762F642F90E0832F1CCFFC0170812F
:10C9A000472F50E0062E02C0559547950A94E2F7AE
:10C9B00040FF14C04091FA0550E0062E02C0559584
:10C9C00047950A94E2F740FF09C021E030E001C03A
:10C9D000220F6A95EAF720952723208308958F92E6
:10C9E0009F92AF92BF92CF92DF92EF92FF92FC01A3
:10C9F000C080D180E280F38020E030E048EC52E457
:10CA0000C701B6010E946CE84B015C0120E030E0F8
:10CA1000A901C701B6010E9407E820E030E040EA22
:10CA200050E487FF04C020E030E040EA50ECC5014C
:10CA3000B4010E9425EF2DEC3CEC4CEC5DE30E9430
:10CA40006CE80E9407F09B018BE237FF05C02227AC
:10CA50003327261B370B8DE280938204C90168EED1
:10CA600073E00E94BFEECB01EAE0F0E0BF010E945C
:10CA7000BFEE805D80938304C90164E670E00E948C
:10CA8000BFEECB01BF010E94BFEE805D80938404A6
:10CA9000C901BF010E94BFEE9C01CB01BF010E94F2
:10CAA000BFEE805D809385048EE280938604205DD6
:10CAB0002093870482E894E0FF90EF90DF90CF907E
:10CAC000BF90AF909F908F9008954F925F926F921A
:10CAD0007F928F929F92AF92BF92CF92DF92EF920E
:10CAE000FF92FC01C080D180E280F38020E030E042
:10CAF0004AE754E4C701B6010E946CE84B015C01AF
:10CB000020E030E040E251ECC701B6010E9407E8A6
:10CB1000181654F420E030E048EC52E4C701B601A6
:10CB20000E94C4F087FD8AC020E030E0A901C7015F
:10CB3000B6010E9407E887FF72C060E070E080EAFB
:10CB400090ECA50194010E9425EF2DEC3CEC4CECFF
:10CB50005DE30E946CE80E9407F06B017C01F7FC2A
:10CB600063C020E137E240E050E00E9457EECA0186
:10CB7000B9012AE030E040E050E00E9457EE605DED
:10CB800060938204C701B60128EE33E040E050E034
:10CB90000E9457EE9AE0892E912CA12CB12CCA014B
:10CBA000B901A50194010E9457EE605D6093830472
:10CBB000C701B60124E630E040E050E00E9457EEA5
:10CBC000CA01B901A50194010E9457EE605D60930E
:10CBD00084048EE280938504C701B601A501940107
:10CBE0000E9457EE6B01CA01B901A50194010E9490
:10CBF00057EE605D60938604F0E3CF0EC092870429
:10CC000082E894E0FF90EF90DF90CF90BF90AF90DC
:10CC10009F908F907F906F905F904F90089560E00D
:10CC200070E080EA90E48DCFF094E094D094C094CA
:10CC3000C11CD11CE11CF11C6DE2A2CF20E030E050
:10CC4000A901C701B6010E9407E887FF6BC060E039
:10CC500070E080EA90ECA50194010E9425EF2DEC94
:10CC60003CEC4CEC5DE30E946CE80E9407F04B0149
:10CC70005C0120E030E0A901C701B6010E9407E88D
:10CC800087FD0BC020E030E040E251E4C701B6016F
:10CC90000E94C4F060E287FD13C0B7FC48C0C50124
:10CCA000B40128EE33E040E050E00E9457EECA01A4
:10CCB000B9012AE030E040E050E00E9457EE605DAC
:10CCC00060938304C501B40124E630E040E050E005
:10CCD0000E9457EE8AE0482E512C612C712CCA011B
:10CCE000B901A30192010E9457EE605D6093840434
:10CCF0008EE280938504C501B401A30192010E94D4
:10CD000057EE6B01CA01B901A30192010E9457EECF
:10CD1000605D6093860480E3C80EC092870483E858
:10CD200094E070CF60E070E080EA90E494CFB0943B
:10CD3000A09490948094811C911CA11CB11C6DE264
:10CD4000BFCF282F81E3243609F080E2809384044A
:10CD500090E22A3040F03AE0822F632F0E9492EE58
:10CD60000E9492EE905D90938504822F6AE00E946B
:10CD700092EE905D9093860485E28093870484E828
:10CD800094E008956091550170915601072E000CB2
:10CD9000880B990B0E940DE82AE037ED43E25CE333
:10CDA0000E946CE86093710170937201809373012B
:10CDB000909374010895CF93DF93EC01CB01BA01F6
:10CDC0000E940DE823E333E343E250E40E946CE861
:10CDD00020E030E040E05FE30E9425EF0E940CF08D
:10CDE0006883DF91CF9108950E940DE823E333E338
:10CDF00043E250E40E946CE820E030E040E05FE372
:10CE00000E9425EF0E940CF024E6629FC0011124CD
:10CE100081589F4F6FEF70E00E94BFEE862F91CF39
:10CE200080915707811104C080912E0780938A0753
:10CE30000895809199148823C1F0815080939914AA
:10CE4000ECEDF2E1882351F08150990B2BE1289F02
:10CE5000F001299FF00D1124E557FC4E8BE1A1EC68
:10CE6000B2E101900D928A95E1F720919914211178
:10CE700005C08091A31480648093A31481E090E0A6
:10CE8000A0E0B0E0211103C080E090E0DC018093DD
:10CE90004D0790934E07A0934F07B0935007109201
:10CEA000480781E080934A0783E080936C010895EE
:10CEB000CF93DF93EC01CB01BA010E940DE86883A8
:10CEC00079838A839B83DF91CF910895CF93DF93FA
:10CED000EC01CB01BA010E940DE82DEC3CEC4CECCE
:10CEE0005DE30E946CE8688379838A839B83DF918A
:10CEF000CF910895CF93DF93EC01CB01BA010E944B
:10CF00000DE82AE037ED43E25CE30E946CE86883B9
:10CF100079838A839B83DF91CF910895CF92DF92AB
:10CF2000EF92FF92CF93DF9300D000D0CDB7DEB762
:10CF30000E940DE82AE037ED43E25CE30E946CE8D2
:10CF40006B017C0120E030E0A9010E9407E82DEB95
:10CF500037E346E055E387FF04C02DEB37E346E0B7
:10CF600055EBC701B6010E9425EF69837A838B8355
:10CF70009C83CE010196A9DD0F900F900F900F902A
:10CF8000DF91CF91FF90EF90DF90CF900895CF93F6
:10CF9000DF93EC01CB01BA010E940DE80E9407F07B
:10CFA00079836883DF91CF9108958F929F92AF929A
:10CFB000BF92CF92DF92EF92FF92FC01C080D180AE
:10CFC000E280F38020E030E0A901C701B6010E94B1
:10CFD00007E887FD99C06DEB77E386E095E3A7014D
:10CFE00096010E9425EF9F7720E030E048EC52E464
:10CFF0000E946CE820E030E040EA50E40E9425EF17
:10D000002DEC3CEC4CEC5DE30E946CE80E9407F0D8
:10D010006B017C0180E28093810460E2F0E1CF1635
:10D02000F7E2DF06E104F1048CF0C701B60120E16C
:10D0300037E240E050E00E9457EECA01B9012AE011
:10D0400030E040E050E00E9457EE605D6093820463
:10D0500060E288EEC81683E0D806E104F1048CF0A3
:10D06000C701B60128EE33E040E050E00E9457EEE1
:10D07000CA01B9012AE030E040E050E00E9457EEDA
:10D08000605D6093830460E2E4E6CE16D104E104BF
:10D09000F1048CF0C701B60124E630E040E050E036
:10D0A0000E9457EECA01B9012AE030E040E050E0AA
:10D0B0000E9457EE605D609384048AE0882E912C74
:10D0C000A12CB12CC701B601A50194010E9457EE15
:10D0D0006B01CA01B901A50194010E9457EE605D80
:10D0E000609385048EE280938604F0E3CF0EC092B5
:10D0F000870481E894E0FF90EF90DF90CF90BF909D
:10D10000AF909F908F9008956DEB77E386E095EB5D
:10D1100066CFA4E0B0E0EFE8F8E60C94FDEE0E94E4
:10D120000DE82DEC3CEC4CEC5DE30E946CE869836F
:10D130007A838B839C83CE01019637DF2496E2E0CD
:10D140000C9419EFCF93DF93EC018D810E94FA408C
:10D1500060E08B810E946BCDDF91CF910895CF92DB
:10D16000DF92EF92FF920F931F93CF938C01C62F04
:10D1700069017A01E7DF0E943ACF8C2F80640E9418
:10D18000EE408F2D0E94EE408E2D0E94EE408D2DA0
:10D190000E94EE408C2D0E94EE4087E8C11101C034
:10D1A00085E90E94EE40CC3011F40E94F340C0E0CB
:10D1B0000E94F340F801868387FF04C0CF3F11F03F
:10D1C000CF5FF6CFCF911F910F91FF90EF90DF903F
:10D1D000CF90089561E0FC0183810E946BCD8FEFB9
:10D1E0000C94EE400F931F93CF938C01ABDF0E9402
:10D1F0003ACFC82F882369F08DEF0E94EE400E943D
:10D200003ACFC82FC801E6DF8C2FCF911F910F9125
:10D21000089582E1F8018483F5CFB0E0A0E0E3E176
:10D22000F9E60C94F3EEEC016A017B014801590127
:10D2300020E030E0A90167E392DFA501980167E1F2
:10D24000CE018DDF81111DC08F81833039F089E0DF
:10D25000CC0CDD1CEE1CFF1C8A95D1F7A7019601B2
:10D2600069E1CE017CDF11E0882319F010E087E04E
:10D270008C83CE01AFDF812FCDB7DEB7ECE00C940D
:10D280000FEF89E08C8310E0F4CFCF93DF93EC01B4
:10D290006EBDFA01CA019E5F0DB407FEFDCF20816D
:10D2A0002EBD0DB407FEFDCF21812EBD3296E817AD
:10D2B000F90791F70DB407FEFDCF8FEF0E94EE4006
:10D2C0008FEF0E94EE400E94F3408E838F71853075
:10D2D00041F083E18C83CE017DDF80E0DF91CF914F
:10D2E000089581E0FBCF0F931F93CF93DF93EC0161
:10D2F0008B0128DF0E943ACF81110BC085E18C831E
:10D3000010E0CE0167DF812FDF91CF911F910F9148
:10D310000895A8016CEFCE01B8DF182F882371F3B0
:10D32000F0CF0F931F93CF93DF93EC0189018F818F
:10D33000833039F089E0440F551F661F771F8A95A7
:10D34000D1F79A01AB0168E1CE0109DF811127C055
:10D35000A8016EEFCE0199DF182F8823A9F00E9453
:10D360003ACF182F8823C1F020E030E0A9016DE00A
:10D37000CE01F5DE882321F086E18C8310E004C025
:10D380000E94F3408111F8CFCE0124DF812FDF917D
:10D39000CF911F910F91089587E18C83F5CF86E09F
:10D3A000ECCF1F93CF93DF93EC01CCDE20E030E095
:10D3B000A9016CE0CE01D3DE11E0882319F010E062
:10D3C00083E08C83CE0106DF812FDF91CF911F9107
:10D3D00008951F93CF93DF93EC018F81833039F051
:10D3E00089E0440F551F661F771F8A95D1F79A0170
:10D3F000AB0162E1CE01B3DE11E0882319F010E049
:10D4000085E08C83CE01E6DE812FDF91CF911F91E5
:10D4100008958F929F92AF92BF92EF92FF920F93D7
:10D420001F93CF93DF938C01EB017A010E9450CEC2
:10D430004B015C012CE2820E21E0921EA11CB11C6A
:10D440000E94F340F80186838F3F69F40E9450CE1A
:10D45000681979098A099B0997FDF2CF81E1F801E2
:10D460008483C0E021C08E3F69F5F1E0EF1AF10836
:10D470008FEF8EBDFE012FEF0DB407FEFDCF8EB5F1
:10D4800081932EBDCF018C1B9D0B8E159F05A0F3A4
:10D490000DB407FEFDCF8EB5CE0DDF1D88830E9433
:10D4A000F3400E94F340C1E0C80194DE8C2FDF916D
:10D4B000CF911F910F91FF90EF90BF90AF909F90F1
:10D4C0008F9008958FE0CBCF0F931F93CF93DF936F
:10D4D000EC018B0137DE40E052E0B801CE0199DF6C
:10D4E000DF91CF911F910F9108950F931F93CF93C9
:10D4F000DF93EC0189018F81833039F089E0440F9B
:10D50000551F661F771F8A95D1F79A01AB0161E11C
:10D51000CE0125DE882351F084E08C83CE015ADED3
:10D5200080E0DF91CF911F910F91089540E052E08C
:10D53000B801CE016EDFF5CFB0E0A0E0E2EAFAE696
:10D540000C94F3EEEC01162F1F821C824B830E9479
:10D5500050CE6B017C0120EDC20E27E0D21EE11CF3
:10D56000F11CA89561E08B810E946BCD8B810E949C
:10D5700019B3249A2C9A279A2698259A81E00E941A
:10D58000FA4085E08D830E94FA400AE08FEF0E9406
:10D59000EE400150D9F7A89520E030E0A90160E005
:10D5A000CE01DDDD8E83813079F00E9450CE6C1982
:10D5B0007D098E099F0997FDEFCF81E08C83CE0115
:10D5C00009DE1A8280E065C0A8952AEA31E040E0D1
:10D5D00050E068E0CE01C3DD853031F581E08F8316
:10D5E000A8958F81812C912C5401823029F4812CB3
:10D5F000912CA12C80E4B82E20E030E0A90167E353
:10D60000CE01ADDDA501940169E2CE01A8DD8E83D6
:10D610008823F1F00E9450CE6C197D098E099F0974
:10D6200097FDEACF8AE0CACF04E00E94F3408E83E0
:10D630000150D9F78A3A11F482E0D1CF0E9450CE3E
:10D640006C197D098E099F0997FDBFCF82E0B6CF87
:10D650008F818230B9F420E030E0A9016AE3CE0185
:10D660007EDD882311F088E0A9CF0E94F340807C02
:10D67000803C11F483E08F830E94F3400E94F340CA
:10D680000E94F340CE01A6DD81E08A83173030F49A
:10D690001D83CDB7DEB7ECE00C940FEF88E18C83EF
:10D6A00091CF0F931F93CF93DF93EC018B0120E079
:10D6B00030E0A90169E053DD882351F080E18C83DB
:10D6C000CE0188DD80E0DF91CF911F910F91089509
:10D6D00040E150E0B801CE019CDEF5CFCF93C82FDA
:10D6E000CB010E945E3488E99DE10E945E3489E8A6
:10D6F0009DE1CC2311F08EE89DE10E945E348AE02A
:10D700000E943D34CF9108950C945CCE40917A05EF
:10D7100021E042276CE070E00C94EDB240917A0574
:10D7200021E0422764E070E00C94EDB240917A056C
:10D7300021E0422761E070E00C94EDB240917A055F
:10D7400021E0422761E070E00C94EDB240917A054F
:10D7500021E0422768E070E00C94EDB240917A0538
:10D7600021E042276CE070E00C94EDB241E061E012
:10D7700070E00C94EDB240917A0521E042270C94C0
:10D78000EDB26CE070E00C94FACD61E070E00C94C6
:10D79000FACD61E070E00C94FACD6CE070E00C948E
:10D7A000FACD64E070E00C94FACD9091990481E098
:10D7B00089270C941E2A61E08EE297E00C94AA2A35
:10D7C00020E030E0A901BC0187E791E00C9407C498
:10D7D00080E090E0A0E8B0E480937F019093800126
:10D7E000A0938101B093820188E492E0E9DF80E0B8
:10D7F00090E0A0EFB1E48093770190937801A0933B
:10D800007901B0937A0180937B0190937C01A0937E
:10D810007D01B0937E01E091D705EE0FFF0BE85D2F
:10D82000FD4F808191818330910539F184309105DC
:10D83000C9F1029761F480E090E0A3E4B3E480933F
:10D84000770190937801A0937901B0937A0180E3F6
:10D8500092E0B6DF10927F01109280011092810158
:10D860001092820188E492E0ABDF8091D7058F5F50
:10D870008430ECF48093D705089580E090E0A3E431
:10D88000B3E48093770190937801A0937901B093EA
:10D890007A0180937B0190937C01A0937D01B093EA
:10D8A0007E01D5CF80E090E0A3E4B3E4F2CF109204
:10D8B000D7050895A4E0B0E0E0E6FCE60C94FDEEA8
:10D8C00084EF91E0A0E0B0E089839A83AB83BC83CE
:10D8D000BE016F5F7F4F88E70E9405332496E2E028
:10D8E0000C9419EFB0E0A0E0E8E7FCE60C94FDEE44
:10D8F00020E24F8158856E818D810E941EC9E2E031
:10D900000C9419EF80912E0790912F070C9491CED3
:10D910006AEE78E982E00C942CCB6EEE78E981E037
:10D920000C942CCB62EF78E980E00C942CCB66EF62
:10D9300078E983E00C942CCB109248070C94D1D456
:10D940004FE350E06DEC7BE18CEE96E00C94D9F166
:10D950008091391390913A13891B8F7011F40C94B4
:10D96000FE2B81E0089580916C01882341F0609145
:10D97000CF057091D00541E081E00C94BEC80895B8
:10D980000F931F93CF93DF93FC012381222331F068
:10D9900080E0DF91CF911F910F9108958B01EC01F1
:10D9A000FB018789803139F582E08B831D8A1E8ACD
:10D9B0001F8A188E808D918DB0E0A0E025E0880F41
:10D9C000991FAA1FBB1F2A95D1F7898B9A8BAB8B06
:10D9D000BC8B1A8F098F81E08983188619861A8675
:10D9E0001B861C821D821E821F82188A1C861D8631
:10D9F0001E861F86CECF803259F683E08B83428D00
:10DA0000538D648D758D4D8B5E8B6F8B788F9E01E2
:10DA10002F5E3F4FC8010E942FD68111DACFB8CFB9
:10DA2000CF93DF93EC010E9498D61B82DF91CF91B8
:10DA30000895CF93DF93EC01462F41706C857D856F
:10DA40008E859F850E9441D3882351F0888920E2EA
:10DA5000829FC001112488589F4EDF91CF91089575
:10DA600090E080E0FACFCF93DF93EB01FC012381BC
:10DA7000211104C080E0DF91CF910895225022301F
:10DA800028F48FE28883198281E0F5CF60E0D1DF4E
:10DA9000009781F3DC0160E080E09EE22D9120326E
:10DAA00099F0883031F49E01260F311DF9019083E1
:10DAB0006F5F9E01260F311DAD0141505109FA01E2
:10DAC0004081F90140836F5F8F5F8B3039F7FE0132
:10DAD000E60FF11D1082D8CFACE0B0E0E2E7FDE642
:10DAE0000C94EEEE5C01DC0159968D909C90F40153
:10DAF00081859285A385B4859C01AD012F5F3F4F41
:10DB00004F4F5F4F29873A874B875C87D501149623
:10DB10004D905D906D907C90179741145104610475
:10DB2000710409F459C0BFEF4B1A5B0A6B0A7B0AF8
:10DB3000312C730162011D821E821F821886F4013E
:10DB400081859285A385B4852D813E814F8158853D
:10DB5000281739074A075B0708F056C089859A8558
:10DB6000AB85BC858C159D05AE05BF0550F482E0E4
:10DB7000C82ED12CE12CF12C92E0492E512C612C95
:10DB8000712C9E012F5F3F4FB701A601C4010E9477
:10DB9000B3D58823C9F189819A81AB81BC81892B56
:10DBA0008A2B8B2B01F1260137019FEF491A590A65
:10DBB000690A790A2D813E814F8158852F5F3F4F39
:10DBC0004F4F5F4F2D833E834F8358873FEFC31ADC
:10DBD000D30AE30AF30AB3CF408051806280738096
:10DBE00033243394A6CFC414D504E604F70411F704
:10DBF0000FEF1FEF2FEF3FE0B701A601C4010E9416
:10DC000039D5782E811106C0712C872D2C96E1E133
:10DC10000C940AEFF50144815581668177814115A5
:10DC200051056105710539F097018601C4010E9413
:10DC300039D5882349F3D5011496CD92DD92ED9222
:10DC4000FC921797332051F0D701C6010196A11D10
:10DC5000B11DF40180839183A283B383F50185898B
:10DC60009689A789B08D892B8A2B8B2B71F6C58A53
:10DC7000D68AE78AF08E818180688183C6CF40E0B2
:10DC800050E0BA010C94E1D64F925F926F927F926E
:10DC9000AF92BF92CF92DF92EF92FF920F931F93BA
:10DCA000CF93DF931F92CDB7DEB78C017B015A0172
:10DCB000C22EDB0159968D919C91F801928F818F34
:10DCC000CB01DDDF712CF70180859185A285B385BD
:10DCD000418952896389748984179507A607B70714
:10DCE00008F052C055E0B695A795979587955A9537
:10DCF000D1F7F82FFF70DF2ED70113968C91823069
:10DD000010F480E0DAC041E050E0BE016F5F7F4F69
:10DD1000C7010E94DCD70197A1F7F70180859185A3
:10DD2000A285B3854F96A11DB11D80879187A287DB
:10DD3000B387F0E2DF9EB001112468587F4E611571
:10DD40007105F9F2DB018C91882341F0853E09F0E1
:10DD50004BC0772029F077247394B5CF71100EC093
:10DD60008091781290917912A0917A12B0917B12E1
:10DD7000F80184879587A687B787D08ADB018C91C5
:10DD80008111E9CF772473948C2D8274823409F049
:10DD9000B8CF772009F4A1C0F801D08861E0C801AC
:10DDA00048DE009709F4ADCF20E2DC011D922A95F0
:10DDB000E9F72BE0F501DC0101900D922A95E1F7DE
:10DDC00021E238E2FC01318B208B40E058E057879C
:10DDD0004687338B228B318F208F578B468B0E9447
:10DDE000F8D2811109C08DCF4BE050E0C5010E94EF
:10DDF00089F1892B09F067CFF0E2DF9ED001112471
:10DE00009D0128583F4EF9018385817121F08C2DA9
:10DE1000827109F000C1F801818D928D40917812D4
:10DE20005091791260917A1270917B1244875587D4
:10DE300066877787D08AFD01E858FF4E4488558869
:10DE4000712C612C320155244424D80155964D92F1
:10DE50005D926D927C925897428D538D70E060E098
:10DE6000442955296629772955964D935D936D93DD
:10DE70007C935897D9011B962C91287109F0BDC04D
:10DE8000848D958DA68DB78DF801818B928BA38B98
:10DE9000B48B81E083838C2D8F70F8018183148291
:10DEA000158216821782108611861286138681E0EB
:10DEB000C4FE03C0C8010E9466D70F90DF91CF91C6
:10DEC0001F910F91FF90EF90DF90CF90BF90AF9098
:10DED0007F906F905F904F900895D70113968C912B
:10DEE0001397823009F40DCF51968D919D910D902D
:10DEF000BC91A02D803E9F4FAF41B10508F001CFEE
:10DF0000C701EADD882309F4FCCE0E94F8D28823F9
:10DF100009F4F7CED7015996ED91FC915A971496D2
:10DF20004D905D906D907C901797B2E04B1A510820
:10DF300061087108858504C0440C551C661C771C5B
:10DF40008A95D2F786859785A089B189480E591E92
:10DF50006A1E7B1E81E080937C1240927812509260
:10DF6000791260927A1270927B12E8E7F0E180E019
:10DF700092E0DF019C011D9221503040E1F7DD2449
:10DF8000D394D7015996ED91FC918481D816C0F4B1
:10DF900080917D1290917E12DC01ED91FC910288BE
:10DFA000F389E02D28E730E1B301A2014D0D511DA9
:10DFB000611D711D0995882309F4A3CED394E1CF87
:10DFC000258580E092E0A0E0B0E004C0880F991FB2
:10DFD000AA1FBB1F2A95D2F7F7014189528963898D
:10DFE0007489840F951FA61FB71F818B928BA38BFB
:10DFF000B48B88E790E1D12CD7CE203161F4980121
:10E000002F5E3F4F0E942FD6882329F084E0D8014D
:10E0100013968C9340CFD80113961C9272CEFC01BC
:10E0200023812111FDCC0895A1E4B0E0EAE1F0E7FD
:10E030000C94EDEE4C015B017A01222E19821C82B8
:10E040001C8E1F8E6115710569F410E0CE014C968F
:10E05000E6DFCE010196E3DF812FCF5BDF4FE2E108
:10E060000C9409EFFC0183818111EFCFFA018081CB
:10E070008F3251F18B01CE0101966C012C0180E2AF
:10E08000382E360122963FAE229721963FAE219739
:10E090003FAE3EAE3DAE3CAE3BAE3AAE39AE38AE34
:10E0A0003FAA970190E047E0D9018D91882309F4B8
:10E0B00046C08F3209F443C08E3201F54A3029F24E
:10E0C00098E04AE09D01F0CFFB01838182508230CD
:10E0D00098F0618D728DCE014C9652DC882309F444
:10E0E000B4CF8E01045E1F4FC7017C010196F7017A
:10E0F00020812F32D1F3BFCF8B01F6CFE9E2FAE2D4
:10E100002491222321F031968213FACF9ECF491712
:10E1100008F49BCF813208F498CF8F3709F495CF5C
:10E120003FE9380F3A3108F420EEE7E3F0E0EC0F76
:10E13000FD1FE90FF11D820F80839F5FC3CF8FA961
:10E14000803209F482CF7901F90180812F5F3F4F3E
:10E150008F32C9F38823C1F021E0AE01495C5F4FE3
:10E16000B801C60191DD882309F46FCF0A151B059C
:10E1700011F0C80155DCCE014C964C145D0409F039
:10E18000C30186016C017ECF222DAE01495C5F4F39
:10E19000B801C40179DD182F59CF8F929F92AF92A9
:10E1A000BF92CF92DF92EF92FF920F931F93CF9384
:10E1B000C82F0DE812E1F80160857185072E000C6B
:10E1C000880B990B0E940DE86B017C01F80184809B
:10E1D0009580A680B78080E20E943D3484E50E944D
:10E1E0003D348AE30E943D3442E0C501B4010E94FF
:10E1F00038B382E29AE20E945E3442E0C701B6017F
:10E200000E9438B362E070E080E090E00E94C7CDE9
:10E2100087E1C802F0011124E357FD4E628570E0EA
:10E2200085E29AE20E94683FCF911F910F91FF9083
:10E23000EF90DF90CF90BF90AF909F908F90089518
:10E240000F930FB70F9300916E000B7F00936E003A
:10E2500078940F930BB70F930CB70F921F922F93D5
:10E260003F934F935F936F937F938F939F93AF935E
:10E27000BF93EF93FF9311240E94D6ABFF91EF91D0
:10E28000BF91AF919F918F917F916F915F914F91CE
:10E290003F912F911F900F900CBF0F910BBF0F91CB
:10E2A0000460F89400936E000F910FBF0F911895C2
:10E2B000CF93DF9310928905CDE8D2E119861886B5
:10E2C0000E945CCE1A865D98DF91CF910895EF92FF
:10E2D000FF920F931F93CF93C82F7B018A018091E8
:10E2E0002D078330E0F00E94F83DC7010E945E34A4
:10E2F00088EA99E20E945E34C7FD0EC086EA99E280
:10E300000E945E346C2FCC0F770B880B990B0E9408
:10E31000EEB08AE00E943D348AE00E943D34C8DFBE
:10E32000A8958091720681110DC081E080937206DC
:10E3300082E080932D07BCDF40E063EA79E2C80108
:10E340000E941A40CF911F910F91FF90EF90089576
:10E35000CF93DF93A89580918F12909190120E9495
:10E3600066B260939112709392128093931290937D
:10E370009412C0918F12D09190128091650190916A
:10E380006601C817D90734F444EE59E261EF79E227
:10E3900080E09DDF809195129091961218161906D3
:10E3A0006CF480916301909164018C179D0734F4A3
:10E3B00043E05AE260E17AE280E089DFDF91CF91C9
:10E3C00008958F929F92AF92BF92CF92DF92EF9279
:10E3D000FF92CF93DF9300D000D0CDB7DEB780910E
:10E3E0002D07811110C0A8950F900F900F900F90DE
:10E3F000DF91CF91FF90EF90DF90CF90BF90AF90E3
:10E400009F908F900895809173068111EDCF81E0E8
:10E410008093730680918A05811103C01092730660
:10E42000E3CF96DF10928A050E9450CE6B017C01EB
:10E430000E9409B14B015C016091690170916A0110
:10E44000072E000C880B990B0E940DE89B01AC0174
:10E45000C501B4010E94C4F018160CF469C06091A3
:10E46000951270919612072E000C880B990B0E9442
:10E470000DE869837A838B839C83CE0101960E9489
:10E480009BCE8090911290909212A0909312B09097
:10E4900094126091670170916801072E000C880B3F
:10E4A000990B0E940DE89B01AC01C501B4010E94CB
:10E4B000C4F01816CCF46091690170916A01072EBE
:10E4C000000C880B990B0E940DE89B01AC01C50163
:10E4D000B4010E9407E887FF07C00E9412B10E94A2
:10E4E00007F07595679501C060E060939712809181
:10E4F000891290918A12A0918B12B0918C12009780
:10E50000A105B10509F48ACFC81AD90AEA0AFB0A9B
:10E51000F7FC84CF0E9409B10E9407F02091871276
:10E52000309188126217730754F00E945CCE76CF48
:10E5300044EE59E261EF79E280E0C9DE90CF46EC2B
:10E5400059E265ED79E280E0C2DE68CFCF92DF92DA
:10E55000EF92FF92CF93DF93EC01C880D980EA80DD
:10E56000FB8089E999E20E945E34C701B6010E94EE
:10E570006826CC80DD80EE80FF8087E290E30E94F9
:10E580005E34C701B6010E946826C884D984EA8433
:10E59000FB8483E290E30E945E34C701B6010E94CF
:10E5A00068268AE00E943D34DF91CF91FF90EF9082
:10E5B000DF90CF900895BC0120915306309154060E
:10E5C00040915306509154062417350731F481E0E9
:10E5D0002617370709F080E008959A01F1CF0F93CD
:10E5E0000FB70F9300916E000F930B7F00936E0097
:10E5F00000916F000D7F00936F000F930BB70F9387
:10E600000CB70F921F922F933F934F935F936F938B
:10E610007F938F939F93AF93BF93EF93FF931124B7
:10E62000E1D4FF91EF91BF91AF919F918F917F9135
:10E630006F915F914F913F912F911F900F900CBF61
:10E640000F910BBF0F910260F89400936F000F9130
:10E6500000936E000F910FBF0F91189500C000C07E
:10E660008091E70680FF1FC0459A8FEF80930C06CC
:10E670008091E70681FF1AC0479A8FEF80930D06BD
:10E680008091E70682FF15C02A988FEF80930E06CF
:10E690008091E70683FF10C028988FEF80930F06C4
:10E6A00000C000C00895459881E0E0CF479881E020
:10E6B000E5CF2A9A81E0EACF289A81E0EFCF8091D6
:10E6C0007B05982F977F90937B05982F937081E01F
:10E6D00011F080E008955E9A08955E9880917B0520
:10E6E000886080937B050895E82FF0E021E030E01A
:10E6F000082E02C0220F331F0A94E2F720953095AE
:10E7000090917B05922390937B05EC5DFD4F2081DA
:10E71000922321E019F020E0822F0895813079F0D2
:10E7200038F08230C9F7159A90915A079B7F04C040
:10E730005E9A90915A079E7F90935A07EDCF5E9A0A
:10E7400090915A079D7FF8CF80E0CEDF81E0CCDF4B
:10E7500082E0CADFB4CF813079F070F0823071F09E
:10E7600021E030E001C0220F8A95EAF780917B0515
:10E77000822B80937B0508955E98F2CF1598F0CF99
:10E78000B0E0A0E0E6ECF3E70C94F5EECCE4DDE0DD
:10E7900002E717E08CE5A82E8DE0B82EC12CD12C15
:10E7A0007601C39469917991899199910E940BE8BE
:10E7B000288939894A895B890E946CE80E940CF09B
:10E7C000F80161937193819391938F01C616D706D7
:10E7D000E806F90610F46B017C01AC16BD0611F7D2
:10E7E0006FEF7FEFCB01A70196010E9435EE2093DA
:10E7F0008207309383074093840750938507CDB7F2
:10E80000DEB7EAE00C9411EF0F931F93CF93DF93E1
:10E8100000E61DE0CBE8D7E0F8012191319141916C
:10E8200051918F0160E070E080E89FE30E949FEFCC
:10E830006993799389939993F7E0CB39DF0761F76F
:10E840000E942AC49DDFDF91CF911F910F910895FF
:10E85000DBCFDACFD9CFD8CF9091391380913A134B
:10E86000981306C08091940D9091950D892B21F0FD
:10E8700080E00E940B41F0CF089590913913809170
:10E880003A13981307C08091940D9091950D892BA0
:10E8900009F45ACF80E00E940B41EFCFCF92DF9274
:10E8A000EF92FF92CF93DF9320919904222319F1E5
:10E8B000EC0108960E94CF276B017C0120E030E03C
:10E8C000A9010E9407E820E030E0A901882349F06F
:10E8D000CE010E944728A70196010E946CE89B0187
:10E8E000AC01688579858A859B850E9424EF6887BD
:10E8F00079878A879B87DF91CF91FF90EF90DF9098
:10E90000CF900895CF92DF92EF92FF92CF93DF9353
:10E9100020919904222319F1EC0108960E94CF2737
:10E920006B017C0120E030E0A9010E9407E820E0B3
:10E9300030E0A901882349F0CE010E944728A701B1
:10E9400096010E946CE89B01AC01688579858A85F7
:10E950009B850E9425EF688779878A879B87DF914F
:10E96000CF91FF90EF90DF90CF900895AEE1B0E0AF
:10E97000ECEBF4E70C94EFEE9E8F8D8F5B018A0138
:10E98000FC01EA5BFF4F2081318142815381298B59
:10E990003A8B4B8B5C8BCA01B9010E940BE86B016F
:10E9A0007C01D5012D913D914D915C910E946CE8C7
:10E9B0000E9489EF2B013C01F801208131814281C5
:10E9C0005381C701B6010E946CE80E9489EF4B0198
:10E9D0005C01C301B2010E940CF06D8B7E8B8F8BAA
:10E9E000988F683771058105910540F428E730E07C
:10E9F00040E050E02D8B3E8B4F8B588FC501B4010A
:10EA00000E940CF0698F7A8F8B8F9C8F683771050D
:10EA10008105910540F488E790E0A0E0B0E0898F9F
:10EA20009A8FAB8FBC8FED8DFE8DEE5AFF4F2081FC
:10EA300031814281538129873A874B875C87CA019C
:10EA4000B9010E940DE82B013C016D897E898F89F7
:10EA5000988D0E940BE86D837E838F83988720E0DA
:10EA600030E0A901C301B2010E9407E8882309F43C
:10EA7000BBC1A7019601C701B6010E946CE84B011A
:10EA80005C012D813E814F815885CA01B9010E94E8
:10EA90006CE89B01AC01C501B4010E9424EF4B015D
:10EAA0005C01A3019201C301B2010E9425EF9B0109
:10EAB000AC01C501B4010E949FEF0E9489EF0E9442
:10EAC0000CF069837A838B839C8369857A858B8537
:10EAD0009C8590958095709561957F4F8F4F9F4F46
:10EAE0000E940DE84B015C01698D7A8D8B8D9C8DA8
:10EAF0000E940BE869877A878B879C8720E030E04B
:10EB0000A901C501B4010E9407E8882309F470C176
:10EB100029853A854B855C85CA01B9010E946CE85C
:10EB20006D877E878F87988BA7019601C701B601F5
:10EB30000E946CE89B01AC016D857E858F8598896C
:10EB40000E9424EF6B017C01A5019401C501B40171
:10EB50000E9425EF9B01AC01C701B6010E949FEF07
:10EB60000E9438F0AD8DBE8D95962D913D914D91C1
:10EB70005C9198972D873E874F87588B69017A0162
:10EB800029813A814B815C81C21AD30AE40AF50AD1
:10EB90000E940CF0C61AD70AE80AF90AF7FE8CC0E0
:10EBA0002D813E814F815885CA01B9010E946CE8D0
:10EBB0006B017C0120E030E0A901C301B2010E9499
:10EBC00007E8882309F418C16D857E858F859889AB
:10EBD0000E940BE89B01AC010E9425EFA30192016A
:10EBE0000E946CE84B015C0129853A854B855C8568
:10EBF000CA01B9010E946CE89B01AC01C501B401D6
:10EC00000E9425EFA70196010E9424EF4B015C01B1
:10EC100020E030E040E850E4C301B2010E946CE81B
:10EC20009B01AC01C501B4010E949FEF0E9489EFD6
:10EC30004B015C0120E030E0A9010E94C4F087FF95
:10EC400003C0812C912C5401C501B4010E940CF029
:10EC500069837A838B839C832D853E854F85588974
:10EC6000261737074807590720F429833A834B832F
:10EC70005C8369817A818B819C810E940BE84B01C6
:10EC80005C01A3019201C301B2010E9425EF9B0127
:10EC9000AC01C501B4010E946CE8A70196010E9475
:10ECA00025EF0E9403F10E940CF0698B7A8B8B8B0D
:10ECB0009C8BC12CD12C760169897A898B899C899E
:10ECC0002D893E894F89588D621B730B840B950BE0
:10ECD0000E940BE8A30192010E949FEF20E034E222
:10ECE00044EF59E40E946CE80E940CF04B015C0177
:10ECF00069897A898B899C89298D3A8D4B8D5C8DA8
:10ED0000621B730B840B950B0E940BE8A30192010D
:10ED10000E949FEF20E034E244EF59E40E946CE847
:10ED20000E940CF06D837E838F839887C501B401A8
:10ED30000E94D4632B013C016D817E818F81988577
:10ED40000E94D46329813A814B815C81AD8DBE8D57
:10ED500099962D933D934D935C939C9789019A01CD
:10ED60000C0D1D1D2E1D3F1DFD0105A716A727A774
:10ED700030ABE65BFF4F2D893E894F89588D20834C
:10ED8000318342835383D5968D929D92AD92BC92EE
:10ED9000D8972D813E814F815885D9962D933D93EB
:10EDA0004D935C93DC973D974082518262827382DF
:10EDB0003496608371838283938329893A894B894E
:10EDC0005C89D1962D933D934D935C93D4973D965A
:10EDD000298D3A8D4B8D5C8D208331834283538303
:10EDE0006E96E0E10C940BEF60E070E0CB0165CE35
:10EDF00060E070E0CB01B4CE60E070E0CB0116CFF4
:10EE000090916F0081E091FD02C080E008959091A3
:10EE10006F009D7F90936F000895EFE6F0E0808192
:10EE2000826080830895CF93C82FEADF94E0C99F62
:10EE300090011124F901EA5AF94F2E59394FD9019D
:10EE40004D915D916D917C91408351836283738379
:10EE500091E0909355068111E0DFCF910895CF9313
:10EE6000DF938091E606811105C08091E806882332
:10EE700009F44EC08091E705329B4DC081608093BC
:10EE8000E7058091E705339B48C082608093E705E2
:10EE90008091E705349B43C084608093E705C0916F
:10EEA0004606C0FF0FC08091E70680FF0BC080912F
:10EEB000E70580FF07C080912C07816080932C07B5
:10EEC00080E0B1DFC1FF0FC08091E70681FF0BC07A
:10EED0008091E70581FF07C080912C0782608093B5
:10EEE0002C0781E0A0DFC2FF13C08091E70682FFFC
:10EEF0000FC08091E806882359F08091E70582FFD2
:10EF000007C080912C07846080932C0782E08BDF00
:10EF1000DF91CF9108958E7FB2CF8D7FB7CF8B7F5A
:10EF2000BCCF6EDF10928607109287071092880779
:10EF300010928907811171CF08950F931F938091CB
:10EF4000391390913A13891B8F7009F449C090913D
:10EF50003613992361F0833040F48FEF890F29F045
:10EF60008093361390E080E038C010923613809181
:10EF70003A132BE5829FC00111248556984FFC015E
:10EF8000208120FDEFCF4091860750918707609147
:10EF9000880770918907E95AFF4F0081118122810A
:10EFA0003381401B510B620B730B409386075093C8
:10EFB0008707609388077093890720913A132F5F22
:10EFC0002F702093371330913A1320913813321356
:10EFD00004C020913713209338131F910F91089587
:10EFE000A0DFC0CFA3E1B0E0E8EFF7E70C94EDEECF
:10EFF0008FEF9FEF90938900809388002AE0298308
:10F00000312C212C789480914F0690915006A0913C
:10F010005106B0915206892B8A2B8B2B09F0C2C165
:10F02000809155068823D1F0809153069091540623
:10F0300010925506892B91F01092540610925306A7
:10F04000109246069091391380913A13981731F037
:10F0500080913A138F5F8F7080933A13809153069B
:10F0600090915406892B09F49DC140914B06509113
:10F070004C0660914D0670914E0680914706909126
:10F080004806A0914906B0914A0600913D0610E05D
:10F0900030E020E0841B950BA60BB70B081719076F
:10F0A0002A073B0710F4D901C8018A8B840F951FEA
:10F0B000A61FB71F80934B0690934C06A0934D0656
:10F0C000B0934E06E1E0C0901406D0901506E09093
:10F0D0001606F09017068091240690912506A091BF
:10F0E0002606B0912706C80ED91EEA1EFB1EC09246
:10F0F0002406D0922506E0922606F0922706F7FC19
:10F1000033C040910C06042E000C550B660B770B98
:10F110008091620690916306A0916406B0916506A5
:10F12000840F951FA61FB71F8093620690936306F6
:10F13000A0936406B0936506809110069091110625
:10F14000A0911206B0911306B701A601481B590BF6
:10F150006A0B7B0BDB01CA01809324069093250682
:10F16000A0932606B0932706009118061091190661
:10F1700020911A0630911B0680912806909129064D
:10F18000A0912A06B0912B06080F191F2A1F3B1FBA
:10F19000009328061093290620932A0630932B0605
:10F1A00037FD33C040910D06042E000C550B660B45
:10F1B000770B8091660690916706A0916806B091E2
:10F1C0006906840F951FA61FB71F8093660690934C
:10F1D0006706A0936806B093690680911006909127
:10F1E0001106A0911206B091130628013901481AA0
:10F1F000590A6A0A7B0AD301C201809328069093B8
:10F200002906A0932A06B0932B0640911C06509124
:10F210001D0660911E0670911F0680912C0690912C
:10F220002D06A0912E06B0912F06480F591F6A1F78
:10F230007B1F40932C0650932D0660932E067093EF
:10F240002F0677FD33C080900E06082C000C99081D
:10F25000AA08BB0880916A0690916B06A0916C0683
:10F26000B0916D06880D991DAA1DBB1D80936A067D
:10F2700090936B06A0936C06B0936D068091100678
:10F2800090911106A0911206B09113063A014B011C
:10F29000681A790A8A0A9B0AD401C30180932C0652
:10F2A00090932D06A0932E06B0932F0680902006F3
:10F2B00090902106A0902206B090230680913006FF
:10F2C00090913106A0913206B0913306880D991DB8
:10F2D000AA1DBB1D8093300690933106A093320681
:10F2E000B0933306B7FD33C040900F06042C000CDA
:10F2F00055086608770880906E0690906F06A0907B
:10F300007006B0907106840C951CA61CB71C8092E8
:10F310006E0690926F06A0927006B0927106809071
:10F32000100690901106A0901206B09013062C01C2
:10F330003D01481859086A087B0853014201809230
:10F34000300690923106A0923206B0923306E11157
:10F3500004C0E0918400F0918500F7FE5F9A37FFCA
:10F36000469A77FF2B9AB7FF299AE0918400F09193
:10F370008500E0918400F0918500F7FE5F9837FFEB
:10F38000469877FF2B98B7FF29985A88552021F087
:10F3900080918400909185002A8921502A8BE0E099
:10F3A000211191CE80914F0690915006A091510667
:10F3B000B0915206892B8A2B8B2B09F01AC74090EB
:10F3C0005306509054065B8A4A8A4114510409F44A
:10F3D0006CC780914B0690914C06A0914D06B09160
:10F3E0004E0640914706509148066091490670913B
:10F3F0004A0684179507A607B70708F4B3C080919B
:10F400005B01882309F465C0F20185899689A78983
:10F41000B08D892B8A2B8B2B81F4818D928DA38DBE
:10F42000B48D892B8A2B8B2B41F4858D968DA78DDE
:10F43000B0A1892B8A2B8B2BB1F1AA89BB8991961C
:10F440006D917D918D919C91949780908005909085
:10F450008105A0908205B0908305AB5BBF4F2C91D6
:10F4600023FF07C090958095709561957F4F8F4FD2
:10F470009F4F0E940DE82091970730919807409187
:10F48000990750919A070E946CE89B01AC01C50155
:10F49000B4010E9424EF60938005709381058093EE
:10F4A0008205909383058091840580FF10C0809130
:10F4B000570190915801A0915901B0915A01809340
:10F4C000800590938105A0938205B09383051092E7
:10F4D000840510925406109253061092460690919D
:10F4E000391380913A13981709F4DFC680913A13C3
:10F4F0008F5F8F7080933A13A0EDCA2EA7E0DA2EAB
:10F50000E12CF12C8091530690915406892B09F03F
:10F5100068C613DD9093540680935306892B09F433
:10F5200060C640905306509054065B8A4A8AD201C6
:10F530008C9183FF08C5C20145960E9473631092A7
:10F5400054061092530610924606909139138091FA
:10F550003A139817F1F280913A138F5F8F7080936E
:10F560003A13D7CF4091420650914306609144062A
:10F5700070914506481759076A077B0708F40FC2C0
:10F5800040913E0650913F066091400670914106C1
:10F59000EA89FB8985A996A9A7A9B0AD481759079B
:10F5A0006A077B0708F0D0C1411551056105710557
:10F5B00009F066C08090850590908605A09087052B
:10F5C000B090880589E799E2A1E0FC0105911591C9
:10F5D00025913491081519052A053B0558F4B69470
:10F5E000A79497948794AA0F0496E5E9F9E2E8179F
:10F5F000F90759F7A0933D06F0E28F169104A10494
:10F60000B10428F4E0E28E2E912CA12CB12C20E242
:10F61000821A9108A108B108811438E09306A10468
:10F62000B10408F49AC1A4E09A9EC001112487583D
:10F630009A4DFC01329625913491B82DEE27B39F57
:10F640008001B29F010D1E1F06940E1F1E1F112464
:10F6500030E020E0FC01C590D490F12CE12CC01AE0
:10F66000D10AE20AF30A4C0D5D1D6E1D7F1D409309
:10F670003E0650933F06609340067093410642CF8A
:10F6800000E01A81942F852E862FBC81AD81FE81EA
:10F69000EF81388529854B80E0917C05E99FA12D7C
:10F6A000FF2730917D05399FA00DF11D10907E053B
:10F6B000199EF00DE89DA00DF11D389DF00DE89FFD
:10F6C000F00D4A2EBF2F4A9EE12D332722274F9E51
:10F6D000E00D311D201FBA9FE00D311D201FBF9F7F
:10F6E000300D211D432EB22F4A9E112D3327222784
:10F6F0004F9E100D311D201FBA9F100D311D201F70
:10F70000BF9F300D211D432EB22FEE27909185050E
:10F7100080908605809187050090A402002A09F454
:10F7200083C03091A002349DE119900B800A800BB8
:10F730002091A102249DE0199109800A800B10916B
:10F74000A202149D90198108800B3B9FE01991093A
:10F75000800A800B2B9F90198108800B1B9F8018BB
:10F7600081094A9E112D332722274F9E100D311DEE
:10F77000201FBA9F100D311D201FBF9F300D211D6E
:10F78000432EB22F30919C02349DE10D901F801EBC
:10F79000801F20919D02249DE00D911D801E801FE1
:10F7A00010919E02149D900D811C801F3B9FE00DC7
:10F7B000911D801E801F2B9F900D811C801F1B9F01
:10F7C000800C811D4A9E112D332722274F9E100D3C
:10F7D000311D201FBA9F100D311D201FBF9F300DFE
:10F7E000211D432EB22F30919802349DE119900BC8
:10F7F000800A800B20919902249DE0199109800ACA
:10F80000800B10919A02149D90198108800B3B9FE8
:10F81000E0199109800A800B2B9F90198108800BB9
:10F820001B9F8018810982C03091A002349DE10D98
:10F83000901F801E801F2091A102249DE00D911D2C
:10F84000801E801F1091A202149D900D811C801FAC
:10F850003B9FE00D911D801E801F2B9F900D811CF2
:10F86000801F1B9F800C811D4A9E112D332722274C
:10F870004F9E100D311D201FBA9F100D311D201FEE
:10F88000BF9F300D211D432EB22F30919C02349D1D
:10F89000E119900B800A800B20919D02249DE019B4
:10F8A0009109800A800B10919E02149D9019810885
:10F8B000800B3B9FE0199109800A800B2B9F9019C8
:10F8C0008108800B1B9F801881094A9E112D3327C8
:10F8D00022274F9E100D311D201FBA9F100D311D84
:10F8E000201FBF9F300D211D432EB22F3091980253
:10F8F000349DE10D901F801E801F20919902249D50
:10F90000E00D911D801E801F10919A02149D900D94
:10F91000811C801F3B9FE00D911D801E801F2B9F2F
:10F92000900D811C801F1B9F800C811D11244B8218
:10F930001A83BC83AD83FE83EF8338872987982C95
:10F94000892EB12CA82E3ECEAA89BB89D1968D9046
:10F950009D90AD90BC90D49735CED501C401B6959D
:10F96000A795979587958C7F87589E4DFC01C590EC
:10F97000D490FC01329625913491E82DE7708E2EBB
:10F98000E29FC001E39F900D112433E09695879587
:10F990003A95E1F7C81AD90AF12CE12C64CE4091CE
:10F9A000390650913A0660913B0670913C06481723
:10F9B00059076A077B0708F030C2809034069090A0
:10F9C0003506A0903606B090370680913806EA8951
:10F9D000FB8981117CC0EF5BFF4FE080F1800281E9
:10F9E0001381EA89FB89E25BFF4F208131814281EB
:10F9F0005381AA89BB89D1966D917D918D919C91FE
:10FA0000D4970E947C63B1E0B0933806EA89FB8901
:10FA100041A952A963A974A989E799E2A1E0FC016F
:10FA2000059115912591349104171507260737077D
:10FA300058F47695679557954795AA0F0496E5E98A
:10FA4000F9E2E817F90759F7A0933D06403251054E
:10FA50006105710520F440E250E060E070E0405242
:10FA60005109610971094115F8E05F0761057105E8
:10FA700008F4B3C124E0529FC001112487589A4D65
:10FA8000FC01329625913491AA27439FF001429FB1
:10FA9000E10DFA1F0694EA1FFA1F1124AF0170E06E
:10FAA00060E0FC01C590D490F12CE12CC41AD50A79
:10FAB000E60AF70A8C0C9D1CAE1CBF1C8092340613
:10FAC00090923506A0923606B09237061BCD81ADD6
:10FAD00092ADA3ADB4AD88169906AA06BB0608F090
:10FAE00072C181149104A104B10449F440918505C7
:10FAF0005091860560918705709188058DCFA0E0B3
:10FB0000FA85982D492D8A2DEB857C856D85BE85DE
:10FB10005F853889298950917C05599F612DBB27C4
:10FB200030917D05399F600DB11D10907E05199EA5
:10FB3000B00D549F600DB11D349FB00D589FB00D96
:10FB4000E62F7B2FE69F512D33272227EB9F500D69
:10FB5000311D2A1F769F500D311D2A1F7B9F300DAE
:10FB6000211DE32F722FE69FF12D33272227EB9FD4
:10FB7000F00D311D2A1F769FF00D311D2A1F7B9F2E
:10FB8000300D211DE32F722F55279091850540914F
:10FB90008605809187050090A4020A2A09F483C093
:10FBA0003091A0023E9F51199A0B4A0B8A0B20916B
:10FBB000A1022E9F501991094A0B8A0BF091A202C3
:10FBC000FE9F901941098A0B379F501991094A0BE2
:10FBD0008A0B279F901941098A0BF79F40198109C9
:10FBE000E69FF12D33272227EB9FF00D311D2A1FB1
:10FBF000769FF00D311D2A1F7B9F300D211DE32FB5
:10FC0000722F30919C023E9F510D9A1F4A1F8A1FEE
:10FC100020919D022E9F500D911D4A1F8A1FF09129
:10FC20009E02FE9F900D411D8A1F379F500D911D12
:10FC30004A1F8A1F279F900D411D8A1FF79F400D65
:10FC4000811DE69FF12D33272227EB9FF00D311DFB
:10FC50002A1F769FF00D311D2A1F7B9F300D211D1D
:10FC6000E32F722F309198023E9F51199A0B4A0B45
:10FC70008A0B209199022E9F501991094A0B8A0BE9
:10FC8000F0919A02FE9F901941098A0B379F5019F3
:10FC900091094A0B8A0B279F901941098A0BF79FFC
:10FCA0004019810982C03091A0023E9F510D9A1FD8
:10FCB0004A1F8A1F2091A1022E9F500D911D4A1F9D
:10FCC0008A1FF091A202FE9F900D411D8A1F379F4F
:10FCD000500D911D4A1F8A1F279F900D411D8A1F9D
:10FCE000F79F400D811DE69FF12D33272227EB9FC3
:10FCF000F00D311D2A1F769FF00D311D2A1F7B9FAD
:10FD0000300D211DE32F722F30919C023E9F51191F
:10FD10009A0B4A0B8A0B20919D022E9F5019910934
:10FD20004A0B8A0BF0919E02FE9F901941098A0BA3
:10FD3000379F501991094A0B8A0B279F9019410947
:10FD40008A0BF79F40198109E69FF12D332722275F
:10FD5000EB9FF00D311D2A1F769FF00D311D2A1FDC
:10FD60007B9F300D211DE32F722F309198023E9F13
:10FD7000510D9A1F4A1F8A1F209199022E9F500DE4
:10FD8000911D4A1F8A1FF0919A02FE9F900D411DFE
:10FD90008A1F379F500D911D4A1F8A1F279F900D64
:10FDA000411D8A1FF79F400D811D1124FA87EB87A3
:10FDB0007C876D87BE875F87388B298B542F492FAF
:10FDC00070E0682F29CE2A893B89225B3F4FD901F9
:10FDD0004D915D916D917C911FCEDB01CA01B6956D
:10FDE000A795979587958C7F87589E4DFC01C59068
:10FDF000D490FC013296259134914770429FC00106
:10FE0000439F900D1124A3E096958795AA95E1F75D
:10FE1000C81AD90AF12CE12C4DCE80915C01909149
:10FE20005D01A0915E01B0915F01B7FF61C0EA89F9
:10FE3000FB89EA5BFF4FC080D180E280F38089E7D5
:10FE400099E221E0FC0145915591659174914C1521
:10FE50005D056E057F0558F4F694E794D794C79432
:10FE6000220F049645E959E24817590759F720939C
:10FE70003D0650E2C516D104E104F10428F470E215
:10FE8000C72ED12CE12CF12C60E2C61AD108E10872
:10FE9000F108C11478E0D706E104F10408F431C098
:10FEA000A4E0DA9EC001112487589A4DFC013296D5
:10FEB00025913491BC2D6627B39FA001B29F410DBF
:10FEC000561F0694461F561F112470E060E0FC0187
:10FED00085919491B0E0A0E0841B950BA60BB70B25
:10FEE00080935C0190935D01A0935E01B0935F01EC
:10FEF000C0905C01D0905D01E0905E01F0905F01E8
:10FF000001CBD701C601B695A795979587958C7FAC
:10FF100087589E4DFC0125913491FC013296459104
:10FF20005491EC2DE770E49FC001E59F900D1124E2
:10FF300063E0969587956A95E1F7281B390BC9010F
:10FF4000B0E0A0E0CDCFEA89FB8985889688A788B4
:10FF5000B08C81E081149104A104B10409F480E023
:10FF6000AA89BB895996CD90DD90ED90FC905C9765
:10FF7000C114D104E104F10409F08260EA89FB892B
:10FF8000458D568D678D70A141155105610571052F
:10FF900009F084608093460610923406109235066C
:10FFA000109236061092370610923E0610923F06C7
:10FFB0001092400610924106EA89FB8985A196A11C
:10FFC000A7A1B0A58093470690934806A093490641
:10FFD000B0934A06442455243201481A590A6A0A41
:10FFE0007B0A409224065092250660922606709263
:10FFF0002706409228065092290660922A0670929F
:020000021000EC
:100000002B0640922C0650922D0660922E0670927E
:100010002F0641A052A063A074A0440C551C661C7E
:10002000771C880C991CAA1CBB1C80921406909209
:100030001506A0921606B0921706CC0CDD1CEE1C1D
:10004000FF1CC0921806D0921906E0921A06F09290
:100050001B06440F551F661F771F40931C065093C5
:100060001D0660931E0670931F0640922006509254
:1000700021066092220670922306880F991FAA1FFC
:10008000BB1F8093100690931106A0931206B093A5
:10009000130610924B0610924C0610924D061092C9
:1000A0004E0681A592A5A3A5B4A580934206909380
:1000B0004306A0934406B093450685A596A5A7A53B
:1000C000B0A98093390690933A06A0933B06B0936B
:1000D0003C06EB5BFF4F80819091E706891721F08A
:1000E0008093E7060E942E730E942F7744244A943F
:1000F000542C320140925C0150925D0160925E018D
:1001000070925F01EA89FB89FD96E080F1800281AF
:100110001381AA89BB89D1962D913D914D915C9116
:10012000D4976D01BAE4CB0ED11CF60160817181C8
:10013000828193810E947C6310923806D6014D9192
:100140005D916D917C9189E799E2A1E0FC010591B7
:10015000159125913491041715072607370758F490
:100160007695679557954795AA0F0496E5E9F9E2C4
:10017000E817F90759F7A0933D064032510561058C
:10018000710520F440E250E060E070E04052510917
:10019000610971094115F8E05F076105710508F40F
:1001A00062C024E0529FC001112487589A4DFC017F
:1001B000329625913491AA27439FF001429FE10D89
:1001C000FA1F0694EA1FFA1F1124AF0170E060E0E5
:1001D000FC01C590D490F12CE12CC41AD50AE60A92
:1001E000F70AC0924F06D0925006E0925106F09264
:1001F000520680914F0690915006A0915106B09101
:100200005206AC01BD01009731E0A307B10520F013
:100210004FEF5FEF60E070E0841B950BA60BB70B10
:1002200080934F0690935006A0935106B0935206C8
:10023000F89480918400909185004096A981A15006
:10024000A983AA2381F1240E351E2816390610F43D
:100250000C940278309289002092880078946396FA
:10026000E2E10C9409EFDB01CA01B695A7959795D9
:1002700087958C7F87589E4DFC01C590D490FC01DA
:100280003296259134914770429FC001439F900D53
:10029000112433E0969587953A95E1F7C81AD90A63
:1002A000F12CE12C9ECF1C01D5CF80EDC82E87E02C
:1002B000D82EE12CF12C2DC9CF93DF9380913913E7
:1002C00090913A13891B80958F7019F40E940B410D
:1002D000F5CF809139138F5F8F70A09139139BE513
:1002E000A99FD0011124FD01E556F84FEF011992A5
:1002F0009A95E9F798E09083A055B84F90E1EBE329
:10030000F3E101900D929A95E1F7209139139091C4
:100310003A13291303C094E690933613809339134C
:100320000E940D77DF91CF910895FC0120813181EA
:100330004281538160916C0D70916D0D80916E0DB5
:1003400090916F0D0E946CE80E94C9F06093471372
:10035000709348138093491390934A1390913913E3
:1003600080913A13981709F0A7CF0E942C740E942D
:100370000077409147135091481360914913709151
:100380004A1340936E0650936F0660937006709305
:10039000710681110C940D7708954F925F926F92C0
:1003A0007F928F929F92AF92BF92CF92DF92EF9205
:1003B000FF92CF93DF93EC0120916C0D30916D0D86
:1003C00040916E0D50916F0D6C857D858E859F855A
:1003D0000E946CE80E94C9F06B017C012091680DBD
:1003E0003091690D40916A0D50916B0D688579854A
:1003F0008A859B850E946CE80E94C9F04B015C01D4
:100400002091640D3091650D4091660D5091670DFE
:100410006C817D818E819F810E946CE80E94C9F071
:100420002B013C012091600D3091610D4091620DD6
:100430005091630D688179818A819B810E946CE86B
:100440000E94C9F060933B1370933C1380933D135B
:1004500090933E1340923F13509240136092411389
:10046000709242138092431390924413A0924513CA
:10047000B0924613C0924713D0924813E0924913AA
:10048000F0924A139091391380913A13981781F0A2
:1004900013DFDF91CF91FF90EF90DF90CF90BF906F
:1004A000AF909F908F907F906F905F904F90089546
:1004B0000E942C740E940077C82F8BE393E10E9466
:1004C0007363CC2331F30E940D77E3CFCF92DF9299
:1004D000EF92FF92CF93DF93C82F0E94007794E0B2
:1004E000C99FE0011124FE01EE59F94FC080D1806F
:1004F000E280F38081110E940D77C557D84FC70164
:10050000B6010E940DE8288139814A815B810E94F1
:100510006CE8DF91CF91FF90EF90DF90CF9008953E
:100520008F929F92AF92BF92CF92DF92EF92FF9203
:100530001F93CF93DF93CDB7DEB760970FB6F894D4
:10054000DEBF0FBECDBF182F80E0C0DF4B015C01C6
:100550008092E8059092E905A092EA05B092EB0539
:1005600081E0B4DF6B017C01C092EC05D092ED0517
:10057000E092EE05F092EF0582E0A8DF6093F005CF
:100580007093F1058093F2059093F3051D861E8606
:100590001F86188A89829A82AB82BC82CD82DE82D3
:1005A000EF82F88669877A878B879C8783E08EDF66
:1005B0006D877E878F87988BCE0101960E944E743F
:1005C0001E3FD9F480E1FE013196A7E7B1E001902A
:1005D0000D928A95E1F760960FB6F894DEBF0FBED4
:1005E000CDBFDF91CF911F91FF90EF90DF90CF9023
:1005F000BF90AF909F908F90089584E0189FF00176
:100600001124DF01A958BE4F81E090E08C0F9D1F9F
:10061000E80FF91F40815181628173814D935D9391
:100620006D937C931397D7CFCF92DF92EF92FF9287
:10063000CF93DF93C82F0E94007794E0C99FE00119
:100640001124FE01EA5AF94FC080D180E280F38084
:1006500081110E940D77C557D84FC701B6010E947E
:100660000DE8288139814A815B810E946CE8DF9125
:10067000CF91FF90EF90DF90CF900895A1E0B0E090
:10068000E4E4F3E80C94FDEE898360E0CE0101968A
:100690000E94CE6461E0CE0101960E94CE6462E0C9
:1006A000CE0101960E94CE6489812196E2E00C94ED
:1006B00019EFA2E1B0E0EFE5F3E80C94F9EEDEDF2C
:1006C0008823C1F1EDB6FEB647E952E082FF02C0D1
:1006D0004EE852E027E932E081FF02C020E932E033
:1006E00080FD25C087E992E05F934F933F932F935E
:1006F0009F938F938AE09EE19F938F938E010F5F6C
:100700001F4F1F930F930E94A0E70E94FC3DC8015A
:100710000E944F34C8010E9493C20FB6F894DEBF06
:100720000FBECDBF81E06296E6E00C9415EF82E942
:1007300092E0DACF80E0F7CFA0E2B0E0E2EAF3E8BF
:100740000C94EDEE80913B01882309F4BEC08091AA
:10075000FA05082F10E080FF3CC0C0903D01D0900A
:100760003E01E0903F01F0904001209189043091DA
:100770008A0440918B0450918C04C701B6010E94F9
:10078000C4F0181644F4C0928904D0928A04E0920E
:100790008B04F0928C04C0904901D0904A01E09003
:1007A0004B01F0904C012091890430918A044091D2
:1007B0008B0450918C04C701B6010E9407E887FFA3
:1007C00008C0C0928904D0928A04E0928B04F0920F
:1007D0008C0401FF3CC0C0904101D0904201E090E8
:1007E0004301F090440120918D0430918E0440919A
:1007F0008F0450919004C701B6010E94C4F01816EE
:1008000044F4C0928D04D0928E04E0928F04F09252
:100810009004C0904D01D0904E01E0904F01F090B7
:10082000500120918D0430918E0440918F0450919D
:100830009004C701B6010E9407E887FF08C0C09274
:100840008D04D0928E04E0928F04F092900402FF07
:100850003CC0C0904501D0904601E0904701F09027
:100860004801209191043091920440919304509159
:100870009404C701B6010E94C4F0181644F4C09253
:100880009104D0929204E0929304F0929404C09068
:100890005101D0905201E0905301F0905401209109
:1008A0009104309192044091930450919404C701B3
:1008B000B6010E9407E887FF08C0C0929104D09259
:1008C0009204E0929304F092940480914B0D83FD86
:1008D00061C0209183013091840140918501509144
:1008E000860160919504709196048091970490918F
:1008F00098040E9407E8882309F44CC00E94E6B3DC
:10090000182F882331F00E94FC3D8FEE9DE10E945C
:100910005E34209183013091840140918501509192
:10092000860160919504709196048091970490914E
:1009300098040E9424EF9F772091710130917201F9
:1009400040917301509174010E946CE820E030E006
:1009500046E154E40E94C4F01816D4F40E94FC3D11
:1009600080ED9DE10E945E34809195049091960403
:10097000A0919704B091980480938301909384018F
:10098000A0938501B093860185E994E0CEDC02C096
:100990001111EACF2AE037ED43E25CE360913501C3
:1009A0007091360180913701909138010E946CE876
:1009B0006B017C016091390170913A01072E000CA6
:1009C000880B990B0E940DE89B01AC01C701B60191
:1009D0000E946CE8698B7A8B8B8B9C8B809199043D
:1009E000882309F180909A0490909B04A0909C0425
:1009F000B0909D04C0909104D0909204E090930434
:100A0000F090940420E030E0A901C501B4010E94F7
:100A100007E88823F9F0A7019601C501B4010E94F7
:100A2000C4F01816BCF020E030E0A901BE016F5EF2
:100A30007F4F89E894E00E9407C480E1E9E8F4E090
:100A4000A7E7B1E001900D928A95E1F7A096E2E167
:100A50000C9409EF20917701309178014091790150
:100A600050917A016091890470918A0480918B047D
:100A700090918C040E9424EF4B015C0120917B013A
:100A800030917C0140917D0150917E0160918D04F7
:100A900070918E0480918F04909190040E9424EFB5
:100AA0006D8B7E8B8F8B988F20917F013091800191
:100AB0004091810150918201C701B6010E9424EF4B
:100AC0006D8F7E8F8F8F98A3209183013091840149
:100AD0004091850150918601609195047091960432
:100AE00080919704909198040E9424EF698F7A8FE7
:100AF0008B8F9C8F20E030E0A901C501B4010E94DA
:100B000007E881110CC020E030E0A9016D897E89E1
:100B10008F89988D0E9407E8882309F484CFA50166
:100B20009401C501B4010E946CE86B017C012D8920
:100B30003E894F89588DCA01B9010E946CE89B011A
:100B4000AC01C701B6010E9425EF6B017C012D8D20
:100B50003E8D4F8D58A1CA01B9010E946CE89B01DE
:100B6000AC01C701B6010E9425EF6B017C01298D04
:100B70003A8D4B8D5C8DCA01B9010E946CE89B01D6
:100B8000AC01C701B6010E9425EF6B017C010E94F8
:100B900003F12B013C012CEC3CEB4CE85BE2C70180
:100BA000B6010E9407E887FF06C0498C5A8C6B8CFF
:100BB0007C8CE89477F82DEB37E346E855E3C301E6
:100BC000B2010E9407E887FD38CF2DEC3CEC4CE4E5
:100BD0005EE3C301B2010E946CE80E940CF01B01AD
:100BE000672B19F422242394312CB10190E080E08A
:100BF0000E940BE89B01AC0160E070E080E89FE39D
:100C00000E949FEF6B017C01AC019B01C301B2010B
:100C10000E946CE82B013C01A7019601C501B401BB
:100C20000E946CE84B015C01A70196016D897E89E9
:100C30008F89988D0E946CE86D8B7E8B8F8B988F3F
:100C4000A70196016D8D7E8D8F8D98A10E946CE815
:100C50006D8F7E8F8F8F98A3A7019601698D7A8DF6
:100C60008B8D9C8D0E946CE8698F7A8F8B8F9C8F07
:100C700080E1E7E7F1E08E010F5F1F4FD80101909F
:100C80000D928A95E1F70E9450CE6B017C0128EC11
:100C9000C20ED11CE11CF11C81E0281A310809F4B4
:100CA00054C00E9450CE9B01AC012C193D094E0945
:100CB0005F0957FD4DC06B017C0128ECC20ED11CB1
:100CC000E11CF11C80E00E940B41A50194016981A7
:100CD0007A818B819C810E9425EF69837A838B8343
:100CE0009C832D893E894F89588D6D817E818F81AE
:100CF00098850E9425EF6D837E838F8398872D8D45
:100D00003E8D4F8D58A169857A858B859C850E9483
:100D100025EF69877A878B879C87298D3A8D4B8D44
:100D20005C8D6D857E858F8598890E9425EF6D8706
:100D30007E878F87988BA3019201BE016F5E7F4FE4
:100D4000C8010E9407C48111A7CFA30192016ECEF2
:100D50000E94E171BACF8091F6059091F705A091BC
:100D6000F805B091F9058093350190933601A09371
:100D70003701B09338018091F4059091F505909377
:100D80003A0180933901089580913501909136019F
:100D9000A0913701B09138018093F6059093F70543
:100DA000A093F805B093F9058091390190913A012B
:100DB0009093F5058093F40584E690E090933A01D2
:100DC000809339010895ACE0B0E0E9EEF6E80C94C8
:100DD000EFEE2B013C0129873A874B875C8747015F
:100DE0005801D601CD90DD90ED90FC9020E030E0F0
:100DF000A901C701B6010E9407E8811171C0809165
:100E00006D0190916E01A0916F01B0917001898385
:100E10009A83AB83BC8320E030E0A901C701B6010F
:100E20000E9407E8811106C0C12CD12C80E8E82E71
:100E300080E4F82ECD82DE82EF82F886A50194014F
:100E400060917F0170918001809181019091820178
:100E50000E9407E887FF0CC080927F01909280017A
:100E6000A0928101B0928201CE0105960E94E06BB2
:100E700040927701509278016092790170927A01E4
:100E800089859A85AB85BC8580937B0190937C0195
:100E9000A0937D01B0937E01CE0101960E94E06B8C
:100EA000A501940160917F01709180018091810181
:100EB000909182010E94C4F0181664F480927F0120
:100EC00090928001A0928101B0928201CE0105969C
:100ED0000E94E06B0E942C742C96E0E10C940BEFC6
:100EE000D701C60194CFCF92DF92EF92FF920F937A
:100EF0001F936B01FC01E080F18002811381E7E721
:100F0000F1E0248135814681578160817181828140
:100F1000938159DF1F910F91FF90EF90DF90CF9059
:100F200008950C942AC40F931F93CF93DF93EC0181
:100F30008B010E94D33F882331F081E0DF91CF9174
:100F40001F910F910895B801CE01CDDF80912C073C
:100F5000C82FC47082FD0AC010922C0782E0E0DA2C
:100F6000E0DF81E0CC2351F380E0E8CF0E94923FA4
:100F7000882391F3E2CFCF930E940077C82F80910E
:100F80003A1380933913809338138093371384E690
:100F9000809336130E94917780ED93E09093950DA6
:100FA0008093940DC1110E940D7781E080935506C6
:100FB0000E942C748EEFB4DAB4DFCF910895ACE0C8
:100FC000B0E0E5EEF7E80C94FDEE0E94A5B30E94B8
:100FD00000779CE0E2E6F6E0DE01119601900D92CA
:100FE0009A95E1F781110E940D77CE0101960E943A
:100FF000A6722C96E2E00C9419EFB0E0A0E0E3E0DA
:10100000F8E80C94EFEE40907701509078016090F2
:10101000790170907A0180907B0190907C01A09082
:101020007D01B0907E01C0907F01D0908001E09062
:101030008101F09082010E94C0736091550170910E
:101040005601072E000C880B990B0E940DE82AE030
:1010500037ED43E25CE30E946CE8609371017093AA
:10106000720180937301909374010DE311E0D0E05D
:10107000C0E0CE01835D9E4D0E94C627F8016193BA
:101080007193819391938F01CE018F5D9E4D0E944C
:10109000C627F80160877187828793872496CC30B2
:1010A000D10539F760E088E096E00E94AA2A0E9404
:1010B000772B0E940474A3019201609177017091D3
:1010C00078018091790190917A010E9407E881115D
:1010D0001BC0A501940160917B0170917C018091FE
:1010E0007D0190917E010E9407E881110DC0209141
:1010F0007F01309180014091810150918201C701AF
:10110000B6010E9407E881115ADFCDB7DEB7E0E1F2
:101110000C940BEFA4E0B0E0E0E9F8E80C94FDEEED
:1011200084EF91E0A0E0B0E089839A83AB83BC8335
:10113000BE016F5F7F4F8CE30E94053386EB9DE11C
:101140000E945E3486B160EB7DE182FB882780F9E6
:101150000E946E6B86B16AEA7DE183FB882780F985
:101160000E946E6B86B164EA7DE1829581700E9477
:101170006E6B80B16BE97DE182FB882780F90E946C
:101180006E6B349907C00E9439332496E2E00C94C8
:1011900019EF06C00E9422332496E2E00C9419EF66
:1011A0008091E606811103C08091E80681110C94BC
:1011B0002F770895ACE0B0E0E0EEF8E80C94FDEE97
:1011C000ACE4BDE090E080E0FC01E759FE4D4591C4
:1011D0005591659174914D935D936D937D93FC0151
:1011E000E75AFE4D459155916591749150964D93F6
:1011F0005D936D937C935397FC01E75BFE4D4591A6
:1012000055916591749190964D935D936D937C93F8
:101210009397049680319105B9F680E29EE4A0E0B0
:10122000B0E080935C0D90935D0DA0935E0DB09344
:101230005F0D80E090E0AAEFB3E48093800D90937F
:10124000810DA093820DB093830D8093840D9093B4
:10125000850DA093860DB093870D8093880D909394
:10126000890DA0938A0DB0938B0D10928C0D109266
:101270008D0D10928E0D10928F0D1092900D109278
:10128000910D1092920D1092930D8AE097EDA3EAC2
:10129000BDE380936E0790936F07A0937007B093A0
:1012A000710710925B010E941E1A80E090E0A0EE90
:1012B000B0E48093570190935801A0935901B093E3
:1012C0005A0180E090E0A0E2B1E480930806909398
:1012D0000906A0930A06B0930B060E94602A8CE0D0
:1012E000E3EBF1E0DE01119601900D928A95E1F7B2
:1012F00089819A81AB81BC818093281390932913B3
:10130000A0932A13B0932B138D819E81AF81B88552
:1013100080932C1390932D13A0932E13B0932F131F
:1013200089859A85AB85BC85809330139093311362
:10133000A0933213B09333138EEB90E09093730528
:1013400080937205109275051092740586EE90E0F8
:101350009093770580937605109279051092780521
:101360008FE892ECADE8B1E48093981290939912D3
:10137000A0939A12B0939B128CE998EFA5E4BEE378
:1013800080939C1290939D12A0939E12B0939F12F3
:1013900081E49CEBABECB3E48093A0129093A11298
:1013A000A093A212B093A3121092E6061092E50643
:1013B000F7DE23DE2C96E2E00C9419EFFBCEA4E0DE
:1013C000B0E0E5EEF9E80C94EEEE9091E80698179F
:1013D00009F455C0382E80E090E0A0E2B1E48983A2
:1013E0009A83AB83BC83C0903013D0903113E090CC
:1013F0003213F090331320E030E0A901C701B601A9
:101400000E9407E887FF0CC0A701960160E070E02A
:1014100080E291E40E9424EF69837A838B839C832A
:10142000CE0101960E94BBC4409077015090780194
:101430006090790170907A0180907B0190907C019E
:10144000A0907D01B0907E013320F1F00E94D33F47
:1014500019821A821B821C82E0907F01F090800129
:101460000091810110918201CE0101966C01A501CC
:101470009401C301B201A7DC3092E80691DE80E05E
:101480002496E1E10C940AEF0E94923FE1CFB0E094
:10149000A0E0EDE4FAE80C94EFEEC82FE82EF12C72
:1014A000F701E352F14DD491823071F481E087DF8E
:1014B000811105C00E94D33F882309F4E2C0CDB753
:1014C000DEB7E0E10C940BEF6D2FDD0F770B880B8F
:1014D000990B0E940DE82B013C01C701880F991F51
:1014E000880F991F875A914E0E94C6274B015C01B5
:1014F000A3019201C501B4010E946CE84B015C019B
:101500006701CC0CDD1CCC0CDD1CC601835B914E4D
:101510000E94C627A30192010E946CE820E030E0FF
:1015200040EC5FE30E946CE8AB01BC0100E010E01E
:1015300098018C2F0E9411C8C23009F0CCC00E94C3
:10154000923F20E030E0A901C501B4010E9407E804
:10155000882329F100E010E020E830E4B501A4017F
:1015600070588C2F0E9411C8C23009F467C0A501C1
:101570009401C501B4010E9425EF4B015C01C2300A
:1015800009F062C000E010E020E030E4B501A40101
:101590008C2F0E9411C8C23011F40E94923F81E04A
:1015A00090E00C2E01C0880F0A94EAF790915A0738
:1015B000982B90935A079091FA05892B8093FA05FE
:1015C000C6018F5B914E0E94C627F601E958FE4F77
:1015D0006083718382839383C230D1F4209130136E
:1015E00030913113409132135091331360917F0148
:1015F0007091800180918101909182010E9424EF7D
:1016000060937F01709380018093810190938201A8
:1016100088DCF601E757FB4FD601A958BE4F8D91E4
:101620009D910D90BC91A02D80839183A283B38363
:10163000C23009F044CF0E94CC2741CF0E94D33F53
:10164000882309F494CF3BCFF701E25CF14E64911B
:10165000611107C00E94FC3D8CE19EE10E945E3456
:101660006AE070E090E080E00E940BE89B01AC0132
:1016700061E070E088E492E40E949FEF8B019C019E
:1016800085CF81E69EE10E94C62720E030E0A901D7
:101690000E9407E8882309F417CF6D2FDD0F770B21
:1016A000880B990B0E940DE82B013C0181E69EE11D
:1016B0000E94C6274B015C0120E030E040EA50E484
:1016C0000E94C4F087FF14CF812C912C90EAA92EA0
:1016D00090E4B92E0DCF20E030E0A901C501B4019E
:1016E0000E9407E8882309F45ACF00E010E098012F
:1016F00035CF80912C07882319F010922C0708957C
:1017000040E070E060E08BE79DE10E941A401F928C
:101710000F920FB60F9211240BB60F922F933F9397
:101720004F935F936F937F938F939F93AF93BF93E9
:10173000EF93FF930E942F77FF91EF91BF91AF91AD
:101740009F918F917F916F915F914F913F912F91D9
:101750000F900BBE0F900FBE0F901F9018950F9318
:101760001F9380916A07813019F50E9450CE009135
:10177000DF051091E0052091E1053091E205601B45
:10178000710B820B930B28EE33E040E050E00E9497
:1017900035EE6091DB057091DC058091DD0590915F
:1017A000DE05620F731F841F951F1F910F9108950F
:1017B0006091E3057091E4058091E5059091E6055F
:1017C000D6CF10926A071092DF051092E0051092B2
:1017D000E1051092E2051092E3051092E4051092E3
:1017E000E5051092E6051092DB051092DC051092DB
:1017F000DD051092DE05089580916A078130E1F0E1
:101800008230C1F4ACDF6093DB057093DC0580931C
:10181000DD059093DE0581E080936A070E9450CE3B
:101820006093DF057093E0058093E1059093E205F6
:1018300081E00895C6DFEFCF80E008950E9409C5DA
:101840000E94112C882351F08091A31482FD06C0C0
:101850008BED98E19093EB068093EA06CDCF8091D3
:101860006A07813079F482E080936A070E9450CE43
:101870006093E3057093E4058093E5059093E60596
:1018800081E0089580E0089580916A078150823058
:1018900070F410926A070E9450CE6093E305709333
:1018A000E4058093E5059093E60581E0089580E0E6
:1018B00008959C0197FF26C0EE27FF27E81BF90B30
:1018C0002D398FEF38070CF05DC08DE280938404D2
:1018D000CF0164E670E00E94BFEECB012AE030E069
:1018E000B9010E94BFEE805D80938504CF01B901EC
:1018F0000E94BFEECB01B9010E94BFEE805D8093D4
:1019000086042AC0283E83E03807B4F1C90168EE96
:1019100073E00E94BFEECB01EAE0F0E0BF010E945D
:10192000BFEE805D80938404C90164E670E00E948C
:10193000BFEECB01BF010E94BFEE805D80938504A6
:10194000C901BF010E94BFEECB01BF010E94BFEEE3
:10195000805D80938604F901CF016AE070E00E9407
:10196000BFEE805D8093870484E894E008958DE263
:1019700037FDC5CF80E2C3CFF90180E224363105BF
:101980000CF0A4CF80E28093840480938504EA3035
:10199000F1056CF38DE237FF80E280938504CF017F
:1019A0006AE070E00E94BFEE605D60938604D4CF71
:1019B0009C0197FD2DC080E2243631055CF0C90101
:1019C00064E670E00E94BFEECB016AE070E00E9426
:1019D000BFEE805D8093850480E22A3031055CF0A3
:1019E000EAE0F0E0C901BF010E94BFEECB01BF01F8
:1019F0000E94BFEE805D80938604C9016AE070E0BA
:101A00000E94BFEE805D8093870485E894E008958E
:101A10003195219531098DE2DDCFCF92DF92EF92A2
:101A2000FF92FC01C080D180E280F38020E030E0B2
:101A3000A901C701B6010E9407E887FD26C06DEB2A
:101A400077E386E095E3A70196010E9425EF6B01FD
:101A50007C0120E030E0A9010E9407E820E030E0AE
:101A600040E05FE387FF04C020E030E040E05FEB50
:101A7000C701B6010E9425EF0E9407F0CB0198DF55
:101A8000FF90EF90DF90CF9008956DEB77E386E0C5
:101A900095EBD9CFA4E0B0E0E0E5FDE80C94FDEED5
:101AA0000E940DE869837A838B839C83CE01019623
:101AB000B4DF2496E2E00C9419EFFC01608171819F
:101AC000828193810E9407F0CB0172CFA4E0B0E045
:101AD000ECE6FDE80C94FDEE0E940DE869837A8344
:101AE0008B839C83CE010196E8DF2496E2E00C9480
:101AF00019EF8F929F92AF92BF92EF92FF920F9346
:101B00001F93CF93DF93EC018B01E42EF22E809193
:101B10004B1390914C138C179D07C9F129EAC632DB
:101B2000D20709F03FC08F519C4271F40E9450CE01
:101B30006E517B4F8F4F9F4F6093CB057093CC05B9
:101B40008093CD059093CE05D0934C13C0934B1347
:101B500030E020E000934D0710934E0720934F078D
:101B600030935007E0924807F0924907CF51DC428A
:101B700021F4109280041092CA0582E080936C01D7
:101B800081E080934A0710927F041092D605DF917E
:101B9000CF911F910F91FF90EF90BF90AF909F90CA
:101BA0008F9008952CE2CF31D20771F68652994A70
:101BB000D9F40E9450CE8090CB059090CC05A09097
:101BC000CD05B090CE05681979098A099B0997FF60
:101BD0000BC080915A078770873031F40E94A86C3F
:101BE000CEEDDDE98111B0CFCFE1DCE2ADCF20E079
:101BF00040E070E060E087E99CE67BCF0E94E6B3BE
:101C0000882339F020E040E070E060E080E09DE96A
